:020000040100F9
:10000000880D00211121000143410001E52000017C
:10001000E5200001E5200001E520000100000000CE
:10002000000000000000000000000000551C00015E
:10003000E520000100000000E5200001E5200001AE
:10004000B11C0001B11C0001B11C0001B11C000178
:10005000B11C0001B11C0001B11C0001B11C000168
:10006000B11C0001B11C0001B11C0001B11C000158
:10007000B11C0001B11C0001B11C0001B11C000148
:10008000B11C0001B11C0001B11C0001B11C000138
:10009000B11C0001B11C0001B11C0001B11C000128
:1000A000B11C0001B11C0001B11C0001B11C000118
:1000B000B11C0001B11C00010000000000000000A4
:1000C0000000000000000000000000000000000030
:1000D0000000000000000000000000000000000020
:1000E0000000000000000000000000000000000010
:1000F0000000000000000000000000000000000000
:1001000000000000000000000000000000000000EF
:1001100000000000000000000000000000000000DF
:1001200000000000000000000000000000000000CF
:1001300000000000000000000000000000000000BF
:1001400000000000000000000000000000000000AF
:10015000000000000000000000000000000000009F
:10016000000000000000000000000000000000008F
:10017000000000000000000000000000000000007F
:10018000000000000000000000000000000000006F
:10019000000000000000000000000000000000005F
:1001A000000000000000000000000000000000004F
:1001B000000000000000000000000000000000003F
:1001C000000000000000000000000000000000002F
:1001D000000000000000000000000000000000001F
:1001E000000000000000000000000000000000000F
:1001F00000000000000000000000000000000000FF
:10020000DEE61E284CBBCE8F023500003C0000000D
:10021000665A00000100000000000001000000011B
:10022000FFFF02910000000000000000000000003D
:10023000000000000000000000000000FFFFFFFFC2
:1002400053B94AB9002908BF00281CBF4FF0FF313D
:100250004FF0FF3000F00CB8ADF1080C6DE904CEA2
:1002600000F0D0F9DDF804E0DDE9022304B07047C6
:10027000704700BF30B44FF0000310F8014B11F885
:10028000015B013A84EA050443EA0403F5D1A3F1D2
:1002900001034FEAD37030BC704700BF4FF000033A
:1002A00010F8012B013943EA0203F9D1A3F101034C
:1002B0004FEAD370704700BF30B411F8014B12F809
:1002C000015B6C4000F8014B013BF6D130BC70473C
:1002D0002DE9F04F90E8F00F00F140004FF0040ED0
:1002E00059E0F0B4826BC36B046805252426875956
:1002F0003C444FEA724787EAF24787EA92273C4438
:1003000042684FEAF21787EAB24787EAD2073C44CD
:1003100040F8044B032D08BF6FF01B0687593A4481
:100320004FEA734787EAF34787EA93273A444368DB
:100330004FEAF31787EAB34787EAD3073A4440F80E
:10034000042B87593B444FEA744787EAF44787EA0E
:1003500094273B4444684FEAF41787EAB44787EA96
:10036000D4073B4440F8043B013DC0D1A0F13C0020
:10037000076A3C444FEA724787EAF24787EA9227C6
:100380003C4402684FEAF21787EAB24787EAD2078D
:100390003C44C463F0BC4FF0020288EA781C8CEA4B
:1003A000F84C0BEBBC1C8AEA090303EA080383EA56
:1003B0000A039C4450F8043B9C4451F8043B9C4481
:1003C000674444EA050B0BEA060B04EA05034BEA13
:1003D000030BE34484EAF42383EA34530BEBB30BBB
:1003E00087EA771C8CEAF74C0AEBBC1C89EA080305
:1003F00003EA070383EA09039C4450F8043B9C4446
:1004000051F8043B9C4466444BEA040A0AEA050A94
:100410000BEA04034AEA030AE2448BEAFB2383EA79
:100420003B530AEBB30A86EA761C8CEAF64C09EBDE
:10043000BC1C88EA070303EA060383EA08039C441A
:1004400050F8043B9C4451F8043B9C4465444AEA00
:100450000B0909EA04090AEA0B0349EA0309E14422
:100460008AEAFA2383EA3A5309EBB30985EA751C51
:100470008CEAF54C08EBBC1C87EA060303EA05038B
:1004800083EA07039C4450F8043B9C4451F8043B26
:100490009C44644449EA0A0808EA0B0809EA0A038A
:1004A00048EA0308E04489EAF92383EA395308EB70
:1004B000B30884EA741C8CEAF44C07EBBC1C86EA93
:1004C000050303EA040383EA06039C4450F8043B53
:1004D0009C4451F8043B9C44E34448EA090707EA7A
:1004E0000A0708EA090347EA0307674488EAF8238A
:1004F00083EA385307EBB3078BEA7B1C8CEAFB4C8F
:1005000006EBBC1C85EA040303EA0B0383EA05033C
:100510009C4450F8043B9C4451F8043B9C44E24406
:1005200047EA080606EA090607EA080346EA030658
:10053000664487EAF72383EA375306EBB3068AEA71
:100540007A1C8CEAFA4C05EBBC1C84EA0B0303EA28
:100550000A0383EA04039C4450F8043B9C4451F88A
:10056000043B9C44E14446EA070505EA080506EA1F
:10057000070345EA0305654486EAF62383EA365312
:1005800005EBB30589EA791C8CEAF94C04EBBC1C39
:100590008BEA0A0303EA090383EA0B039C4450F83D
:1005A000043B9C4451F8043B9C44E04445EA060467
:1005B00004EA070405EA060344EA0304644485EAFE
:1005C000F52383EA355304EBB304013A7FF4E5AE37
:1005D000A0F14000BEF1010E7FF483AEA0F1400C0B
:1005E0009CE80F00001949199219DB19ACE80F00BB
:1005F0009CE80F004044494452445B44ACE80F007F
:10060000BDE8F08F2DE9F04786468C460846089EE7
:10061000154674461946002B40F0C1808542B2FA57
:1006200082F245D94AB1C2F1200300FA02FC95409A
:1006300094402EFA03F343EA0C0C4FEA154EA8B28D
:10064000230CBCFBFEF80EFB18CC08FB00F943EAB8
:100650000C43994528D9EB1808F1FF3704D2994586
:1006600002D9A8F102072B44A3EB0903A4B2B3FB00
:10067000FEFC0EFB1C330CFB00F044EA0344A042DA
:1006800014D92C190CF1FF3304D2A04202D9ACF1D9
:1006900002032C44241A43EA07401EB1D44000232D
:1006A00034607360BDE8F0874746DDE76346F1E7F5
:1006B00092BB431B01214FEA154EAFB2200CB3FB96
:1006C000FEFC0EFB1C330CFB07F840EA0343984585
:1006D00061D9EB180CF1FF3004D2984502D9ACF186
:1006E00002002B44A3EB0803A4B2B3FBFEFC0EFBF9
:1006F0001C330CFB07F744EA0344A7424DD92C19DD
:100700000CF1FF3304D2A74202D9ACF102032C440E
:10071000E41B43EA0040C0E7C2F120039540944047
:1007200020FA03F12EFA03F34FEA154E9040AFB2D0
:100730000343B1FBFEFC0EFB1C10190C0CFB07F86D
:1007400041EA0041884522D969180CF1FF3004D2F2
:10075000884502D9ACF102002944A1EB08019BB203
:10076000B1FBFEFC0EFB1C110CFB07F743EA014337
:100770009F420ED9EB180CF1FF3104D29F4202D9EF
:10078000ACF102012B44DB1B41EA004193E76046D8
:10079000E3E76146F7E76046A4E76346B8E78342CC
:1007A00006D916B9002108467CE7C6E900E0F9E75A
:1007B000B3FA83F78FB9834201D3724508D8BEEBF1
:1007C000020460EB030301209C461EB9002169E787
:1007D0003846FAE7C6E9004CF8E7C7F1200CBB4001
:1007E0000EFA07F522FA0CF42EFA0CF1BA401C436B
:1007F00020FA0CF3B8404FEA144901431FFA84FE73
:10080000B3FBF9F809FB18300B0C08FB0EFA43EAAE
:1008100000439A4540D9E31808F1FF3004D29A45C5
:1008200002D9A8F102002344A3EB0A0389B2B3FB67
:10083000F9F809FB183308FB0EFE41EA03418E4527
:100840002CD9611808F1FF3304D28E4502D9A8F1E2
:100850000203214443EA0040A1EB0E01A0FB0298F1
:100860004145CE46434602D306D14D4504D2013818
:10087000B9EB020E68EB0403002EA7D0B5EB0E0215
:1008800061EB030101FA0CFC22FA07F3F9404CEA90
:100890000303C6E9003199E74046C5E74346D9E777
:1008A0002DE9F04D0FF2D82BDBE900AB0027B2B0F9
:1008B000CDE900AB0FF2D02BDBE900AB1446CDE95C
:1008C00002AB0FF2CC2BDBE900AB0546CDE904AB64
:1008D0000FF2C42BDBE900ABCDE93072CDE906ABFA
:1008E000002A78D180273A2101200E236E46CDF8C8
:1008F00081200DEB07080DF185028DF8807000272F
:10090000022B176021D0032B57601ED0042B976059
:100910001BD0052BD76018D0062B176115D0072BDD
:10092000576112D0082B97610FD0092BD7610CD0DB
:100930000A2B176209D00B2B576206D00C2B97623B
:1009400003D00E2BD76208BF1763B1EB830F00EB08
:10095000830012D0431C002232A901443B2B01F832
:10096000482C0AD032A90B4403F8482C392800F14E
:1009700002031CBF5B1803F8482C630F8DF8BB30D3
:10098000630D8DF8BC30630B41468DF8BD303046A9
:100990006309E4008DF8BE308DF8BF4003F042FAE1
:1009A000DDE90001DDE9022306BA14BA18BA09BA72
:1009B000DDE9042312BA69602A6119BADDE9062368
:1009C00012BA1BBA2E60AC60E8606961AA61EB6183
:1009D00032B0BDE8F08D6E463046884603F0C4F96B
:1009E000241A034608EB0401002800F0B880421ED8
:1009F000022A45D958F8042020928208012A3AD0C8
:100A00004868022A219036D08868032A229032D082
:100A1000C868042A23902ED00869052A24902AD079
:100A20004869062A259026D08869072A269022D070
:100A3000C869082A27901ED0086A092A28901AD067
:100A4000486A0A2A299016D0886A0B2A2A9012D05E
:100A5000C86A0C2A2B900ED0086B0D2A2C900AD055
:100A6000486B0E2A2D9006D00F2A886B18BFCA6BD0
:100A70002E9018BF2F9223F00307BB42394414D0A5
:100A8000087832AA3A4402F8480C7A1C93420CD9EE
:100A900032A8024402374878BB4202F8480C04D915
:100AA0008A7832A90F4407F8482C8021581C32AAB2
:100AB0001A443828309302F8481C5AD93F282DD8B8
:100AC000002232A908443E2B03F1020100F8482C11
:100AD00024D032A801443D2B01F8482C03F1030136
:100AE0001CD001443C2B01F8482C03F1040115D023
:100AF00001443B2B01F8482C03F105010ED00144C1
:100B00003A2B01F8482C03F1060107D003463E2991
:100B10000B4403F8482C01D18DF8BF200DF180085B
:100B20004146304603F07EF93A28319C3FF625AF26
:100B3000431C3B2BC0F13A02C0F13B0188BF0121AD
:100B4000022A7FF608AF002300F18002B3508B0821
:100B50003244012B02F104027FF4D1AEF5E680228B
:100B600030903A210120319C0DEB02088DF8802055
:100B7000E9E7319C0DF18008DAE700BFAFF30080B0
:100B800067E6096A85AE67BB72F36E3C3AF54FA51E
:100B90007F520E518C68059BABD9831F19CDE05B4A
:100BA0002DE9F04385B0324803F064FD28B931489F
:100BB00005B0BDE8F04303F072B94FF408414FF0BF
:100BC000807003F0B0FC38B12B4803F068F905B031
:100BD000BDE8F04302F0CABB02F0C0FB054602F0DC
:100BE000CDFBE8B903F017FD04460146284603F0A3
:100BF000D6FC10B92146214805E01D4802F0D0FB83
:100C0000014618B11E4803F04AF9E0E72946284694
:100C100003F0C5FC10B102F0FFFBFEE72946EAE74E
:100C20004FF45E31174803F07EFC014608B11648C8
:100C3000E9E70446DFF85490DFF8548001AF59F833
:100C4000046B98E807002E4487E807000C22394619
:100C5000304603F08DFA00B91EB90134052CEED1EF
:100C60000026304605B0BDE8F04302F0B1B900BF40
:100C700018470001E44A0001FC4A00012A4B000128
:100C8000544B000100880001734B0001D84800015B
:100C900090480001014B1B68184700BF000000216D
:100CA000014B1860704700BF0000002107B50B46DC
:100CB000002102460091034800F008FA03B05DF8F5
:100CC00004FB00BF950C00012DE9F0471646028B8E
:100CD0000446100712D4022902F007025BD1204615
:100CE00003F0EAF888B10138042800F21081DFE847
:100CF00010F052000E017400B300E00001290CBF97
:100D000042F0100242F02002228386F31188BFF3E2
:100D10006F8FBDE8F08703F00701481F01281ED838
:100D2000002006292768C4E9000014D1394603E0F1
:100D3000608B0130608309680029F9D123F0070333
:100D400043F002012046218303F0B6F890B341F04E
:100D5000200121832EE023F0070399B2F2E7042952
:100D600030D123F0070399B22046218303F0A4F881
:100D700010B141F020012183238B03F00709914535
:100D800040F0CE80228BD10640F1F68022F0100395
:100D9000238302F00702D4F81480238BB8F1000FEC
:100DA000B9DA0021276823F00703C4E9001143F0F2
:100DB00001032383238B03F00709914500F0E580AD
:100DC000002536E07C4940F21B127C4803F04CF9C8
:100DD00040F21B11784803F040F942B176494FF4D4
:100DE000AB72764803F040F94FF4AB71F2E7236839
:100DF00043B9714940F25712704803F035F940F297
:100E00005711E7E723691D6845B96B494FF4AD7287
:100E10006A4803F029F94FF4AD71DBE717469046B5
:100E20004FF00609238B23F0070343F006039BB220
:100E30002383A268002A76D1002F40F0AA80002DDB
:100E4000A0D043F00803238386F31188BFF36F8F8C
:100E500020465B49A84782E0022A08D0564940F262
:100E60005D12564803F000F940F25D11B2E7678B5E
:100E700047B151494FF4AF72504803F0F5F84FF4C1
:100E8000AF71A7E723695D6845B94B4940F261122C
:100E90004A4803F0E9F840F261119BE7238BB8461A
:100EA00023F0070343F004039BB24FF004092383AC
:100EB000BFE7012A08D040494FF4B2723F4803F01F
:100EC000D3F84FF4B27185E7236843B93A4940F249
:100ED00065123A4803F0C8F840F265117AE72369D1
:100EE0009D6845B934494FF4B472344803F0BCF8F6
:100EF0004FF4B4716EE70027238BB84623F0070345
:100F000043F005039BB24FF00509238391E72A497B
:100F100040F26B12294803F0A7F840F26B1159E731
:100F200000273D4685E743F00803238386F31188B5
:100F3000BFF36F8FA168002932D00E6881B343469A
:100F40004A462046D1F804A0D0471EB13368314646
:100F50001E46F3E73346FAE7002D7FF479AF4FF0F2
:100F60002003EFF3118683F31288BFF36F8F238B77
:100F700023F00803238305E793067FF5C6AE22F02E
:100F80002003238302F00702A9E6002F3FF4FAAE04
:100F9000002543F00803238386F31188BFF36F8F86
:100FA000002FD9D03E68394643464A46204602F0D3
:100FB000AFFF3746F4E700BFA64B0001C84B000166
:100FC0003D3F000170B505460E4602F091FF041E3C
:100FD00015DB4FF02003EFF3118283F31288BFF388
:100FE0006F8F4FF6FF716B8B2C8B8B4204F00704D5
:100FF00007D182F31188BFF36F8F6FF00A04204688
:1010000070BD022C0CD101336B8382F31188BFF3C6
:101010006F8F002322463146284602F079FFEEE723
:10102000062C11D8DFE804F0041E1010042504007B
:10103000002333606B6893B9C5E9006604BB0221E5
:101040002846FFF741FEDAE7104911484FF4E472F1
:1010500003F00AF84FF4E4710C4802F0FEFF1E6042
:101060006E60EBE782F31188BFF36F8F6FF00404BB
:10107000C5E782F31188BFF36F8F6FF08504BEE779
:1010800082F31188BFF36F8FB9E700BFA64B000151
:10109000C84B000108B54268034602F00302032A68
:1010A000816002D02AB1002000E0006800225A606E
:1010B00008BD04490448452202F0D6FF45210148F5
:1010C00002F0CBFFE04B0001C84B00012DE9F04FCF
:1010D00081468B4617461C46002595B0387808B9DE
:1010E000284657E37B1C2528039306D05946C8475A
:1010F0000028C0F24F830135FBE1182200210EA821
:1011000003F051F87B78252B7DD0002398469E462E
:101110009C461E46781C014610F8012B2B2A00F035
:10112000A18000F29880202A00F09F80232A00F0FE
:101130009F802BB19DF8403043F040038DF8403044
:10114000B8F1000F05D09DF8403043F020038DF832
:101150004030BEF1000F05D09DF8403043F0100341
:101160008DF84030BCF1000F05D09DF8403043F0C1
:1011700008038DF840302EB19DF8403043F0040351
:101180008DF840309DF8403003F04400442803D1EE
:101190006FF386138DF840309DF840302A2A43F0D3
:1011A00080038DF840307FD19DF841204B1C42F0E8
:1011B00001028DF841201A782E2A0CBF012100214E
:1011C0009DF8412061F341028DF8412078D15A7891
:1011D0002A2A6ED000224FF00A0C0133194611F86A
:1011E000010BA0F13006092E40F295809DF84010C9
:1011F0001292C1F3400040EAD2700A4660F3410205
:101200008DF840205CE0BA1C03928DF843309DF8C5
:101210004130DA0740F12E8154F8048BB8F1000F09
:1012200007DA9DF84020C8F1000842F004028DF86A
:1012300040205E0740F1278154F804ABBAF1000F5B
:1012400080F226819DF841306FF341038DF84130E3
:101250004FF0FF3A1CE12D2A0DD0302A7FF469AF00
:10126000012358E74FF0010C55E74FF0010E52E70C
:101270004FF001084FE701264DE703460EFB0262DF
:10128000303A184610F8016BA6F1300CBCF1090F8A
:10129000F3D999428FD09DF840101192D20F62F38A
:1012A00041018DF8401086E70B4600224FF00A0EF0
:1012B000E7E79DF84120023342F004028DF8412017
:1012C0001A786C2A47D02BD8682A31D06A2A4BD09A
:1012D0004C2A51D01A4612F8013B782B03928DF814
:1012E00043309DF8412000F2BE806D2B51D8692B10
:1012F00000F2B980572B67D8412B03D0453B022B16
:1013000000F2B18004229DF8423062F302038DF8AE
:101310004230012373E00CFB02020B46303A5DE7DA
:10132000742A25D07A2AD5D106219DF841200CE0D7
:101330005A78682A9DF8412006D1012161F3C6023E
:101340008DF841200233C5E7022161F3C6028DF812
:1013500041200133BEE75A786C2A9DF8412001D123
:101360000421EBE70321F0E705219DF84120ECE79C
:1013700007219DF84120E8E7BDF8402022F4F04223
:1013800022F0020242F4804242F00202ADF8402014
:10139000DFE76E3BD9B201238B4040F282410B4222
:1013A00037D113F0240F51D1D8075CD503219DF814
:1013B000423061F302038DF8423002F07803A3F16A
:1013C00040014B424B411AE00120A3F15801C9B240
:1013D00000FA01F111F4624F94D140F60106314256
:1013E0001DD111F4043F3ED09DF8423060F302035A
:1013F00002F07802402A8DF8423034D000239DF864
:101400004020C2F340010B4363F341028DF84020BA
:10141000FDE602219DF8423061F30203E8E7022075
:101420009DF8421002F0780260F30201402A8DF824
:10143000421002BF9DF8401041F001018DF84010AC
:10144000632BDBD1131E18BF0123D8E703219DF8BE
:10145000423012F0780F61F302038DF8423014BF6E
:1014600001230023CBE79DF8403043F001038DF8C2
:101470004030C3E79DF94020002AACBF4FF0FF3851
:10148000DDF84480D5E698077FF5E2AEDDF848A0A8
:101490000023CDE911339DF842309DF8411003F04F
:1014A0000703012BC1F3C30133D1CB1E042B04D896
:1014B000DFE803F0214646212100236801294FEA95
:1014C000E372CDE90E321CD19DF93830DA17CDE93F
:1014D0000E3204349DF8403013F0030650D03A46E3
:1014E00059464846039B02F0A1FD0028C0F25281F4
:1014F0000544039FF2E554F8043BDA17CDE90E32B8
:10150000E8E70229E5D11AB243F3C033CDE90E234F
:10151000DFE7022B24D1CB1E042B04D8DFE803F035
:1015200018101018180001294FF0000254F8043B5D
:1015300014D00229CDE90E32CCD19BB20E93C9E76B
:10154000073424F00704F4E80223CDE90E23C1E7B1
:1015500054F8043B0E9300230F93BBE7DBB2CDE7B7
:10156000042B08D1073424F00704D4E900230834FD
:10157000CDE90E23AEE7032BACD154F8043BDDE7F5
:101580009DF843007828B4D862281CD825283FF459
:10159000ADAD5828ADD1DDE90E010DF13603009354
:1015A00010AA08AB02F0FCFCBAF1000F074680F26B
:1015B0009980002F9DD00DF13603D81B002E00F02E
:1015C000C0800130BDE06338152892D801A252F8DE
:1015D00020F000BFA9160001BB160001F3140001A2
:1015E000F3140001F3140001F3140001BB16000111
:1015F000F3140001F3140001F3140001F3140001CB
:1016000047170001DF16000105170001F314000160
:10161000F31400012D160001F3140001DF16000180
:10162000F3140001F3140001DF160001BAF1000FFA
:101630000E9F35DB5146384602F091FD07EB000A5C
:10164000002F3FF456AF00269DF8423013F01002F1
:10165000059200F0928002305B06119A48BF129BFF
:10166000104448BFC018B8F1000F049240F39F80A7
:101670009DF84020A8EB0008C2F3800350070693B2
:1016800000F19580510640F188803EB159463046C0
:10169000C84700287EDB069B01351E4630227DE0D0
:1016A000384602F055FDC9E70E9B002601208DF853
:1016B000203008AF0DF1210AC6E719075ABFC3F35E
:1016C00000135E012B26DDE90E23002BBFF663AF6E
:1016D000524263EB43032D26CDE90E235BE7002640
:1016E00059E700269DF840200DF13603DB1B6FF310
:1016F00086129A458DF840207FF65BAFAAEB030374
:10170000119356E70E9890B30DF136030093002124
:1017100008AB10AA02F044FCBDF84230BAF1000F49
:1017200003F0EF0343F4F04343F010030746ADF832
:101730004230D6DA00283FF4DCAE00260DF1360345
:10174000181A9A4680E70E9B07293FF6D2AEDFE8CB
:1017500001F00C04060C08080C0C1D70C9E61D8075
:10176000C7E6EA17C3E90052C3E61D60C1E62F4F82
:10177000064607F1050A052066E71A0748BF01304B
:101780006AE71046079306925946C847DDE90623E3
:10179000002804DA15B0BDE8F08F20224346194630
:1017A000002903F1FF33ECDC454498466D1A2EB155
:1017B00059463046C8470028ECDB01359DF84230D9
:1017C000DA0601D41B0705D559463020C847002842
:1017D000E0DB0135059B33B159469DF84300C8470E
:1017E0000028D7DB0135049E2E4405E05946302001
:1017F000C8470028CEDB0135731B002BF6DC5346AF
:101800003A465946484602F011FC0028C2DB05441E
:10181000A844A8EB0503002B7FF76BAE59462020A8
:10182000C8470028B6DB0135F3E700BF034C0001D1
:101830004FF02003EFF3118183F31288BFF36F8F12
:1018400001237F200B4AC2F840350B4BC3F8180127
:101850000020C2F8040EC2F8080EC3F82401C3F831
:101860002C0103F57F23C3F8100181F31188BFF326
:101870006F8F70470000084100200041F8B5052334
:10188000194D1A4F2C781A4E0134B4FBF3F303EBC5
:101890008303E41A02F0D1FD164A137873B157F8A6
:1018A0002430C01A072809D833782BB95721124899
:1018B00002F0E8FB012333700020F8BD00210F4B3C
:1018C0003170D3F8140138B1C3F81411D3F81431BE
:1018D0002C700CB9012313702C7802F0AEFD47F880
:1018E00024000120E9E700BF82010021E00000217F
:1018F0008001002181010021094C000100500041BC
:1019000020B1034B800143F001031847704700BF2B
:10191000D048000101F04ABE10B543680A680C4681
:101920009A4207D90548452102F0ACFB002318462E
:10193000636010BD4A6801201344F9E73B4C000185
:101940007FB50546C06801AA02F0D8FC044638B14C
:10195000024645210D4802F095FB204604B070BDBB
:1019600001992B6A8B42F8D0E868029A83689B68D9
:101970009847064630B102464521054802F082FBF1
:101980003446EAE7019B2B62E7E700BF604C0001A9
:10199000864C0001F8B58168054600293CD0D0E9A5
:1019A000043601391E443144FFF7CAFF041E07DA2A
:1019B0003346224645212A4802F064FB2046F8BD02
:1019C000E86802F06CFBAC68B4FBF0F300FB134476
:1019D0005CB1041BE8688368DB6898472F68AB68D4
:1019E00001792246F81802F0DEFBAB68E8682A6845
:1019F000234481684C683146A047044620B1024622
:101A0000334645211748D7E7EB695BB92B69AA68CC
:101A100013442B610023AB600024CFE7135DDB434D
:101A200013550134AB682A689C42F7D3E868816893
:101A30000C683146A047044628B1452102460A48B1
:101A400002F020FBBAE73246EB69A968286898479C
:101A500004460028DAD0024645210448F0E700BFDA
:101A6000A74C0001DA4C0001034D00011E4D00019E
:101A70002DE9F7430D46DDE90A8691461F460446E7
:101A800080B179B172B1009300230846019302F04E
:101A900006FBB7FBF0F303FB107040B1452119487A
:101AA00002F0F0FA6FF00D0003B0BDE8F0836A4673
:101AB0002846154902F026FC019B002BF2D008EBCA
:101AC0000602934202D245211048E9E7284602F077
:101AD000E6FAB8FBF0F303FB10800028F3D1C4E969
:101AE0000097E5602061A060C4F8148016B9019EDB
:101AF000A6EB08060C9B0020E3614FF0FF33A661C4
:101B00002362D1E7374D000119190001734D00011F
:101B1000014910220A60704710ED00E072B649409A
:101B200081F3118801B5FFF7A9FE002802D0BFF3A9
:101B30004F8F20BFBDE8014080F3118862B6704727
:101B400037B505460C46C9B18B6810480093D1E9FA
:101B50000023452102F096FA636945210093D4E9F8
:101B600003230B4802F08EFA4521E269094802F08E
:101B700089FA4521A269084802F084FA21462846DC
:101B800003B0BDE8304001F063BF00BF994D0001D4
:101B9000CD4D0001014E0001154E000140B200285C
:101BA00007DB01234109034A00F01F00834042F88C
:101BB0002130704700E100E0054B420953F8222034
:101BC000012300F01F0003FA00F01040704700BF2F
:101BD00000E100E00131072908B508D90D490E4898
:101BE0005B2202F041FA5B210A4802F036FA40B269
:101BF0000028ACBF00F16040084B4FEA4111C9B268
:101C0000ABBF00F5614000F00F0080F800131954DD
:101C100008BD00BF484E0001C84B000114ED00E0B4
:101C200030BFFFF7FDBF00BF08B5084B084A23F0DF
:101C30007F039360BFF34F8FBFF36F8F01F08EFF71
:101C400001F0D0FF00F058FA01F094FF000000010D
:101C500000ED00E01EF0040F0CBFEFF30880EFF37F
:101C60000980816911F8021C0229FFD001B502F038
:101C700060FA01BD0446084611461A46002383F364
:101C80000B880A4B2025A3F5806686F30B8883F327
:101C9000098863B64FF0000383F31188BFF36F8F99
:101CA000A04785F31188BFF36F8FFEE7880D0021F1
:101CB00001B5EFF30580A0F110004FEAC000044920
:101CC000014409C99847BDE801400249084700009E
:101CD00030470001D91C0001704700BF38B5214CC6
:101CE0004521214802F0CEF9A36A9D0103D5452183
:101CF0001E4802F0C7F9A36ADC0103D545211C4840
:101D000002F0C0F9174DAC6A14F4801404D04521D8
:101D1000184802F0B7F90224AB6A180303D545212D
:101D2000154802F0AFF90F4DAB6A590303D54521B1
:101D3000124802F0A7F9AB6A9A0303D5452110486F
:101D400002F0A0F9074DAB6ADB0303D545210D482E
:101D500002F098F9AB6A20466FEA03436FEA134337
:101D6000AB6238BD00ED00E07E4E00019B4E0001ED
:101D7000B34E0001D24E0001014F0001244F00017B
:101D80004E4F00016D4F000170B5204C06460D46C8
:101D90001F48452102F076F9A36ADB0403D54521EB
:101DA0001C4802F06FF9A36A1C0503D545211A48A7
:101DB00002F068F9154CA36A980510D5452117481B
:101DC00002F060F9A26BA36A190408D545211448F2
:101DD00002F058F91EB1A36A23F40043A3620B4C2E
:101DE000A36A5A0503D545210E4802F04BF9A36AB0
:101DF000DB0503D545210C4802F044F90020034AD5
:101E0000936A43F47F439362287070BD00ED00E055
:101E10009D4F0001B84F0001CE4F0001E64F000179
:101E2000045000011E5000013E50000170B5274CC7
:101E300006460D462648452102F024F9A36AD80635
:101E400003D54521234802F01DF9A36A190703D5DC
:101E50004521214802F016F91C4CA36A9A0710D5B7
:101E600045211E4802F00EF9626BA36A1B0608D5D5
:101E700045211B4802F006F91EB1A36A23F0800336
:101E8000A362124CA36AD80703D54521154802F076
:101E9000F9F8A36AD90602D4A36A9A070ED50B4BA8
:101EA0009B6ADB060AD5104910484FF4AE7202F067
:101EB000DBF84FF4AE710C4802F0CFF80020034A73
:101EC000936A43F0FF039362287070BD00ED00E059
:101ED0005B50000176500001CE4F0001AE50000172
:101EE000CB500001E65000010A510001C84B00012F
:101EF00070B5694B0546586800268AB0C0F30803E0
:101F000086F31188BFF36F8F02F07F44B4F17F4FE7
:101F100007D102F00C04082C0ED145215F4802F0D5
:101F2000B1F85F494FF484625E4802F09DF84FF4C7
:101F300084615B4802F091F814074CBF0D460126FE
:101F4000002DEED00024DA1E8DF80740092A00F299
:101F50009280DFE802F00585897090909090908DD6
:101F60004521514802F08EF88DF807404A4CE36A4B
:101F70009A0705D545214D4802F084F8002429E050
:101F8000E36A002B02DA45214948F5E7E36A5B0082
:101F90005DD54521474802F075F86369AA6943F4A5
:101FA00080736361BFF34F8FBFF36F8F636932F844
:101FB000022C23F480736361BFF34F8FBFF36F8FE5
:101FC0004DF602739A421ED145212A683A4802F022
:101FD00059F82C689DF807309BB92022294602A8A1
:101FE00002F0D6F8099B002E51D0C3F3080222B9A3
:101FF0006FEA53236FEA43230993204602A9FFF7B0
:102000009FFD0AB070BDA36ADBB233B101200DF1B0
:102010000701FFF70BFF0446DCE7A36A13F47F4FC9
:1020200005D001200DF10701FFF7AEFEF3E7A36A2B
:10203000B3F5803F02D3FFF751FEECE7184940F2B9
:10204000F222184802F010F840F2F22171E7144928
:1020500040F2F622134802F007F840F2F62168E752
:1020600000200DF10701D4E700200DF10701DBE7A7
:102070004521124880E7124910F4F87F114A1248AE
:1020800008BF0A46103B452101F0FCFF76E723F428
:10209000FF7323F00103AFE700ED00E07251000190
:1020A0000A510001C84B0001A2510001BE510001BC
:1020B000E4510001F75100011B5200013C520001A4
:1020C000445100015951000165520001044B5A6905
:1020D00042F010025A615A6942F480625A617047B4
:1020E00000ED00E0EFF30880EFF3098101B57246DF
:1020F000FFF7FEFE01BD00BF002320210348C218E8
:1021000001331E2B82F80013F9D1704700E100E083
:10211000002080F31488BFF36F8F002080F30A88BB
:1021200080F30B88FFF7F6FB00200E490860BFF331
:102130004F8F0D4880F3088800F03EF8202080F390
:1021400011880A484FF40061401880F30988EFF3C2
:1021500014800221084380F31488BFF36F8FFFF7C8
:1021600063FD000094ED00E0880D0021880100214E
:10217000BFF34F8F0549064BCA6802F4E062134370
:10218000CB60BFF34F8F00BFFDE700BF00ED00E065
:102190000400FA05002318460649D1F89020C2F33E
:1021A0000722934200DB7047C1F89830C1F8A000C5
:1021B0000133F6E700ED00E010B572B6002484F3B9
:1021C0001388FFF7E7FF23464FF0FF300C4A03F177
:1021D00020010133102B42F82100F8D100234FF0E9
:1021E000FF30074A03F160010133102B42F8210050
:1021F000F8D162B6BFF34F8FBFF36F8F10BD00BF32
:1022000000E100E0014B1860704700BF04000021AE
:10221000402373B50B4C0093041B0B460D460A4933
:10222000A41061430646094A094801F0DBFF011E7C
:1022300005DA30462B4602B0BDE87040184702B0C0
:1022400070BD00BF08010021B76DDBB6554200012B
:10225000E8460001C9B2012908B508D9084909486A
:102260007A2201F001FF7A21054801F0F6FE0C22E6
:10227000036901FB0233186C00F0070008BD00BFC2
:102280007D520001C84B000170B5C9B20129036934
:102290000AD91849184840F25D1201F0E5FE40F2F3
:1022A0005D11144801F0D9FE4FF02004EFF31185C1
:1022B00084F31288BFF36F8F0C2606FB0134246C65
:1022C00014F0C00408D0A24206D085F31188BFF3F1
:1022D0006F8F4FF0FF3070BD012271430B441A64C1
:1022E00085F31188BFF36F8F43680B445B68984791
:1022F0000020F0E77D520001C84B0001084B70B58B
:10230000C31A0D4607499B1004465943402206480C
:10231000FFF7BAFF2B4601462046BDE8704018473C
:1023200008010021B76DDBB6E846000170B5002258
:10233000012104460520FFF74DFC0F4801F00CFA7F
:102340000E4B984215D101F029FA26690C49304606
:1023500001F002FE00280BDB0125356424690849E1
:1023600004F11C0001F0F8FD002801DB0020E56409
:1023700070BD6FF00400FBE7B92300010000AD0B56
:10238000EC48000101460C23002270B54B4308487D
:10239000C4184033D4E90E561844A26301F00FFF6D
:1023A0002DB132462B46BDE870400248184770BD3B
:1023B00008010021E8460001012808B506D00328DD
:1023C00008D090B90E4B1B6C5B0717D1BDE80840D5
:1023D000FFF7D8BF0B4940F26E220B4801F044FED4
:1023E00040F26E21074801F038FE064940F27222A1
:1023F000054801F039FE40F27221F3E708BD00BF45
:10240000080100217D520001C84B000108B54FF0C2
:102410002003EFF3118183F31288BFF36F8F114A0A
:10242000136843F002001060DA0708D481F31188C2
:10243000BFF36F8FBDE80840012001F0D5B90A4B0A
:10244000D3F80C24D3F80C34D307EFD5074801F0A8
:10245000B6FE81F31188BFF36F8FBDE808400020FE
:10246000FFF790BF580100210050004148010021B2
:1024700010B54FF02003EFF3118483F31288BFF3FC
:102480006F8F074A136823F00201DB07116002D443
:10249000012001F005FA84F31188BFF36F8F10BD9E
:1024A000580100212DE9F843012206463E49D1E8B2
:1024B000EF3FC1E8E02F0028F9D19BB93B493C48E8
:1024C0004B60CB608A60FEF77DFD00280ADA39494F
:1024D0004FF40C72384801F0C7FD4FF40C713548C9
:1024E00001F0BBFD6EB3731E012B53D8012E06D134
:1024F000324BD3F81C3403F00303022B21D002F03B
:10250000C8F80546F8B92E4B1B78E3B102220746FE
:102510002A4BC3F808234FF00008284CDFF8A4909A
:10252000D4F81834D4F81824D20316D503F00303D2
:10253000022B01D0012E10D13DB387F31188BFF3D8
:102540006F8FBDE8F8834FF02003EFF3118783F31B
:102550001288BFF36F8F0125DDE73846FFF7DEFAFB
:10256000D4F81835DBB2012BDAD1D4F80421002AD3
:10257000D6D0C4F80481D4F804210222C4F8182566
:102580002022C9F88021A360CAE702220B4BC3F8BE
:102590000423D6E7074940F24222074801F064FDD0
:1025A00040F242219BE700BF04010021F40000211A
:1025B000240100217D520001C84B00010050004160
:1025C0008501002100E100E008B5074802F052F85B
:1025D00038B10648FFF716FE0448FEF761FB0020FD
:1025E00008BD6FF01200FBE700470001F125000174
:1025F0000A2838B50446074D04D1AB680D2128469A
:102600005B689847AB6803485B68E1B2984720462F
:1026100038BD00BF00470001024B0B60012313606F
:10262000704700BF5C01002100487047404900012D
:1026300010B502F01CF8034C206002F015F8606041
:10264000002010BD5C01002170B50C46154602F05B
:102650000BF829460646204601F00EFE10B3B4FBE7
:10266000F6F306FB134323B9B5FBF6F306FB13534E
:1026700043B12B46224645210D4801F003FD6FF082
:10268000150002E0AE4201D9002070BD01F0ECFF60
:10269000064604F18074204601F062F9AD1B344413
:1026A000F9D1F1E72B46224645210248E5E700BF74
:1026B000E352000107530001F8B50C4619462046C5
:1026C00016461D4601F0D8FD50B104F180772C4329
:1026D00014F003040DD02B463A4645210E4803E082
:1026E0002B46224645210D4801F0CCFC6FF0150029
:1026F000F8BD4DB12B19032BA7EB040006D8084AEF
:10270000D2F80034DB07FBD50020F1E7331B196852
:1027100001F056F9043CEDE729530001075300018D
:102720000000084170B50D461946284616461C465D
:1027300001F0A2FD40B12CB12246304605F1807176
:1027400001F026FD002007E0044823462A464521E3
:1027500001F098FC6FF0150070BD00BF0753000139
:10276000F8B504460D46076901F093FF90B92C4B6C
:102770001B787BB16426606801F013FEE0B901208C
:1027800001F059FF013EF6D1F4E786F31188BFF35B
:102790006F8FEFE74FF02003EFF3118683F312887A
:1027A000BFF36F8F6068314601F0FBFD90B986F38F
:1027B0001188BFF36F8FEDE74FF02003EFF3118621
:1027C00083F31288BFF36F8F6068314601F0E9FD33
:1027D0000028DAD03B691D70626838691368C3F855
:1027E00044050120C3F848050020C3F82001D3F8B0
:1027F0002051C3F858015268D3F85801D20608D5C1
:10280000082062681268C2F800054FF48002C3F81D
:10281000042301229A6081F31188BFF36F8FF8BD02
:1028200085010021F0B54B79012B29D0032B24D150
:1028300010278B79032B20D1CE790EB1012E1CD11C
:102840000A79012A1ED0022A20D0B2B914460B6898
:102850004568B3F5164FD5F800C06ED033D8B3F540
:10286000165F6DD01CD8B3F5966F6BD010D8B3F54A
:10287000967F6AD0B3F5167F6AD06FF085005BE073
:102880000027D6E74FF480740E22E0E70024FBE730
:10289000B3F5166F5FD0B3F5965FEED1384B3CE0E1
:1028A000B3F5E14F5AD007D8B3F5615F58D0B3F50F
:1028B000964FE2D1334B30E047F61225AB42DCD1E4
:1028C0004FF4000329E0B3F5613F4BD013D8B3F5C3
:1028D000963F4AD009D84DF6C025AB4247D0B3F554
:1028E000614FCAD14FF46B0317E0B3F5E13FC4D198
:1028F0004FF0EB7311E0B3F5612F3BD008D8224DB8
:10290000AB423AD0B3F5E12FB7D14FF0E86304E022
:102910001E4DAB42B1D14FF080530569CCF8243540
:1029200043683A431B6834432243C3F86C252B1D8C
:1029300003C983E803000020F0BD4FF41D03ECE75A
:10294000134BEAE74FF49E23E7E74FF4A033E4E7A5
:102950004FF41C33E1E74FF41D23DEE70D4BDCE7BA
:102960000D4BDAE74FF06C73D7E70C4BD5E74FF41C
:102970006503D2E74FF07063CFE74FF08063CCE799
:1029800000B0130000A04E0090D0030040420F00A2
:102990000050270000C0750000F03A0000903A0196
:1029A0002DE9F7438046002201211320FFF712F999
:1029B0001320FFF7F3F80021D8F80470D8F810605E
:1029C0003C6801AAC4F80015C6F80080D7F80C903E
:1029D000484601F036FD051E1EDB019BD9F800209C
:1029E0001979186801F040FD051E15DB4046311DC0
:1029F000FFF718FF054678B97B6899072BD506F1D4
:102A0000180000F09BFF284B984209D04521274829
:102A100001F038FB6FF00405284603B0BDE8F083F1
:102A2000337E14F10C0F43F00043C4F8A0310AD1F7
:102A30001F49204840F24E2201F016FB40F24E2181
:102A40001B4801F00AFBC4F88C300123327E93400E
:102A5000194AC2F804350823C4F800353B7A53B943
:102A6000C4F81031D4F810317369C4F83435012337
:102A7000C4F8383523607B689A075CBF4FF48073D5
:102A8000C4F804337B68DB0644BF4FF48003C4F80A
:102A900004333369C4F844350023C4F848350123AE
:102AA000A360E360B8E700BF0000AD0B7053000106
:102AB00094530001C84B000100F000410D4B186811
:102AC000010A0006BFF35F8F0B4BD3F804351818CB
:102AD00041F10001B3F5801F0AD2084BD3E900236E
:102AE000904271EB030303D210F1807041F10001B9
:102AF000704700BF6C0100210060014158000021B7
:102B00002DE9F7432E4BD3F8042390070BD5D3F8C8
:102B1000042142B10022C3F804212A4AD3F8043127
:102B2000136801331360264AD2F80433D90327D53A
:102B3000254BD3E8EF1F21F00100C3E8E40F002C80
:102B4000F7D1CB0702D4D2F84031CBB100251C4CD1
:102B5000C4F84051D4F84031FFF7B0FF4FF02003E4
:102B6000EFF3118283F31288BFF36F8F174BD3E912
:102B70000267B042B94106D282F31188BFF36F8F6A
:102B800003B0BDE8F0834FF0FF38D3E900104FF0F9
:102B9000FF391D60C3E902894FF48033C4F848331C
:102BA000C4F84051D4F8403182F31188BFF36F8FDD
:102BB0000029E5D0009032463B4628468847DFE7AB
:102BC000006001416C0100216401002140000021EE
:102BD0002DE9F74F4FF0010808FA00F814460646B1
:102BE0001D466FEA0802DFF830A1DAE8EF3F03EA9A
:102BF0000201CAE8E01F0028F7D14FF48037DFF860
:102C00001C91B740C9F80873BFF35F8FBFF36F8F94
:102C100008EA03030093FFF751FFA04271EB05039D
:102C20004BD23F4B201A65EB0101984271F1000134
:102C300056D23C4B03EB0613D3E902239D4208BF57
:102C4000944243D04FF0000B24F07F4EF446032013
:102C500006F150039B009BB203F1824303F5B033AE
:102C6000C9F84873C3F800B01A6806F5A872019253
:102C700001992CF07F4249F821206FF00202C9F837
:102C80004473D9F80415521A6244DFF89CC022F04C
:102C90007F4262451AD91A685AB1D9F80415A1EBD6
:102CA0000E0222F07F42B2F5000F0FD9C3F800B038
:102CB0001A6800EB010C0130DAE71C4BD3E8EF1F78
:102CC00041EA0801C3E8E21F002AF7D11549184874
:102CD0003301C850002301EB0612C2E902455360DC
:102CE000009BABB1DAE8EF3F43EA0803CAE8E23FF2
:102CF000002AF7D1094BC3F804730C4BD3E8AF3F5C
:102D0000F340DB0742BF4FF480020A4BC3F80021B7
:102D100003B0BDE8F08F00BF6801002100600141F1
:102D20000100800040000021FDFF7F0064010021C0
:102D3000A92D000100E100E070B54FF0FF30002543
:102D40004FF0FF31144C154BC4F80855C3E902018C
:102D50004FF4803302264FF48002C4F80433104B42
:102D60000121C4F804631620C3F880212A46FEF727
:102D700031FF1620FEF712FF01230A4AA3602846FE
:102D8000236013604FF480720023FFF721FF304669
:102D9000FFF788FB284670BD00600141400000211C
:102DA00000E100E068010021F8B5144922F07F45F8
:102DB000D1E90063921B140A22F0FF02921943F139
:102DC0000003C1E90023A5F50011B1F5400F0AD2B7
:102DD0000B4909684FEA112C09064E1909494CF1B3
:102DE0000007C1E9006712F5807243F10003FFF7A5
:102DF000EFFE2046BDE8F84000F054BF500000212F
:102E00006C0100215800002108B503685A090CD054
:102E1000012A12D00E490F4840F2472201F024F94E
:102E200040F247210A4801F018F94FF0FF3222FA28
:102E300003F3D907EED5084808E04FF6FF7203F018
:102E40001F03DA40D207E5D50360044808BD00BF80
:102E5000EA530001C84B000100058C4100088C4179
:102E600030B5024600240B490B4D0B6805EB0310EF
:102E7000D0F80808C0B218B904B10B60002007E010
:102E80000133072B4FF00104F0D96FF01B000B60EA
:102E9000136030BD7001002100000841F7B5434DBB
:102EA0000646D5F820320C46B3F5006F174608D019
:102EB0003F494048212201F0D7F821213C4801F048
:102EC000CCF801A8FFF7CCFF002867D1D5F8202265
:102ED000B6FBF2F302FB1363002B61D1D5F820227D
:102EE000B4FBF2F302FB1343002B59D1D5F8202297
:102EF000D5F824325343A34252D3002C50D0019B27
:102F0000072B07D92C4977222A4801F0ADF8772101
:102F10002948D4E7D5F82012B6FBF1F201FB126282
:102F200032B125497822234801F09EF87821EFE755
:102F3000D5F82022D5F824124A43944206D91E49D6
:102F400079221C4801F090F87921E1E7D5F82012A8
:102F5000B4FBF1F201FB124232B117497B22154852
:102F600001F082F87B21D3E71B0103F1824101F5D7
:102F70000021C1F80068C1F80448C1F80878D1F808
:102F8000002896420FD1D1F8042894420BD1D1F8F1
:102F90000838DBB29F4218BF6FF00D0003B0F0BDE0
:102FA0006FF01500FAE76FF00D00F7E70000FF0182
:102FB0001D540001C84B000149540001034845213C
:102FC00008B501F05FF80020FFF7D2F87B5400014C
:102FD00038B5044681692B4800F061FF00232A4A76
:102FE0002A49C2F800354FF0FF32C1F80823BFF379
:102FF0006F8F72B6264903F120000133102B41F880
:103000002020F8D100234FF0FF30214A03F1600166
:103010000133102B42F82100F8D14FF0E0230022B9
:103020001A61D3F8042D03F5506342F000725A6020
:103030005A6A22F4E0225A62EFF31482920707D50B
:10304000EFF3148222F0020282F31488BFF36F8F31
:10305000BFF34F8FBFF36F8FA26901219A602046A3
:10306000A56900F031FA58B1002383F30B8883F38C
:103070000A882A6882F3088883F309886B6898476E
:1030800038BD00BF9D540001003001410050004197
:1030900000E100E01FB50446074A01AB07CA83E818
:1030A00007000C221946204601F062F800280CBFE8
:1030B0002046002004B010BD9C48000170B50546B4
:1030C0000024054E56F8040B2844FFF7E3FF10B91F
:1030D0000134052CF6D170BD904900012DE9F04F67
:1030E000814687B010460E4614461D46D768D2F872
:1030F0001080FFF7CFFF38B915B96D4800F0CFFE4B
:10310000002007B0BDE8F08FA069484503D0002D2E
:10311000F6D16848F2E71DB9B0423DD06648EDE708
:103120003046FFF7CBFF8442EAD1226A634B9A42D2
:10313000E6D1E3192CBF012700270DF10A0018EB97
:10314000060A2CBF4FF0010B4FF0000B019301F06A
:1031500014FA0146002840D065BB594800F09FFE94
:10316000584800F09CFEADF80A50002F4BD1BBF13F
:10317000000F48D1B44246D3544544D2019B5F1E50
:10318000BE423DD8BA453BD918EB0908E3693CD3A8
:10319000002DB5D14C48B1E7FFF790FF844201D034
:1031A0004A48ABE7216A454B9942C2D0484800F0F3
:1031B00076FEA5E70022ADF80A20002FA0D1BBF1D2
:1031C000000F9DD1B4429BD3544599D2019B5F1E01
:1031D000BE4295D8BA45D7D892E76169BDF80A20B2
:1031E000914205D2002D8BD13A4800F058FE87E776
:1031F00037B9BBF1000F03D1B44201D35445BDD35D
:10320000002D7FF47DAF344878E74B45C0D343456C
:10321000BED2321DA2EB0902D358994504D9002D24
:103220007FF46EAF2D4869E79845F8D92769DFF834
:10323000B090374407F1050A0DF10C0899E8070032
:1032400088E807000C224146384600F091FF00B99B
:103250003FB90137BA45F1D1002D7FF451AF214874
:103260004CE7FA68A3699A4209D1246901F062F92E
:10327000014648B1002D7FF443AF1B4897E7002D6E
:103280007FF43EAF194839E72146304607F1100276
:1032900001F057F9014620B1002D7FF431AF1448F9
:1032A00085E715B9134800F0FAFD012029E700BFB2
:1032B000AF540001CF54000102550001FFFF0291FD
:1032C0007F550001A6550001565600012F550001FB
:1032D00058550001E95500012956000182560001A8
:1032E000A8480001AF56000113570001E056000145
:1032F000335700015F5700012DE9F041154B074698
:10330000D3F8B030BFF34F8F1422134D02FB035597
:10331000284600F083FB012803D000242046BDE8A6
:10332000F0814FF000082C1DAE1C304600F076FBFB
:103330004045F2D9A01C00F071FB0546204600F084
:103340006DFBB842EAD0023504EB450408F10108F0
:10335000EBE700BF00850001B4850001024BD3F804
:10336000A800BFF34F8F7047008500014FF0005356
:10337000014A1A60704700BF15FCBA254FF0005390
:103380001868054B984205D0044B98420CBF0120A9
:103390000220704700207047B6B3B4B55DCE03F18C
:1033A00030B54FF00055184B2A6801469A42ADF5EA
:1033B0000F7D26D10023CDE90133EB680EAA0093DF
:1033C00005A84FF40073FEF753FB044640B14521B6
:1033D00002460E4800F056FE20460DF50F7D30BD2A
:1033E0000123D5E9011205A800F05FFE044618B1DB
:1033F000024645210648EDE74921064800F042FE15
:10340000EAE76FF00D04E7E7B6B3B4B5795700010A
:103410009B570001C55700014FF00053014A1A6045
:10342000704700BF5DCE03F12DE9F043224885B01F
:1034300001F0F5F8002504461F4B204ED3F83880E4
:10344000DFF87C90A84503D8002005B0BDE8F083E4
:10345000636A96E807001F6801AB83E807000C2247
:103460001946384600F084FE88B987B1636A21693D
:103470001B681A6991420AD19A69A169914206D8DA
:10348000E169914203D962695B699A430AD0276A6C
:1034900067B10C4800F003FD404080F311884FF005
:1034A000040002DFE36801351C44CBE7484600F026
:1034B000F6FC636A1F60F5E700020001B4480001F2
:1034C00005580001DC5700012DE9F04F0F46064674
:1034D00087B0A0B301F0A3F84FF000080446B36B27
:1034E00043454ED94FF00009DFF8ACB04FF0000A69
:1034F0005BF8043B0093294B53F8045B0193009B5A
:103500001D44274B93E8070003AB83E807001946E7
:103510000C22284600F02CFE019B00B99DB90AF14F
:10352000010ABAF1050FE7D11E4B09F101099945CE
:10353000DCD317B10022636A1A60236A33B3002018
:1035400007B0BDE8F08F2B6A174A9342ECD1AE4228
:10355000EAD0696B05F13C038842E5D025691A6918
:1035600095420AD19A69A569954206D8E5699542BE
:1035700003D962695D69AA4305D0DA680130134452
:10358000EAE70120DCE70FB1626A1360E36808F143
:1035900001081C44A3E700BF245A0001A44900010C
:1035A000C048000101000000FFFF02910022D3008B
:1035B00003F1FF7303F58033D3F80013013107D013
:1035C000D3F800130132D3F80433202A0B60EED174
:1035D000144BD3E94C32072B07D1023A032A124B82
:1035E0000CD9D3F80024D10716D4104B1A68104B0D
:1035F000C3F844250F4B104A1A6070470F498A5C84
:10360000002AEED0D3F80024D207EAD50022C3F86E
:103610001421C3F81821E4E76FF00102C3F8002475
:10362000E3E700BF0000FF01005000410080FF0100
:1036300000600041240000210090D00338580001B0
:1036400070B501250268B2FA82F3C3F11F03DBB241
:1036500005FA03F422EA0404D0E8EF6F964204D19D
:10366000C0E8EC4FBCF1000FF6D1EBD101480B7074
:1036700070BD00BF0000AD0BF7B5334B044650B131
:10368000012825D031493248D82200F0EDFCD8215C
:103690002E4800F0E2FC0222C3F80823C3F804011C
:1036A000D3F8042101220746DA60012342F21075A3
:1036B000254E8DF80730B4B1012C32D0254924486D
:1036C00040F2473200F0D0FC40F247312148E0E7B9
:1036D0000022C3F80803C3F80021D3F800210DF13C
:1036E00007075860E1E78FB1D6F8183403F00303F9
:1036F0003B70D6F81834DA0311D59DF8070001287D
:103700000DD100F098FF013DD5D108E0D6F818346E
:10371000D90304D5012000F08EFF013DF6D103B09E
:10372000F0BD3FB1D6F80C3403F001033B70D6F87E
:103730000C34E0E7D6F80C34DB03F0D5012000F0C0
:103740007AFF013DF6D1EAE7005000413C58000104
:10375000C84B00017958000108B550B90A490B4817
:1037600040F2151200F080FC40F21511064800F0FE
:1037700074FC074B1A7922B90122186005481A71A6
:1037800008BD0548FCE700BF3C580001C84B0001DC
:10379000740100210000AD0B0C00AD0B08B50E4B01
:1037A0001B7953B90D490E484FF4977200F05CFC39
:1037B0004FF49771094800F050FC0520FEF7FCF922
:1037C00010B90520FEF7EAF90122064BC3F81825C7
:1037D000C3F8142508BD00BF740100213C58000146
:1037E000C84B00010050004108B5294B1B7953B963
:1037F00028494FF4B472284800F036FC4FF4B471F5
:10380000244800F02AFC254B50B1012836D021492C
:103810004FF4D372204800F027FC4FF4D371EFE748
:10382000D3F81824D3F81814C90311D502F00303F0
:10383000022B1CD1194AC2F818350023C2F80431F2
:10384000D2F804310223C2F80433012393600DE05F
:10385000D3F81424D2070FD5D3F81C2402F00302A6
:10386000013A012A05D80222C3F8042308BD012B1E
:1038700002D00020FFF700FF0123DBE70022C3F89E
:103880000021D3F80021C3F804031860EEE700BF5D
:10389000740100213C580001C84B00010050004158
:1038A00008B5094B1B7953B90849094840F2AD12D4
:1038B00000F0DAFB40F2AD11044800F0CEFBBDE8A9
:1038C0000840FFF7D9BE00BF740100213C58000139
:1038D000C84B000110B5174BD3F8002152B100209E
:1038E000C3F80001D3F800210122C3F80823124BCA
:1038F0001B6898470F4BD3F804218AB10022C3F804
:103900000421D3F80421D3F81824D3F8181402F0B2
:103910000302012A4FF0020103D1C3F818159A607F
:1039200010BDC3F80813044B0120BDE810401B680C
:10393000184700BF005000417401002101460148B2
:10394000FFF77EBE28000021044AD2F80034DB07CE
:10395000FBD50160BFF35F8F704700BF00000841D7
:1039600008B500F17F43B3F5802F04D2C0F30A03FA
:1039700063B10E4819E00E490E484FF4837200F00F
:1039800073FB4FF483710A4800F067FB02220A4B75
:10399000C3F804254FF0FF320260D3F80024D207A9
:1039A000FBD500220548C3F8042508BD0A00AD0B6D
:1039B000C2580001C84B0001000008410000AD0BD7
:1039C000F8B50D460121044600F037FE50B9104904
:1039D0004FF4CA720F4800F047FB4FF4CA710C480D
:1039E00000F03BFB14F0030708D0094940F29512A0
:1039F000084800F039FB40F29511F0E7064E2046EA
:103A0000C6F804152946FFF79FFFC6F80475F8BDF0
:103A1000C2580001C84B000100000841C10708B5A9
:103A20000AD50949094840F2EB1200F01DFB40F2AB
:103A3000EB11054800F011FB20F003031B6882071F
:103A40000CBF98B2180C08BDC2580001C84B000149
:103A500073B504460D464FF02003EFF3118683F350
:103A60001288BFF36F8F0022042896BF164B174BA6
:103A700053F82030009245210246154800F002FB21
:103A80003DB1EB69C3F308031BB14521114800F0B8
:103A9000F9FA00224521104B104800F0F3FA2946AC
:103AA0002046FFF78BFA042C08D10D490D489322CC
:103AB00000F0DAFA93210A4800F0CFFA86F3118871
:103AC000BFF36F8F02B070BDB8490001FE5800010E
:103AD0000C590001395900015F5900016759000173
:103AE00084590001C84B00010F4B70B553F82040BA
:103AF000013053F82060A64200D870BDD4E90035EB
:103B0000284698476DB138B10028B8BF4042FF2819
:103B1000A8BFFF20EB681870EA68537843F00103F0
:103B200053700834E7E700BFCC490001012208B513
:103B3000084B03201A70FFF7D7FF00F00FF904209D
:103B4000FFF7D2FFFDF72CF8034A137B23F00103A4
:103B5000137308BD850100216000002108B50348EA
:103B6000034A0021121A00F090FD08BD4000002118
:103B70008801002108B50020FFF7B6FF164B03F5BA
:103B8000006282F3088883F30A880025E023134C3F
:103B900084F82230E57725766576A57684F820507E
:103BA000636A43F4E023636284F82350FEF78EFADD
:103BB000FDF7AEFF4FF0FF33A362E36200F059FD63
:103BC0000120FFF791FF0220FFF78EFF2B462A46C8
:103BD00029460348FEF74EF88801002100ED00E079
:103BE0002D3B000108B50648064A0749121A00F0A5
:103BF0004EFDBDE80840054A0549064800F047BDAE
:103C0000000000213A000021285A000100000000B5
:103C1000285A000100000021034B1B680BB900F07B
:103C20000ABC0020704700BF7C01002110B50E4B7C
:103C30001C689C4204D1FFF7EFFF6FF0004010BDFD
:103C4000FFF7EAFF002CF8D0D4E904321B1A62EB2C
:103C5000E072B3F1004F72F10001EEDA002AACBF5E
:103C600018460020EBE700BF2C00002130B570B1F2
:103C70000B4B5B6898420AD0036843B1D3E9042137
:103C8000D0E90445121941EB0501C3E90421D0E94B
:103C9000003213605A600023C0E9003330BD00BF1A
:103CA0002C0000212DE9F84303464FF02002EFF3EA
:103CB000118482F31288BFF36F8F254FDFF8949041
:103CC000D9F80000DFF890C048453B604FEAE37543
:103CD000DCE9001E0CD058B1D0E90486434575EBF1
:103CE000060217DAB8EB030266EB0506C0E9042604
:103CF00059184EEB0505CCE9001500253D60FFF78E
:103D000095FF294600F096FB84F31188BFF36F8F6F
:103D1000BDE8F88318EB01014EEBE8730022CCE913
:103D200000130023C0E90423FFF7A0FF84F31188E8
:103D3000BFF36F8F836898474FF02003EFF3118430
:103D400083F31288BFF36F8F3B68A3EB0803B7E7D9
:103D50007C0100212C000021D8000021014800F046
:103D60009EB800BFF35900013F2A2DE9F0411746E4
:103D700053D905460C46A2F1400626F03F064036D0
:103D8000DFF89C800E44236840341BBA2B6454F83F
:103D90003C3C41461BBA6B6454F8383C28461BBA7D
:103DA000AB6454F8343C1BBAEB6454F8303C1BBA97
:103DB0002B6554F82C3C1BBA6B6554F8283C1BBA95
:103DC000AB6554F8243C1BBAEB6554F8203C1BBA95
:103DD0002B6654F81C3C1BBA6B6654F8183C1BBA93
:103DE000AB6654F8143C1BBAEB6654F8103C1BBA93
:103DF0002B6754F80C3C1BBA6B6754F8083C1BBA91
:103E0000AB6754F8043C1BBAEB67FCF761FAB442A9
:103E1000B9D107F03F00BDE8F0811046BDE8F08160
:103E2000E44900010A4610B514681A4924BA04642A
:103E3000546824BA4464946824BA8464D46824BA64
:103E4000C464146924BA0465546924BA4465946945
:103E500024BA8465D46924BAC465146A24BA046691
:103E6000546A24BA4466946A24BA8466D46A24BA2A
:103E7000C466146B24BA0467546B24BA4467946B09
:103E800024BA8467D26B12BAC267FCF721FA002009
:103E900010BD00BFE44900017047002070470FB417
:103EA00007B504A951F8040B0191FCF7FFFE03B01C
:103EB0005DF804EB04B07047038B13F0070305D1E2
:103EC0000368002B0CBF002003207047022B05D194
:103ED000408BB0FA80F0400980007047012B05D17B
:103EE0000368002B0CBF002005207047002070479E
:103EF00010B50C4600B111B96FF0150010BD081DCA
:103F000000F03DF80028F9D1A368032BF6D9F3E7B8
:103F10002DE9F0410D4607461946281D90461E46DC
:103F2000FDF7B8F8044638B13346424629463846CC
:103F3000A446BDE8F0416047BDE8F08110B44FF001
:103F40002004EFF3118284F31288BFF36F8F416175
:103F500010BC0121FCF7B8BE38B50C46054658B177
:103F600051B10B6843B14B6833B11C22002100F002
:103F70001AF900202C6138BD6FF01500FBE70346ED
:103F800058B1426802F00302012A03D0032A04D187
:103F9000026812B10020986070476FF015007047FA
:103FA0002DE9F84F9A46D37880466F2B0F46154679
:103FB000A3F1410B29D024D8582B0CBF10260A2678
:103FC000DDF828903246002340463946FCF738F9A0
:103FD000092AD4B21ED83034B045E4B277F10007D4
:103FE00009F8014D01D3D14511D82B789B0605D591
:103FF000082E15D1AB7843F00803AB704846BDE8F6
:10400000F88F03F0F703702BD7E70826D8E7804630
:104010000F46D7E7BBF1190F94BF37345734DBE7AE
:10402000102EEBD1AB7843F01003E6E72DE9F04119
:104030000746884615461E461446B44205D30EB1BF
:10404000601B08E02378002BFAD0414614F8010BDE
:10405000B8470028F1DABDE8F081404080F31188CC
:104060004FF0040002DF70470FB407B504A951F800
:10407000040B0191FCF71AFE03B05DF804EB04B0E9
:10408000704770470FB407B504A951F8040B0191AC
:10409000FCF70CFE03B05DF804EB04B0704708B504
:1040A0008368DB689847006808BD2DE9F0478946BA
:1040B00016469846044698B3826803691344826999
:1040C0003344934230D80025D4E90170A6EB050AA9
:1040D0003F1ABA4515D2B54209D223685246184450
:1040E00009EB050100F054F8A3685344A360B8F14C
:1040F000000F1CD0A068A8B12046BDE8F047FDF72E
:1041000049BC23683A46184409EB050100F040F821
:1041100063682046A360FDF73DFC18B93D44D3E732
:104120006FF00D00BDE8F0876FF00B00FAE7404636
:10413000F8E701460068FDF703BD00210120FDF707
:10414000FFBC08B5FDF76CFDBDE80840FDF7C4BD38
:10415000034600201A5C02B970470130FAE70346B3
:1041600000201A5C0AB1884200D170470130F8E79C
:1041700010B55AB10139841810F8012B11F8013F1C
:10418000A04201D09A42F7D0D01A10BD1046FCE7E9
:1041900010B5431E0A44914200D110BD11F8014BE5
:1041A00003F8014FF7E70346C9B20244934200D136
:1041B000704703F8011BF9E74FF0FF3070474FF0ED
:1041C0002003EFF3118283F31288BFF36F8F03682C
:1041D00003F0C00343F00203036082F31188BFF3CE
:1041E0006F8F7047F8B5069F0469C9B24FF020057C
:1041F000EFF3118685F31288BFF36F8F0C256943A7
:104200000C44256C05F0070CBCF1010F0BD12764A1
:1042100086F31188BFF36F8FC4E90E2343685B58A0
:1042200098470020F8BD05F0C005AF4286F311881D
:10423000BFF36F8F0CBF6FF077004FF0FF30F1E7E7
:1042400013B580240094FFF7CDFF02B010BD6FF0CE
:104250008500704710B41C240069CBB203FB040036
:10426000002110BC10470020FFF7BEBA0020FFF766
:1042700017BB8022FEF708B838B505460C4600F09B
:10428000F0F9002D07DBA84205D9401B84428CBF02
:104290000020012038BD0020FCE7F7B51C460023B4
:1042A000164682682360A3600D461369694601AA19
:1042B0009847019B5A1E01921BB96FF0150003B07D
:1042C000F0BD0098A26847682168676085B9B31A95
:1042D000D0F800C0634528BF634603FB07111A44AA
:1042E0002160A26002689A4206D808300090E0E798
:1042F0006B1AB3FBF7F3EBE70020E0E7134600226D
:10430000FFF7CBBF2DE9F0470024836886B08846CD
:1043100091461B6902AA01A99847A2462546029B1D
:10432000AB4202D806B0BDE8F0870026019F07EB3C
:10433000C5077B6804933A680AEB0603B24202D8C9
:104340009A460135EBE749460394059303A8C04715
:104350000028E7D0049B01361C44ECE70B460269B9
:10436000D2E9010183E803000020704743681B681D
:10437000D3F88004C3F880047047436802691B685F
:10438000D3F8100150B10020526912780A70C3F8B6
:104390001001D3F8102101221A6070474FF0FF304E
:1043A000704702680346D2F8580140B95B689B0722
:1043B00006D4D2F82001003818BF01207047012030
:1043C000704742681368D3F80413C90518D5D3F8A9
:1043D0002011A9B14FF02000EFF3118180F3128872
:1043E000BFF36F8FD3F8200130B10020C3F8200154
:1043F000D3F820010120D86081F31188BFF36F8FBB
:104400005268D20615D54FF02001EFF3118281F3E7
:104410001288BFF36F8FD3F8581111B10021C3F880
:1044200000154FF48001C3F8081382F31188BFF31D
:104430006F8F704770470020704708B5FEF73EFB4E
:1044400008BD30B543681360057A446804EBC504C1
:10445000A34202D36FF0010030BD5C798C4201D0E1
:104460000833F0E70020F7E72DE9F04F914680464A
:10447000012685B000EB8105454503D1002005B03C
:10448000BDE8F08FD8F8003003F07F07C3F3432472
:104490007F2F4FEA134308BF4FF0FF37032B3FD85E
:1044A000DFE803F0020F383BC9F80C7503A8039747
:1044B000FEF7AAFC039B4FF0010B06FA03F383609F
:1044C00003E0C9F814754FF0000B58F8043B03A83B
:1044D00003F40052002A0EBFDA464FF0010A4FF0F3
:1044E000000B01930397FEF78FFC039A019B00EBEF
:1044F0008200D0F80012C3F3C112230243EA820300
:1045000043EA0B0301F0E042134343EA4A03C0F8D5
:104510000032B1E7C9F80875C8E7C9F81075D2E7E5
:104520006FF08500ABE70222FEF7B8BC00207047B1
:104530000020704708B5FFF7F9FF08B9FFF7F8FF4B
:1045400008BD30B589B0154601230A4601466846C4
:1045500000F00EF8044640B9202269462846FBF7D1
:1045600089FE002808BF6FF06404204609B030BD02
:1045700008B5FCF795F9002008BD13B5044658B1FD
:1045800001200DF1060100F043F818B9BDF806301E
:104590005B08238002B010BD6FF01500FAE770B51C
:1045A000054608460C46FEF789FD214602460123D2
:1045B0002846BDE87040FEF791BD2DE9F8430D4651
:1045C0001646FEF799FE0446F8B1F5B10230FFF742
:1045D00025FA00278146B8460434B94507D8002497
:1045E00006B134600020A5F80080BDE8F8832046BD
:1045F000FFF714FAC3439BB2A21C002BF0D09845DE
:1046000038BF984614460137E7E76FF01500ECE72E
:104610000022FFF7D2BF4FF000535868704703469F
:104620005A6B00233C309A4200D17047C168013375
:104630000844F8E7004700F032B8034603F17F4230
:10464000B2F5802F08460AD351B103F17E4000F540
:104650000040B0F5607F2CBF002001207047012092
:1046600070474FF4802070474FF4006070478020FF
:104670007047704740B1C368587810F001001EBF02
:104680001878B0FA80F040097047FFF78CBDFFF74B
:104690007FBDEFF30580003818BF0120704708B1D7
:1046A000FDF72EB9704700005CBFFF7F01000000DE
:1046B00031180001000000002D230001E846000130
:1046C000A129000100470001C925000100000000E8
:1046D000392D0001000000003126000118470001BB
:1046E0002934000100000000BA520001F84800011E
:1046F0001049000134000021080100212C4800016C
:10470000CC530001484900017C49000138000021D8
:1047100008000021264800014C5300010000000061
:104720002C49000136000021000000002048000153
:10473000000000003B410001000000003B4100017F
:10474000000000003B410001000000003B4100016F
:10475000000000003B410001D53800013546000152
:10476000000000003B410001000000003B4100014F
:10477000000000003B410001000000003B4100013F
:10478000000000003B410001000000003B4100012F
:10479000000000003B410001000000003B4100011F
:1047A000000000003B410001000000003B4100010F
:1047B000000000003B410001000000003B410001FF
:1047C000000000003B41000100470001C34300011D
:1047D000000000003B410001000000003B410001DF
:1047E00000000000012B0001000000003B4100011F
:1047F000000000003B410001000000003B410001BF
:10480000000000003B410001000000003B410001AE
:10481000000000003B410001000000003B4100019E
:1048200000800080FF7F00800080FF7F008000808C
:10483000FF7FFFFFAD58000100000000B8580001E5
:10484000000000008C4D000103000000954B0001AA
:1048500003000000D5520001030000009154000144
:10486000030000006653000103000000F05900013E
:1048700003000000D857000103000000374C00017E
:1048800003000000DA53000103000000FFFFFFFFF8
:10489000DEE61E284CBBCE8F02350000DEE61E2869
:1048A0004CBBCE8F02350000DEE61E288384518685
:1048B00002350100DEE61E28EAAC45B802350000EC
:1048C000DEE61E284CBBCE8F023500000000000043
:1048D0000338FDD87047000000000000000200000F
:1048E0000004000000080000001000001122000178
:1048F000FD220001000000000D24000171240001D0
:10490000C9520001674200016D420001CF5200010F
:104910004F420001734200014142000100000000CB
:1049200055220001000000000000000025270001C2
:10493000B926000149260001292600011926000197
:1049400004000000FF0000000030014102000000F0
:104950000000000058490001003001416449000195
:10496000010000006C49000104000000210000006B
:104970000B000200A00101008A0103007B4300013B
:10498000612700016D430001252800015D430001FE
:104990000000000000020000000400000008000009
:1049A00000100000000000000002000000040000F1
:1049B0000008000000100000A6590001B4590001D1
:1049C000C8590001D7590001E3590001B046000160
:1049D000B0460001D0460001D8460001E84600017B
:1049E000E8460001982F8A4291443771CFFBC0B549
:1049F000A5DBB5E95BC25639F111F159A4823F92AA
:104A0000D55E1CAB98AA07D8015B8312BE85312402
:104A1000C37D0C55745DBE72FEB1DE80A706DC9BC3
:104A200074F19BC1C1699BE48647BEEFC69DC10F6F
:104A3000CCA10C246F2CE92DAA84744ADCA9B05CAB
:104A4000DA88F97652513E986DC631A8C82703B06E
:104A5000C77F59BFF30BE0C64791A7D55163CA067C
:104A600067292914850AB72738211B2EFC6D2C4D88
:104A7000130D385354730A65BB0A6A762EC9C28176
:104A8000852C7292A1E8BFA24B661AA8708B4BC20C
:104A9000A3516CC719E892D1240699D685350EF436
:104AA00070A06A1016C1A419086C371E4C774827ED
:104AB000B5BCB034B30C1C394AAAD84E4FCA9C5B63
:104AC000F36F2E68EE828F746F63A5781478C884B4
:104AD0000802C78CFAFFBE90EB6C50A4F7A3F9BE96
:104AE000F27871C6466C61736820646576696365A7
:104AF000206E6F742072656164790A004661696C8A
:104B0000656420746F2070726F7465637420623006
:104B10006E20666C6173682C2063616E63656C2027
:104B2000737461727475700A0D00556E61626C6504
:104B300020746F2066696E642076616C69642066FB
:104B400069726D7761726520696E7369646520258D
:104B5000700A0D004661696C656420746F20747280
:104B6000616E7366657220696D6167653A202564C0
:104B70000A0D004661696C656420746F2070726F65
:104B8000746563742061707020666C6173683A208C
:104B900025640A0D0063627072696E74665F7061ED
:104BA000636B61676500574553545F544F504449E8
:104BB000522F7A65706879722F6C69622F6F732F2C
:104BC0006F6E6F66662E6300415353455254494FD2
:104BD0004E204641494C20402025733A25640A0066
:104BE000574553545F544F504449522F7A6570686B
:104BF00079722F6C69622F6F732F6E6F746966798B
:104C00002E6300286E696C290025633A20416E6F7F
:104C10006D616C7920313630207472696767657216
:104C200020636F6E646974696F6E73206465746568
:104C3000637465642E0A00736F630025633A204233
:104C400075666665722073697A652069732062698A
:104C500067676572207468616E20706167650A001D
:104C600025633A204572726F722025642077686947
:104C70006C652067657474696E6720706167652074
:104C8000696E666F0A0025633A204572726F722062
:104C90002564207768696C652065726173696E6749
:104CA00020706167650A0025633A2073747265613C
:104CB0006D5F666C6173685F65726173655F70617B
:104CC000676520657272202564206F66667365745F
:104CD0003D30782530387A780A0025633A20666CB2
:104CE0006173685F7772697465206572726F722094
:104CF0002564206F66667365743D30782530387A98
:104D0000780A0025633A20666C61736820726561D9
:104D100064206661696C65643A2025640A00256335
:104D20003A2063616C6C6261636B206661696C65DB
:104D3000643A2025640A0025633A20427566666558
:104D4000722073697A65206973206E6F7420616CBC
:104D500069676E656420746F206D696E696D616C42
:104D60002077726974652D626C6F636B2D73697A3D
:104D7000650A0025633A20496E636F727265637439
:104D800020706172616D657465720A0053545245FA
:104D9000414D5F464C4153480025633A2072302F05
:104DA00061313A2020307825303878202072312F38
:104DB00061323A2020307825303878202072322F26
:104DC00061333A20203078253038780A0025633A5C
:104DD0002072332F61343A20203078253038782003
:104DE0007231322F69703A2020307825303878209F
:104DF0007231342F6C723A20203078253038780A9E
:104E00000025633A2020787073723A20203078258C
:104E10003038780A0025633A204661756C74696EF3
:104E20006720696E737472756374696F6E20616454
:104E3000647265737320287231352F7063293A20AC
:104E40003078253038780A00574553545F544F5016
:104E50004449522F7A65706879722F617263682FA6
:104E600061726D2F636F72652F6161726368333297
:104E70002F6972715F6D616E6167652E63002563D6
:104E80003A202A2A2A2A2A205553414745204641BA
:104E9000554C54202A2A2A2A2A0A0025633A20201F
:104EA000204469766973696F6E206279207A657231
:104EB0006F0A0025633A202020556E616C69676E89
:104EC0006564206D656D6F727920616363657373CE
:104ED0000A0025633A202020537461636B206F76AB
:104EE0006572666C6F772028636F6E7465787420C6
:104EF00061726561206E6F742076616C6964290A45
:104F00000025633A2020204E6F20636F70726F631C
:104F10006573736F7220696E737472756374696FF1
:104F20006E730A0025633A202020496C6C65676126
:104F30006C206C6F6164206F66204558435F52455A
:104F40005455524E20696E746F2050430A002563F9
:104F50003A202020496C6C6567616C207573652070
:104F60006F662074686520455053520A0025633AE5
:104F7000202020417474656D707420746F206578F2
:104F8000656375746520756E646566696E65642019
:104F9000696E737472756374696F6E0A0025633A83
:104FA000202A2A2A2A2A20425553204641554C5469
:104FB000202A2A2A2A2A0A0025633A20202053740C
:104FC00061636B696E67206572726F720A00256398
:104FD0003A202020556E737461636B696E6720659B
:104FE00072726F720A0025633A2020205072656346
:104FF00069736520646174612062757320657272E3
:105000006F720A0025633A20202042464152204117
:105010006464726573733A20307825780A002563DA
:105020003A202020496D7072656369736520646160
:10503000746120627573206572726F720A00256355
:105040003A202020496E737472756374696F6E2004
:10505000627573206572726F720A0025633A202AA6
:105060002A2A2A2A204D5055204641554C54202AA0
:105070002A2A2A2A0A0025633A20202053746163D1
:105080006B696E67206572726F722028636F6E7431
:105090006578742061726561206D6967687420624B
:1050A00065206E6F742076616C6964290A0025633F
:1050B0003A2020204461746120416363657373204A
:1050C00056696F6C6174696F6E0A0025633A20201F
:1050D000204D4D46415220416464726573733A20FD
:1050E000307825780A0025633A202020496E7374B1
:1050F00072756374696F6E204163636573732056C4
:10510000696F6C6174696F6E0A00574553545F5440
:105110004F504449522F7A65706879722F617263DB
:10512000682F61726D2F636F72652F6161726368A2
:1051300033322F636F727465785F6D2F6661756CA3
:10514000742E6300526573657276656420457863DA
:10515000657074696F6E20280053707572696F7581
:105160007320696E7465727275707420284952518B
:10517000200025633A20535053454C20696E20741B
:105180006872656164206D6F646520646F6573206B
:105190006E6F7420696E646963617465205053504A
:1051A0000A0025633A202A2A2A2A2A204841524402
:1051B000204641554C54202A2A2A2A2A0A002563CF
:1051C0003A202020427573206661756C74206F6EE2
:1051D00020766563746F72207461626C65207265FD
:1051E00061640A0025633A202020446562756720C7
:1051F0006576656E740A0025633A20202046617545
:105200006C7420657363616C6174696F6E202873C0
:1052100065652062656C6F77290A0025633A204135
:105220005243485F4558434550542077697468207D
:10523000726561736F6E2025780A0A0025633A2033
:105240002A2A2A2A2A204465627567206D6F6E69B2
:10525000746F7220657863657074696F6E202A2A96
:105260002A2A2A0A0025633A202A2A2A2A2A2025BD
:105270007320256429202A2A2A2A2A0A00574553FE
:10528000545F544F504449522F7A65706879722F99
:10529000647269766572732F636C6F636B5F636FA3
:1052A0006E74726F6C2F636C6F636B5F636F6E7481
:1052B000726F6C5F6E72662E6300636C6F636B401F
:1052C0003431303035303030006866636C6B006CE0
:1052D00066636C6B00636C6F636B5F636F6E74729D
:1052E0006F6C0025633A20756E616C69676E65644A
:1052F00020616464726573733A2030782530386CAD
:10530000783A257A750A0025633A20696E76616CD1
:10531000696420616464726573733A203078253063
:10532000386C783A257A750A0025633A206E6F74D6
:1053300020776F72642D616C69676E65643A203006
:10534000782530386C783A257A750A00666C617376
:10535000682D636F6E74726F6C6C6572403431309F
:10536000383030303000666C6173685F6E72660092
:1053700025633A204661696C656420746F20616C16
:105380006C6F6361746520505049204368616E6E94
:10539000656C0A00574553545F544F504449522F8F
:1053A0006D6F64756C65732F68616C2F6E6F7264BE
:1053B00069632F6E7266782F68656C706572732FE3
:1053C0006E7266785F677070692E680075617274BE
:1053D00040343130313330303000756172745F6E7B
:1053E0007266785F756172746500574553545F54F7
:1053F0004F504449522F6D6F64756C65732F68610F
:105400006C2F6E6F726469632F6E7266782F68619D
:105410006C2F6E72665F6770696F2E680057455318
:10542000545F544F504449522F6E72662F6C69621C
:105430002F6670726F746563742F6670726F746517
:1054400063745F61636C2E6300574553545F544F20
:10545000504449522F6D6F64756C65732F68616C91
:105460002F6E6F726469632F6E7266782F68616C3D
:105470002F6E72665F61636C2E680025633A20525E
:105480006573657474696E672073797374656D0AEA
:1054900000666174616C5F6572726F7200426F6F5B
:1054A00074696E67202830782578292E0D0A004906
:1054B0006E76616C6964206669726D7761726520D1
:1054C000696E666F20666F726D61742E0A0D0054EE
:1054D0006865206669726D7761726520646F6573B7
:1054E0006E27742062656C6F6E672061742064653E
:1054F0007374696E6174696F6E20616464722E0AE0
:105500000D0073726320616E6420647374206D7586
:10551000737420626520657175616C20666F7220FE
:105520006C6F63616C2063616C6C732E0A0D0046B6
:1055300069726D7761726520696E666F20646F6550
:10554000736E277420706F696E7420746F20697495
:1055500073656C662E0A0D00466972776D6172651F
:1055600020686173206265656E20696E76616C6982
:1055700064617465643A20307825782E0A0D004302
:10558000616E6E6F74207265616420746865206658
:1055900069726D776172652076657273696F6E2EC0
:1055A0002025640A0D00576520617373756D6520B1
:1055B000746869732069732064756520746F207442
:1055C0006865206669726D776172652076657273B1
:1055D000696F6E206E6F74206265696E6720656EFC
:1055E00061626C65642E0A0D004669726D776172A6
:1055F000652076657273696F6E202825752920698C
:105600007320736D616C6C6572207468616E206DBF
:105610006F6E6F746F6E696320636F756E74657201
:1056200020282575292E0A0D004669726D77617252
:105630006520696E666F206973206E6F74207769CC
:105640007468696E207369676E6564207265676946
:105650006F6E2E0A0D00426F6F7420616464726574
:105660007373206973206E6F742077697468696E34
:10567000207369676E656420726567696F6E2E0AB4
:105680000D0052657365742068616E646C657220EC
:105690006973206E6F742077697468696E2073690E
:1056A000676E656420726567696F6E2E0A0D004330
:1056B0006F756C64206E6F742066696E642076610D
:1056C0006C6964206669726D776172652076616CC1
:1056D00069646174696F6E20696E666F2E0A0D00D1
:1056E00056616C69646174696F6E20696E666F20C3
:1056F000646F65736E27742062656C6F6E672074CB
:105700006F2074686973206669726D776172652EA7
:105710000A0D00626C5F63727970746F5F696E6905
:105720007428292072657475726E65642025642E54
:105730000A0D004669726D776172652076616C6949
:10574000646174696F6E206661696C656420776955
:105750007468206572726F722025642E0A0D0046EF
:1057600069726D7761726520686173682076657211
:1057700069666965642E0A0D0025633A20737472A8
:1057800065616D5F666C6173685F696E69742066E0
:1057900061696C65643A2025640A0025633A2073C8
:1057A000747265616D5F666C6173685F6275666671
:1057B000657265645F7772697465206661696C3AC9
:1057C0002025640A0025633A205472616E73666571
:1057D0007220646F6E650A00706364004552524F18
:1057E000523A2043616E6E6F742066756C66696C08
:1057F0006C204558545F415049207265717565733E
:10580000742E0D0A005741524E494E473A204F70B0
:1058100074696F6E616C204558545F415049207225
:10582000657175657374206E6F742066756C66693A
:105830006C6C65642E0D0A0001000000574553543E
:105840005F544F504449522F6D6F64756C65732FD0
:1058500068616C2F6E6F726469632F6E7266782F49
:10586000647269766572732F7372632F6E726678D5
:105870005F636C6F636B2E6300574553545F544FE7
:10588000504449522F6D6F64756C65732F68616C5D
:105890002F6E6F726469632F6E7266782F68616C09
:1058A0002F6E72665F636C6F636B2E68004E52469C
:1058B000585F434C4F434B004E5246585F44505044
:1058C0004900574553545F544F504449522F6D6F10
:1058D00064756C65732F68616C2F6E6F7264696399
:1058E0002F6E7266782F647269766572732F737289
:1058F000632F6E7266785F6E766D632E6300556EF1
:105900006B6E6F776E206572726F720025633A203E
:105910003E3E3E205A455048595220464154414C43
:10592000204552524F522025643A202573206F6E35
:10593000204350552025640A0025633A20466175AE
:105940006C7420647572696E6720696E746572721A
:105950007570742068616E646C696E670A0A007500
:105960006E6B6E6F776E0025633A204375727265B9
:105970006E74207468726561643A20257020282551
:1059800073290A00574553545F544F504449522FCE
:105990007A65706879722F6B65726E656C2F6661BF
:1059A00074616C2E63004350552065786365707494
:1059B000696F6E00556E68616E646C656420696E17
:1059C0007465727275707400537461636B206F76C6
:1059D0006572666C6F77004B65726E656C206F6FD9
:1059E0007073004B65726E656C2070616E69630048
:1059F0006F73002A2A2A20426F6F74696E67205ADB
:105A00006570687972204F53206275696C642076E6
:105A1000332E322E39392D6E637332202A2A2A0A08
:105A200000000000000000019B3E0001B9410001A0
:105A30000000000000C2010000010300000000009F
:105A40008401002183010021000000000090D003A8
:105A5000FFFFFFFF2C0000212C00002100000000B0
:065A6000000015E015E056
:1085A800008800010088000101000000FFFFFFFFB4
:1085B800A00A14E2B002C51491C99F96A9D18FCF21
:0885C800010001000100F000B8
:10880000A05E002149D50201213203011DD50201DC
:108810001DD502011DD502011DD502010000000079
:1088200000000000000000000000000091D20201E2
:108830001DD502010000000039D202011DD5020140
:1088400011D3020111D3020111D3020111D302018C
:1088500011D3020111D3020111D3020111D302017C
:108860009F38030111D3020111D3020111D3020178
:108870005538030111D3020111D3020111D30201B2
:1088800011D302018938030111D3020111D302016E
:1088900011D3020111D3020111D3020111D302013C
:1088A00011D3020111D3020111D3020111D302012C
:1088B00011D3020111D302010000000000000000EA
:1088C00000000000000000000000000000000000A8
:1088D0000000000000000000000000000000000098
:1088E0000000000000000000000000000000000088
:1088F0000000000000000000000000000000000078
:108900000000000000000000000000000000000067
:108910000000000000000000000000000000000057
:108920000000000000000000000000000000000047
:108930000000000000000000000000000000000037
:108940000000000000000000000000000000000027
:108950000000000000000000000000000000000017
:108960000000000000000000000000000000000007
:1089700000000000000000000000000000000000F7
:1089800000000000000000000000000000000000E7
:1089900000000000000000000000000000000000D7
:1089A00000000000000000000000000000000000C7
:1089B00000000000000000000000000000000000B7
:1089C00000000000000000000000000000000000A7
:1089D0000000000000000000000000000000000097
:1089E0000000000000000000000000000000000087
:1089F0000000000000000000000000000000000077
:108A0000DEE61E284CBBCE8F023500003C00000085
:108A10003CDC020001000000008800010088000129
:108A2000FFFF0291000000000000000000000000B5
:108A300000000000000000000000000053B94AB927
:108A4000002908BF00281CBF4FF0FF314FF0FF3056
:108A500000F00CB8ADF1080C6DE904CE1FF06CFB12
:108A6000DDF804E0DDE9022304B07047704700BF81
:108A70002DE9F00791E8F807B2E802105B1854EB13
:108A80000C04B2E802104D4156EB0C06B2E802109D
:108A90004F4158EB0C08B2E8021059EB01095AEBB0
:108AA0000C0A80E8F80780410130BDE8F007704704
:108AB0002DE9F00791E8F807B2E802105B1A74EBB1
:108AC0000C04B2E802108D4176EB0C06B2E80210FD
:108AD0008F4178EB0C08B2E8021079EB01097AEBD0
:108AE0000C0A80E8F80780414042BDE8F007704773
:108AF0002DE9F007524290E87800B1E8800717406E
:108B0000DB1918EA020854EB080419EA020955EBCC
:108B100009051AEA020A56EB0A0678C090E87800BE
:108B2000B1E8800717407B4118EA020854EB0804BB
:108B300019EA020955EB09051AEA020A56EB0A0678
:108B400078C080410130BDE8F00770472DE9F0079B
:108B5000524290E87800B1E880071740DB1B18EA22
:108B6000020874EB080419EA020975EB09051AEA10
:108B7000020A76EB0A0678C090E87800B1E8800730
:108B80001740BB4118EA020874EB080419EA02090D
:108B900075EB09051AEA020A76EB0A0678C08041ED
:108BA0004042BDE8F00770472DE9F00152424FF016
:108BB000040890E8300091E8C000A31B1340E41AB9
:108BC000F618EB1B1340ED1AFF1830C0C0C1B8F106
:108BD0000108EED1BDE8F001704700BF00B592E892
:108BE000DC072DE9DC07B1E8805702B4A7FB02518E
:108BF0000A95A8FB020B09180020E7FB03105BEBAA
:108C0000000B00204041E9FB02B00B91A8FB03518F
:108C1000401800214941EAFB02011BEB050B00252E
:108C2000E7FB04B568410025E7FB0605694100251F
:108C30006D41E8FB0615CDF830B0A9FB03B68919E4
:108C40000026EAFB0316754100267641ECFB03562D
:108C500010EB0B005FF0000BE8FB040B51EB0B017A
:108C60005FF0000BE9FB041B55EB0B055FF0000BFD
:108C7000EAFB045B56EB0B065FF0000B5BEB0B0BA8
:108C8000ECFB046B0D90ACFB0230059C2D18002012
:108C9000EEFB025046410020E9FB04605BEB000B59
:108CA00000204041EAFB04B05B180021E7FB0431DF
:108CB0004D410021E8FB0451069C4E410021E8FB98
:108CC00004615BEB010B0021E9FB04B14841002189
:108CD0004941EAFB04010E93A7FB0432079CB61836
:108CE0000022E7FB04625BEB020B0022E8FB04B20C
:108CF00050410022E9FB0402514100225241EAFBAB
:108D00000412049CED180023E9FB04535E41002388
:108D1000EAFB0463089C5BEB030B0023E7FB04B353
:108D200058410023E8FB040359410023E9FB0413E5
:108D30005A4100235B41EAFB04230F955DF8049B35
:108D400099E80006DDF80080A9FB08541BEB040B32
:108D50000024EAFB08B4DDF8108060410024ECFB3D
:108D6000080461410024EEFB081462410024E9FB81
:108D70000824634100246441EAFB0834DDF80480E0
:108D800076190025EEFB08655BEB050B0025E9FB7A
:108D900008B568410025EAFB0805DDF81480694143
:108DA0000025ECFB08156A410025EEFB08256B4108
:108DB0000025E9FB08356C4100256D41EAFB0845BB
:108DC0000F96DDF80880AEFB087680190026E9FBD7
:108DD000080671410026EAFB0816DDF8188072418A
:108DE0000026ECFB082673410026EEFB0836744192
:108DF0000026E9FB0846754100267641EAFB085645
:108E0000DDF80C801BEB070B0027ECFB08B7784163
:108E10000027EEFB080779410027E9FB08177A4194
:108E20000027EAFB0827DDF81C807B410027ECFBCC
:108E300008377C410027EEFB08477D410027E9FB0E
:108E400008577E4100277F41EAFB086708B000BD54
:108E50002DE9F14F87B0FFF7C1FEDDF81C8008F166
:108E6000200888E8FF00FFBC87E87F08BDE8F08F96
:108E700000B591E84C57A2FB02410194A2FB0345C7
:108E800024190020E2FB06506D417F4164180294D2
:108E90000021E2FB0801A3FB034B6541039500247D
:108EA000E3FB060440417F41091900246441E2FBD1
:108EB0000914FF0750EB0B0004900025E2FB0A4564
:108EC0005FF0000BE3FB081B49415FEA370714EB37
:108ED0000B045FF0000BE3FB094B55EB0B055FF058
:108EE000000B5BEB0B0BE2FB0C5BFF0F0020E2FBCC
:108EF0000EB000225141E6FB061205910021E6FB6F
:108F0000084164417F416D180021E3FB0A515BEB8E
:108F1000010B0021E3FB0CB1484100214941E3FB77
:108F20000E010023E6FB09531BEB030B0023E6FBBA
:108F30000AB358410023E6FB0C03594100235B416F
:108F4000E6FB0E13FF07544106946D417F41A8FBD9
:108F50000826554107950022E8FB09B25BEB0B0B95
:108F60007F4180180022E8FB0A0251410022E8FB01
:108F70000C125A4100235B41E8FB0E230024E9FB5D
:108F80000E340025E9FB0A1552190025E9FB0C25D2
:108F90006B410025EAFB0C356C4100256D41EAFB75
:108FA0000E45FF075BEB060B0026ECFB0E5640411F
:108FB000494152415B4164416D417641AEFB0EE84F
:108FC00048F100087F00A9FB0979784151EB0901BC
:108FD000AAFB0A7A7A4153EB0A03ACFB0C7C7C4176
:108FE00055EB0C0556EB0E0648F1000700BD00BF1F
:108FF0002DE9F14F87B0FFF73BFFDDF81C8008F14A
:10900000200888E8FF00FFBC87E87F08BDE8F08FF4
:1090100030B44FF0000310F8014B11F8015B013A36
:1090200084EA050443EA0403F5D1A3F101034FEAFE
:10903000D37030BC704700BF4FF0000310F8012B15
:10904000013943EA0203F9D1A3F101034FEAD370D6
:10905000704700BF30B411F8014B12F8015B6C404F
:1090600000F8014B013BF6D130BC70472DE9F00709
:1090700091E8F807B2E802105B1854EB0C04B2E870
:1090800002104D4156EB0C06B2E802104F4158EB6E
:109090000C08B2E8021059EB01095AEB0C0A89419D
:1090A000B3F1FF3374F1FF3475F1FF3576F100064B
:1090B00077F1000778F1000879F101097AF1FF3AB8
:1090C00051F100015B184C414D4156F1000657F13A
:1090D000000758F1000859EBD1795AEB010A80E8F2
:1090E000F807BDE8F00770472DE9F00791E8F807A9
:1090F000B2E802105B1A74EB0C04B2E802108D4166
:1091000076EB0C06B2E802108F4178EB0C08B2E85F
:10911000021079EB01097AEB0C0A89415B184C418A
:109120004D4156F1000657F1000758F1000859EB80
:10913000D1795AEB010A80E8F807BDE8F0077047DB
:1091400018EB040859EB05095AEB060A5BEB070B11
:109150005FF0000C4CF1000C18EB050859EB060908
:109160005AEB070A5BEB070B50EB0C005FF0000CAF
:1091700051EB0C0152EB0C0263414CF1000CB8EBCB
:10918000070879F100097AF1000A7BEB040BA8418A
:10919000B141A241B3416CF1000CBBEB050BB041F6
:1091A000B941AA41BB416CF1000C6FEAEC74B8EB19
:1091B000040879EB04097AEB040A7BF1000B70F1E7
:1091C000000071F1000172EBD472A3416CF1000C4C
:1091D00018EBEC7859EBEC795AEBEC7A5BF1000B7D
:1091E00050F1000451F1000552EBDC7653EBEC77C3
:1091F0004CF1000C18EBEC7059EBEC715AEBEC7283
:109200005BF1000354F1000455F1000556EBDC76E8
:1092100057EBEC77704700BF2DE9F14F87B0FFF7B0
:10922000DDFCDDF81080DDF81490DDF818A0FFF704
:1092300087FFBDE8000FFFF783FF03B05DF8048BE5
:1092400088E8FF00BDE8F08F2DE9F14F87B0FFF708
:109250000FFEDDF81080DDF81490DDF818A0FFF7A0
:109260006FFFBDE8000FFFF76BFF03B05DF8048BE5
:1092700088E8FF00BDE8F08F2DE9F047002386B0B5
:10928000704EC41C05460F46B27D24F00304CDE9A0
:10929000033333788DF812208DF80D307378F27E19
:1092A0008DF80E30B3788DF814208DF80F30327FA2
:1092B000F3788DF815208DF8103096F8202033794A
:1092C0008DF811300AB18DF81330002F03A94FF03B
:1092D00000080CBF2046002000F02EFF96F80090FA
:1092E00073780444C24699445FFA89F95FFA88F3B7
:1092F000994500F299800334002F4946524624F0E4
:10930000030414BF0020204601F08CF8B1782044FB
:1093100059B10330002F738A20F00304F27814BF90
:109320000020204601F020FA204496F821308BB12D
:10933000317C79B196F822300330002B20F0030401
:1093400014BFFF222522002F0CBF2046002001F071
:10935000A1FB20443C4B1B685BB1317949B1033020
:10936000002F327D20F0030414BF002020469847D0
:109370002044364B1B6853B1717D41B10330002F3F
:1093800020F0030414BF0020204698472044304BAF
:10939000D3F80080B8F1000F0FD0B17D69B1033070
:1093A000002F737E20F00304F27D009318BF00208D
:1093B000337E08BF2046C047204496F8203063B172
:1093C000317951B10330002FB27E20F0030414BF75
:1093D0000020204601F0F2FB2044737F6BB1033084
:1093E00020F0030457BB204619F020FA20464FF422
:1093F0008C72717F20F009FE2044B37F6BB1033083
:1094000020F00304E7B9204622F05BFB20464FF42E
:109410008C72B17F20F0F9FD2044073020F0070066
:10942000401B06B0BDE8F087337A08F10108F279F5
:10943000B179707920F08AFD824457E70020D6E7A1
:109440000020E4E7580700214C00002154000021CF
:10945000500000218FB572B61A4B5D6AE5B9BFF3B3
:109460004F8F1949194BCA6802F4E0621343CB606D
:10947000BFF34F8F00BFFDE7B4FBF6F4D3B2013268
:10948000002CF9D103F110026A4402F80C4C0A24B2
:1094900033B901A8A847E2E7044600220A26EDE70F
:1094A000013BDBB203F110020DEB0206C2B2B2FBCC
:1094B000F4F704FB17223032B0FBF4F006F80C2C62
:1094C000E6E700BF5807002100ED00E00400FA05C0
:1094D0001FB51A4C02A8237A8DF80930E3798DF86C
:1094E0000830A379ADF80C306379ADF80A3017F085
:1094F0000DFA18B1A7210320FFF7ACFFE36801A81C
:10950000019317F019FA08B1AB21F4E7012368467B
:109510008DF8003022F037F908B1AF21EBE7607E1B
:1095200017F01CFA08B1B821E5E7207E17F010FA11
:1095300008B1B921DFE704B010BD00BF5807002112
:1095400038B5054600283CD01DF01AF910B94FF087
:10955000FF3038BD1CF0D2FDB0F5FA7FF7D81A4CB9
:109560001A48656200F008FB19490220194A0023D5
:10957000194D84F8283084F8293084F8213084F893
:10958000223084F82030C4E9001241F64C52C4E97C
:109590000202124AC4E90452114AC4E90623EFF355
:1095A000108472B601F094FB0E4801F057FC18B11C
:1095B000C5210320FFF74EFF002CCAD162B620461A
:1095C000C7E76FF01500C4E758070021D1940001E8
:1095D00001010100001B1B0303001F00020000012A
:1095E00049000100E998000110B5002871D13D4CF7
:1095F00094F82830002B69D179B1002A6CD0013958
:109600000C2966D8DFE801F0071417272A4A5230E0
:1096100055585D363C001378237001210020FFF778
:109620002BFEB0F5803F5ADA012384F8293010BDB3
:1096300013786370F1E79378002B4DD0D378002B2B
:109640004AD013781A2B47D953781A2B44D910686B
:10965000C4F80500E1E71368E360DEE71378E27819
:10966000934239D3A370D8E71378A278934233D8C2
:10967000E370D2E71378A27893422DD8A375CCE794
:1096800013784BB35378013BDBB2F82B24D8138803
:109690009278A4F81730144B9A70BEE7137894F8B8
:1096A00021200AB1012B17D92374B6E713886382EE
:1096B000B3E713782371B0E71378012B0CD9237526
:1096C000ABE71378082B07D86375A6E74FF0FF3098
:1096D000ADE76FF02C00AAE76FF01500A7E76FF079
:1096E0000B00A4E7580700216F07002170B50D4655
:1096F0000646F0B1E9B111F007041AD100F04CF9B7
:10970000D0B130460E4E1DF07FF8214686F82A0073
:109710002846FFF7B1FD17F07DFA96F82A0021469A
:1097200017F0EEF9FFF7D4FE0123204686F8283023
:1097300070BD6FF01500FBE74FF0FF30F8E700BF9A
:109740005807002110B5094C94F828302BB117F0B8
:10975000F3F994F82A001DF073F801F0CDFA01F046
:1097600093FB002084F8280010BD00BF580700219B
:1097700050B1074B03F1140253F8041B934240F815
:10978000041BF9D1002070476FF01500704700BF2F
:10979000B05C0301074B93F8292010B532B993F858
:1097A00028401CB917F03EF9204610BD4FF0FF309D
:1097B000FBE700BF58070021074B93F8292010B59D
:1097C00032B993F828401CB917F040F9204610BD73
:1097D0004FF0FF30FBE700BF5807002110B50B4CDE
:1097E00094F829307BB994F8283063B994F8223082
:1097F00033B117F069F90123002084F8213010BD3E
:1098000017F046F9F7E74FF0FF30F8E75807002167
:10981000074B93F8292010B532B993F828401CB9AA
:1098200017F0B0F8204610BD4FF0FF30FBE700BF47
:1098300058070021074B93F8292010B532B993F847
:1098400028401CB917F090F8204610BD4FF0FF30AB
:10985000FBE700BF58070021074B93F8292010B5FC
:1098600032B993F828401CB921F0B5FF204610BD4D
:109870004FF0FF30FBE700BF58070021074B93F87C
:10988000292010B532B993F828401CB921F0A6FF61
:10989000204610BD4FF0FF30FBE700BF5807002106
:1098A000074B93F8292010B532B993F828401CB91A
:1098B00021F097FF204610BD4FF0FF30FBE700BFBF
:1098C00058070021074B93F8292010B532B993F8B7
:1098D00028401CB921F087FF204610BD4FF0FF3013
:1098E000FBE700BF5807002137B5114C256801A8D8
:1098F00001F080FA034618B1052816D035210BE097
:10990000019A022A05D0032AF1D1226852B92D21E9
:1099100002E022681AB928210420FFF79BFD23608A
:10992000A847E4E701202360FAE703B030BD00BF99
:109930008407002107C8024B83E807000020704716
:1099400088070021054B5B6810B51BB98C210420EA
:10995000FFF780FDBDE81040184700BF84070021D5
:10996000054B9B6810B51BB992210420FFF772FDCF
:10997000BDE81040184700BF84070021054BDB6895
:1099800010B51BB998210420FFF764FDBDE8104015
:10999000184700BF84070021044B586828B1986815
:1099A00018B1D868003818BF01207047840700211B
:1099B000014B1870704700BF940700212DE9F74351
:1099C000334D031D04462F4647F8043F95F80C31EC
:1099D0007BB195F80E2105F20D11204604260232C6
:1099E0001CF0A6FF002385F80C31304603B0BDE81B
:1099F000F083384605F0E0FC0228064604D12549EC
:109A000020461EF006FDF0E704283AD12B790A2BF8
:109A100015D13E2000F054F860B92B8901A96846A1
:109A2000ADF800301FF01EFA0028CFD0A721082083
:109A3000FFF710FD052000F08FF80028EDD0394623
:109A400020461EF093FD0028C0D094F8009094F8B2
:109A50000280484600F034F80028B7D0B9F13E0F34
:109A6000C3D1B8F1120F06D195F80E32022B02D0F5
:109A70002B78002BAAD0404600F06EF80028B4D115
:109A8000A4E70828B1D1034920461EF0FAFCACE750
:109A90009407002198070021074B4FF0FF3141F652
:109AA000FF72C3E9001205490022C1E900221F210B
:109AB000C3E90212704700BF00000021A409002181
:109AC0003F280CD801380B4BC0F3421200F01F00A6
:109AD00053F8223023FA00F000F001007047FF280D
:109AE00006D04038044BC0F3421200F01F00EFE7ED
:109AF0000120704700000021A4090021074B014606
:109B0000006849681A4603C240F48C221A6041F08A
:109B1000107242F4FF625A60704700BF00000021DB
:109B20000246024B0068516803C37047A409002134
:109B3000084B01460068496803F1080203C219692D
:109B400020EA010259699A60DA6822EA0102DA60C1
:109B5000704700BF000000210138064BC0F34212DD
:109B600000F01F0003EB82039B6823FA00F000F073
:109B70000100704700000021014B1860704700BFD2
:109B8000AC09002110B5FFF787FF0020FFF710FF99
:109B900021F049F8034B04461B6803B1984720465F
:109BA00010BD00BFAC09002138B5274C0546D4F8DC
:109BB000A432013306D1D4F8A8324FF6FF729BB21B
:109BC00093423ED0D4F8A032DB073AD5D4F8A42291
:109BD000D4F8A832C5F80120A5F80530C3F307234F
:109BE00063F03F03AB71D4F89032013323D0D4F843
:109BF000943201331FD0D4F8983201331BD0D4F8FB
:109C00009C32013317D0002001F03CFA98B9D4F807
:109C10009002D4F89412D4F89822D4F89C32C5F863
:109C20000700C5F80B10C5F80F20C5F81330012345
:109C300000202B7038BD10220021E81D1CF0EEFE24
:109C4000F5E70023F4E700BF0000FF0110B5102284
:109C5000002104461CF0E2FE10220021A0181CF096
:109C6000DDFE224BD3F8802201320BD1D3F88422BF
:109C7000013207D1D3F88822013203D1D3F88C22E4
:109C800001320BD0D3F88002D3F88412D3F88822A3
:109C9000D3F88C3220616161A261E361002001F0A0
:109CA000F1F9124B18B9D3F8A022D2071CD4D3F87B
:109CB000902201320BD1D3F89422013207D1D3F88C
:109CC0009822013203D1D3F89C3201330CD0074BD8
:109CD000D3F89002D3F89412D3F89822D3F89C3298
:109CE00020606160A260E360002010BD0000FF0101
:109CF00080B588B000AF786039603B681B88BB8353
:109D0000BB8BC3F30E037B837B68DB7C18461FF0A1
:109D1000D3F803463B837B681A883B8B1344FB8252
:109D20007B6818333B617B8B3A691344FB603B8B48
:109D3000FA68128892B21A44FB8A13445A1EFB8AAC
:109D400092FBF3F39BB2FA8A02FB03F37B817A8BDB
:109D50007B891344FB837B685B88FA8B9A420AD227
:109D6000B7F91C200A4B13401AB2B7F91E3013433F
:109D70001BB2FB8305E0BB8BDB439AB2044B134061
:109D8000FB833B68FA8B1A8000BF2037BD4680BD3D
:109D90000080FFFF80B483B000AF0346FB71FB7906
:109DA000064A32F8133003339BB223F003039BB20D
:109DB00018460C37BD4680BC704700BFF450030105
:109DC00080B483B000AF0023FB71254B1A78FB7978
:109DD0001344FB71224B5A78FB791344FB71204BDF
:109DE0001A7AFB791344FB711D4B9B78BB71FA798E
:109DF000BB79934238BF1346FB71194BDB787B71FB
:109E0000FA797B79934238BF1346FB71144B1B7967
:109E10003B71FA793B79934238BF1346FB71104B83
:109E20005B79FB70FA79FB78934238BF1346FB717C
:109E30000B4B9B79BB70FA79BB78934238BF1346C2
:109E4000FB71074BDB797B70FA797B78934238BFE3
:109E50001346FB71FB7918460C37BD4680BC704732
:109E6000B009002180B588B000AFF8600B467A6079
:109E7000FB72FB68002B0CBF01230023FB77FB7FE9
:109E8000002B01D0002301E007F10C03BB617968CE
:109E9000B8691FF012FD7861FB7F83F00103DBB22C
:109EA000002B06D0FB7AFA68044902339B000B446E
:109EB0005A607B6918462037BD4680BDB009002135
:109EC00080B586B000AF78600B46FB700023FB7551
:109ED00029E07B681B68033323F003031A467B6881
:109EE0001A60FB7D1846FFF755FF03461946FB7DB8
:109EF000114AD35C01FB03F33B61FB78002B01D0DB
:109F0000002301E07B681B68F97D3A691846FFF77A
:109F1000A9FFF8607B681A68FB681A447B681A60BE
:109F2000FB7D0133FB75FB7D082BD2D900BF00BF41
:109F30001837BD4680BD00BFB009002180B485B090
:109F400000AF78600B46FB701346BB700023FB73B9
:109F500032E07B681B68033323F003031A467B68F7
:109F60001A60BB7883F00103DBB2002B1AD0FB7BB5
:109F70007A68126815490C3341F823200023BB731B
:109F80000CE0FB7B114A0C3352F82320BB7B9B0077
:109F9000134400221A60BB7B0133BB73BA7BFB788E
:109FA0009A42EED37B681A68FB789B001A447B6860
:109FB0001A60FB7B0133FB73FB7B082BC9D900BF05
:109FC00000BF1437BD4680BC704700BFB0090021F8
:109FD00080B485B000AF0346FB710023FB81FB79A1
:109FE000012B02D1194B1B78FB81FB79082B07D180
:109FF000164B1B789AB2154B5B789BB21344FB81CE
:10A000000023BB8113E0BA89FB8913447B81FB7970
:10A010000E4A0C3352F823207B899B0013441B68A3
:10A02000002B01D17B890BE0BB890133BB81FB791C
:10A03000064AD35C9BB2BA899A42E4D34FF6FF73C7
:10A0400018461437BD4680BC704700BFB0090021D8
:10A0500090B585B000AF03460A46FB8013467B717E
:10A060000023FB60FB8818461FF0F7FC0346002B1B
:10A0700004D140F289111720FFF7ECF97B791D4AD2
:10A080000C3352F82320FB889B0013441B68002BE1
:10A0900004D04FF4C5711720FFF7DCF97B79154A1E
:10A0A00002339B0013445B68002B01D100231DE0A9
:10A0B0007B79104A02339B0013445C687B79184615
:10A0C000FFF768FE0346194620461FF04BFCF86078
:10A0D000FB68002B09D07B79064A0C3352F8232009
:10A0E000FB889B001344FA681A60FB681846143713
:10A0F000BD4690BDB009002180B582B000AF0346D7
:10A100000A46FB8013467B71FB8818461FF0A5FCAE
:10A110000346002B09D07B79064A0C3352F82320E2
:10A12000FB889B0013441B6800E000231846083797
:10A13000BD4680BDB009002180B584B000AF786015
:10A1400039603B689B781A463B685B781344FF2B69
:10A1500004D940F2AD111720FFF77CF93B681A785B
:10A160003B685B789A4204D940F2B1111720FFF79F
:10A1700071F90023FB737B68BB607B68002B0CBF0D
:10A1800001230023BB733B685A78FB7B1344FB73AA
:10A190003B689A78FB7B1344FB73FB7B7B733B68C8
:10A1A0001A7A7B7B13447B733B685A7A7B7B13441C
:10A1B0007B733B685B797A7B934238BF13467B7332
:10A1C0003B68DB787A7B934238BF13467B737B68AE
:10A1D00003F00303002B04D04FF4E5711720FFF7C1
:10A1E00039F93B685A781B4B1A703B689A78194BBF
:10A1F0005A703B68DA78174B9A703B681A79154B9E
:10A20000DA703B685A79134B1A713B689A79114B93
:10A210005A713B68DA790F4B9A713B681A7A0D4B89
:10A22000DA713B685A7A0B4B1A72BA7B07F1080352
:10A2300011461846FFF744FEBA7B797B07F1080305
:10A240001846FFF77BFEBA687B68D31A18461037AA
:10A25000BD4680BDB009002180B582B000AF034685
:10A26000FB71FB79082B04D940F203211720FFF77B
:10A27000F1F8FB79024AD35C18460837BD4680BD29
:10A28000B009002190B585B000AF03460A46FB80B7
:10A2900013467B71FB884FF6FF72934202D143F263
:10A2A000020334E07B79082B01D907232FE07A7968
:10A2B000FB8811461846FFF71FFFF860FB68002B6C
:10A2C00023D07B79144A52F82330FA88F968104673
:10A2D00098477B79114A0C3352F82320FB889B0066
:10A2E000134400221A607B790C4A02339B0013440A
:10A2F0005C687B791846FFF74DFD03461A46F968FE
:10A3000020461FF091FB002301E043F202031846B0
:10A310001437BD4690BD00BFD0500301B0090021E5
:10A3200080B584B000AF78607B689B79BB73FFF722
:10A3300047FD03467B737B68DB79FB7323E0BB7BC4
:10A34000174A0C3352F82320FB7B9B0013441B68F5
:10A35000002B15D0FB7B0133DAB27B68DA71FB7B13
:10A360009AB27B689A80BB7B0D4A0C3352F823204B
:10A37000FB7B9B0013441A687B681A6000230AE089
:10A38000FB7B0133FB73FA7B7B7B9A42D7D37B68E1
:10A39000FA7BDA71052318461037BD4680BD00BF31
:10A3A000B009002180B582B000AF03460A46FB80A9
:10A3B00013467B717B79084AD35C9BB2FA889A4238
:10A3C00004D340F2B2211720FFF744F8FB88DBB238
:10A3D00018460837BD4680BDB009002180B483B05F
:10A3E00000AF0023FB710023FB710DE00C4B1B68D9
:10A3F0005A68FB799B0013441B68002B01D0002393
:10A4000009E0FB790133FB71054B1B681B7AFA7974
:10A410009A42EBD3012318460C37BD4680BC7047E7
:10A42000040A002180B586B000AFF8600B467A6060
:10A43000FB7200237B61FB68002B0CBF0123002310
:10A44000FB74FB6803F00303002B03D08621182064
:10A45000FFF700F8FB7A002B36D0796800201FF058
:10A460002CFA78617B690C337B61FB7A9B007A69FB
:10A4700013447B61FB7C83F00103DBB2002B23D010
:10A48000144AFB681360134B1B68FA7A1A72114B5B
:10A490001B68FA680C325A600E4B1B685968FB7ACD
:10A4A0009A000C4B1B680A441A600A4B1B685868D8
:10A4B000FB7A9B001A4600211CF0B0FA054B1B6882
:10A4C000796818461FF0F9F97B6918461837BD46B8
:10A4D00080BD00BF040A002190B589B002AF0446D8
:10A4E000084611461A462346FB800346BB800B46AE
:10A4F0007B8013463B80344B1B68002B03D1A52186
:10A500001820FEF7A7FF304B1B681B7A9BB2FA8816
:10A510009A4208D22C4B1B685A68FB889B00134454
:10A520001B68002B02D043F2020348E03A88BB8844
:10A53000114618461FF0C8FC0346FB823A8D7B8803
:10A54000114618461FF0D8FC0346BB82FB8ABA8A24
:10A55000114618461FF0E8FC03467B821A4B1B6825
:10A560001B687A8A114618461FF0FCF9F860FB68F0
:10A57000002B01D1042322E0BA8A7B8A1946F868AD
:10A580001FF076FCF8681FF086FC7A88B98A3B8D4C
:10A59000009309231FF086FBF8681FF087FCBA8838
:10A5A000F98A3B8800930A231FF006FC064B1B68C0
:10A5B0005A68FB889B001344FA681A600023184607
:10A5C0001C37BD4690BD00BF040A002180B584B091
:10A5D00000AF0346FB80224B1B68002B03D1C62132
:10A5E0001820FEF737FF1E4B1B681B7A9BB2FA88B8
:10A5F0009A4208D21A4B1B685A68FB889B00134486
:10A600001B68002B02D143F2020324E0144B1B68A9
:10A610005A68FB889B0013441B68FB60104B1B6847
:10A620005A68FB889B00134400221A600C4B1B687D
:10A630001868FB685B881A46F9681FF0F5F9FFF7A0
:10A64000CDFE0346002B05D0054B1B681B68184642
:10A650001FF068F9002318461037BD4680BD00BFC3
:10A66000040A002180B582B000AF0C4B1B68002BA0
:10A6700010D00023FB7107E0FB799BB21846FFF76F
:10A68000A5FFFB790133FB71044B1B681B7AFA7938
:10A690009A42F1D300BF0837BD4680BD040A0021AD
:10A6A00080B584B000AF0346FB800023FB60144BF1
:10A6B0001B68002B03D1EC211820FEF7CBFE104BBA
:10A6C0001B681B7A9BB2FA889A4213D20C4B1B6808
:10A6D0005A68FB889B0013441B68002B0AD0084B68
:10A6E0001B685A68FB889B0013441B6818461FF0C0
:10A6F000D2FBF860FB6818461037BD4680BD00BF2E
:10A70000040A002180B584B000AF0346FB8000231B
:10A71000FB60144B1B68002B03D1FA211820FEF7B5
:10A7200099FE104B1B681B7A9BB2FA889A4213D28F
:10A730000C4B1B685A68FB889B0013441B68002B5A
:10A740000AD0084B1B685A68FB889B0013441B689F
:10A7500018461FF0ABFBF860FB6818461037BD4683
:10A7600080BD00BF040A002180B586B000AF7860CC
:10A77000084611461A460346FB700B46BB7013464B
:10A780003B807B68002B0CBF012300233B7400231C
:10A790007B61FA78BB781344DAB23F4B1A707B685E
:10A7A00003F00303002B03D04E210920FEF752FED5
:10A7B0003B881F2B03D83B889B007B821CE03B8897
:10A7C000FF2B0FD93B8803F1FF023B885B009A42C5
:10A7D00003DA3B88FF339BB202E03B885B009BB20D
:10A7E0007B8209E03B885B007C2B03DD3B885B00C0
:10A7F0009BB200E07C237B827B8A03339BB223F0F5
:10A800000303FB813B7C83F00103DBB2002B05D00B
:10A81000224A7B681360224AFB8913801E4B1B78F7
:10A820001A4613469B001344DB001A467B69134407
:10A830007B6100237B7422E03B7C83F00103DBB26D
:10A84000002B15D0154B19687A7C13469B001344D6
:10A85000DB000B4401221A70104B19687A7C1346F6
:10A860009B001344DB000B4479687A690A445A6000
:10A87000FB897A6913447B617B7C01337B74064BD3
:10A880001B787A7C9A42D7D37B69073323F007037E
:10A8900018461837BD4680BD080A00210C0A002161
:10A8A000100A002180B588B000AF78600B46FB70BD
:10A8B0007B685B687B61FB78002B30D07B68012272
:10A8C0005A70404B1B8818461FF0DAFB0346FB8189
:10A8D0000023FB611FE07B68FA690C32002123F83A
:10A8E00012107B68FA691032F98923F81210FB897B
:10A8F000FA6902FB03F37A691A447968FB699B00E1
:10A900000B445A607A68FB691344143300221A70AE
:10A91000FB690133FB61FB69032BDCD94DE07B68EC
:10A9200000225A700023BB611AE07B68BA690C32BE
:10A93000002123F812107B68BA691032002123F835
:10A9400012107A68BB699B00134400225A607A682F
:10A95000BB691344143300221A70BB690133BB6115
:10A96000BB69032BE1D9174B1B8818461FF095FBD9
:10A9700003467B82134B1B8818461FF0A1FB03463E
:10A980003B827B687A695A607B683A8A1A843B8A80
:10A990007A691A447B689A607B687A8A5A847B68F1
:10A9A0007A69DA607B683A8A9A843B8A7A691A44BF
:10A9B0007B681A617B687A8ADA8400BF2037BD46DB
:10A9C00080BD00BF100A002180B584B000AF002315
:10A9D000FB600023FB7217E01D4B1968FA7A1346DF
:10A9E0009B001344DB000B441B78002B09D0184B51
:10A9F0001968FA7A13469B001344DB000B44FB6092
:10AA000007E0FB7A0133FB72124B1B78FA7A9A4209
:10AA1000E2D3FB68002B03D1A9210920FEF71AFD20
:10AA2000FB68002B0ED0FB6802337B6000BF7B68A5
:10AA300000221A7000BF0121F868FFF733FFFB689E
:10AA400000221A70FB6818461037BD4680BD00BF53
:10AA50000C0A0021080A002180B582B000AF0C4B1F
:10AA60001B8818461FF00CFB0346FB80084B1B8815
:10AA700018461FF025FB0346BB80FA88BB8893422B
:10AA800038BF13469BB218460837BD4680BD00BF8D
:10AA9000100A002180B586B002AF78600B46FB70CB
:10AAA0001346BB702E23FB73BB789BB2FA7892B22D
:10AAB000F97B18461FF058F90346BB817B68002BD1
:10AAC00013D0BB789AB2FB789BB2F87BB98900931C
:10AAD000034678681FF000F9064A7B681360064A4F
:10AAE000FB781370054ABB781370BB891846103782
:10AAF000BD4680BD140A0021180A0021190A002150
:10AB000080B500AF054B1B68054A1178054A1278DD
:10AB10001846FFF7BFFF00BF80BD00BF140A002129
:10AB2000180A0021190A002180B400AF024B1B68EB
:10AB30001846BD4680BC7047140A002180B400AF9F
:10AB4000024B1B781846BD4680BC7047190A00218D
:10AB500080B584B000AF03460A46FB8013467B7184
:10AB60007B79002B0FD1FB8805211846FFF71AFCD3
:10AB70000346BB730D4B1B68BA7B0D49098801FB6B
:10AB800002F213440EE0FB8806211846FFF70AFC88
:10AB90000346FB73074B1B68FA7B0749098801FBD7
:10ABA00002F2134418461037BD4680BD240A002126
:10ABB0002A0A0021300A0021340A002180B586B01B
:10ABC00002AF78600B46FB701346BB70BB789BB23C
:10ABD0001A460321F7201FF037F9034603339BB2CF
:10ABE00023F00303BB817B68002B28D07B6803F034
:10ABF0000303002B03D071211920FEF72BFC144A0C
:10AC00007B681360134ABB8913800023FB8111E02A
:10AC1000FB8901211846FFF79BFFB860BB789BB208
:10AC2000B98900930323F722B8681FF0DFF8FB8986
:10AC30000133FB81FB789BB2FA899A42E8D3FB7817
:10AC4000BA8902FB03F318461037BD4680BD00BF2A
:10AC5000300A0021340A00210122104B4FF0FF304E
:10AC600000215A60C3F8080303F580539A60C3F8C3
:10AC70000012C3F80803C3F80015C3F804259A604E
:10AC8000C3F80803C3F80015C3F8042503F580537F
:10AC900041F6F872C3F80825704700BF00D00041A4
:10ACA0000A4B4FF40052C3F88020BFF34F8FBFF31D
:10ACB0006F8FC3F880214FF48042C3F88020BFF328
:10ACC0004F8FBFF36F8FC3F88021704700E100E022
:10ACD00008B5FFF7C1FFFFF7E3FF00F01BF8054BD6
:10ACE00041F6F872C3F8082500F0AAF8BDE808405C
:10ACF00000F0AEB800F0004108B5FFF7ADFFFFF778
:10AD0000CFFF034B41F6F872C3F8082508BD00BF1A
:10AD100000F0004110B5054C204620F0F5FE18B1BA
:10AD200027211D20FEF796FB607010BD360A00211A
:10AD30002DE9F04707462B4E2B4C2A4820F0E8FE21
:10AD4000054608B1FF2373704FF001080023DFF8B8
:10AD50009C90C4F80480C4F80031C4F80431C4F8ED
:10AD60000475C4F80080D4F8003113B9D4F8043164
:10AD7000E3B1D4F80431002BE8D1A5B996F80180ED
:10AD8000032375704FF400523046C4F80833184B53
:10AD9000C4F80451C4F80051C3F8802120F0C7FE64
:10ADA000B8F1000FC9D10020BDE8F087D9F8103004
:10ADB000DB06D8D50E4B4FF40052C3F88021EFF3D9
:10ADC000108A72B60323C4F80433D4F8003123B9CF
:10ADD000D4F804310BB920F0B5FEBAF1000FC2D19E
:10ADE00062B6C0E7360A002100D0004100ED00E065
:10ADF00000E100E0114B1A6870B5E2B15A680C210D
:10AE0000012501321E680C2A28BF002205FA02F42F
:10AE100026420DD05A60EFF3108172B61A6822EA0A
:10AE200004021A6001B962B65B680360002070BD5D
:10AE30000139E6D15A600520F9E700BF380A002140
:10AE4000024B00221A605A60704700BF380A002186
:10AE5000014B00221A707047400A0021084B10B5C0
:10AE60001C784CB91BF0D0FC064BFF28187005D19C
:10AE700073211F20FEF7EEFA0F2010BD2046FCE7DD
:10AE8000400A00211800002110B5044C2078FF284A
:10AE900003D01BF0D5FCFF23237010BD1800002148
:10AEA000044B4FF6FF7200219A86DA8683F832103F
:10AEB0001A8770478C0A0021044B4FF6FF7200215D
:10AEC0009A86DA8683F832101A8770478C0A002136
:10AED000054B9A8E824205D100214FF6FF7283F80E
:10AEE00032109A86704700BF8C0A0021014BD88629
:10AEF000704700BF8C0A00210A4A4FF6FF710346D3
:10AF0000B2F834C08C4503D0002210461A60704756
:10AF100092F83210012902D001201A6070470020F7
:10AF2000704700BF8C0A0021064B93F83220012A9B
:10AF300006D00122D98E104683F8322099867047B8
:10AF4000002070478C0A0021014B1887704700BF12
:10AF50008C0A0021074B0246B3F834C0198F8C4588
:10AF600001D00020704793F832000028FAD0012069
:10AF7000136070478C0A0021094B998E1A8F9142F9
:10AF800001D0002070474FF6FF7193F83220998668
:10AF9000002AF6D00022012083F83220704700BF3B
:10AFA0008C0A0021064B998E1A8F914201D0012004
:10AFB000704793F83200B0FA80F04009704700BF44
:10AFC0008C0A0021704700BF034648B9094B4FF077
:10AFD000010C08688A88586003F804CB9A8070478F
:10AFE000012800D07047034A086889889372D060AE
:10AFF00011827047C80A002140B90C4A13781BB16E
:10B000005068128908608A8018467047012809D163
:10B01000064A937A002BF7D0D068128A0860184647
:10B020008A80704700231846704700BFC80A002175
:10B0300000B580EA020C1A78087891F805E05040D3
:10B040004A78604493F801C082EA0C0291F802C089
:10B05000024498788CEA000CC8789444DA7850401E
:10B060000A7900EB0C0193F804C0587982EA0C03CA
:10B070008EEA00020B44DA420CBF012000205DF88A
:10B0800004FB00BF10B9054B18787047012802D1A6
:10B09000024B987A70470020704700BFC80A002111
:10B0A00030B503468DB0CA780D4600240068596853
:10B0B000EC468DF81F209A68DB6806948DF81C40DA
:10B0C000CDE90444ACE80F002B7968468DF81E30BA
:10B0D0006B798DF81D301FF0D3FA2A789DF82F3048
:10B0E0009A4202D020460DB030BD6A789DF82E30CD
:10B0F0009A42F7D1AC789DF82D00201AB0FA80F072
:10B1000040090DB030BD00BF30B50C4603210546E7
:10B110008DB0601852B3FEF723FC6379EC4603F060
:10B120003F0343F0400363718DF81D30002328680E
:10B1300006938DF81C306968AA68CDE90433E3787A
:10B140008DF81F3023798DF81E30EB68ACE80F00C6
:10B1500068461FF095FA9DF82F109DF82E209DF857
:10B160002D3021706270A3700DB030BDFEF706FC6B
:10B17000D3E700BF10B5044639B10621FEF7F0FB56
:10B18000637903F03F03637110BD0621FEF7F6FB00
:10B19000637903F03F03637110BD00BFF0B52E2348
:10B1A0000E460A4C8446002726F8043B8CF80870AB
:10B1B000334620686168A268B4F80CE09CF8085037
:10B1C00007C3A3F800E0002DF0D1F0BDEE0A002186
:10B1D00070B5224D296BEC6A0B78A83403F0030399
:10B1E000032B1AD1EB8E0120AA8E0343207442F464
:10B1F0000062EB86AB6BAA869847296B237E013BE6
:10B2000018BF012323764B7833B1D4E920320133C0
:10B2100042F10002C4E9203270BD002BEED04B7821
:10B22000002BEBD0AA8E42F40062AA86EA6B002AB9
:10B23000F2D0FB2B08D895F8403063B1AB6B0021FE
:10B240002020BDE87040184795F8413043F01003C6
:10B2500085F8413070BD01230370CFE7E00A00217B
:10B2600070B57E4C002382B0E56A8DF8053095F804
:10B27000CB2005F1A80694F876300AB10433DBB28E
:10B28000FF2B11D180B995F86F3095F86E108B4275
:10B2900002D0FF2016F030F8B37D032B00F2D980E6
:10B2A000DFE803F0051F7F6F95F86E10F1E794F863
:10B2B00077306B48ADF80630A5F85430FFF74AFEFA
:10B2C000002840F09D800DF105020DF10601E06FB0
:10B2D0001DF073FFA06720B196F85D30002B00F0E1
:10B2E000A280604B1846A367F37DDB0003F00802E1
:10B2F000037803F0F3031343327E920002F004025A
:10B30000134303F0EF0203F00303032B027002D197
:10B31000C378022B11D0E06F1EF07AF848B9A06F05
:10B32000027802F00303032B07D0FFF73BFE00284F
:10B3300076D1A06F027842F01002027096F82230A7
:10B3400013B14378002B46D116F062FA15F0F8FDE0
:10B350006A6941F64B539A4236D8012195F86F201D
:10B36000084616F01DFBA26F01233F491088927812
:10B3700084F8B030A4F8B40084F8B7308A7002B012
:10B3800070BD3748FFF7E6FD00285DD0A06FC37899
:10B390001B2BA9D1012105F1100015F0DFFFA06FD3
:10B3A000A2E7B5F854300DF105020DF10601E06F8A
:10B3B000ADF806301DF001FFA067002894D140F2DF
:10B3C000E9212720FEF746F895F86F20012100209B
:10B3D00016F0E6FAC7E7D4F8800016F019FA94F8E8
:10B3E0002810D4F88000D6E91E23B1FA81F6A16FA7
:10B3F0007609C4E9262384F8A06015F047FDA7E785
:10B40000E38E8020A16F43F08003A26BE386904718
:10B410000121A06F7174C3781B2B7FF465AFBAE76D
:10B42000A06F027889E79DF805302BB1BDF80610B2
:10B4300003F008FEA06F57E7038001218370A06F1F
:10B4400003F0C6FBA06FF1E740F2F2212720FEF7E0
:10B4500001F840F2FF212720FDF7FCFFE00A002160
:10B46000580B0021240B0021940B002110B5134C24
:10B4700016F0A4F815F064FD0021A36BA08E984788
:10B48000237F53B9D4F8BC3094F8411094F8B80035
:10B490009847002384F8B73010BD234607CB1B889C
:10B4A000C4F80E0004F11D00C4F81210C4F81620F0
:10B4B00024220349638304F067F9E3E7E00A0021EB
:10B4C0009DB10001034B93F8B73003B97047FFF704
:10B4D000CDBF00BFE00A0021174A92F828307BB1A7
:10B4E00080B992F8B410C9060ED503B30021D38EEB
:10B4F0009B0714D5936FDB78981E18BF0120704707
:10B500000128EED000207047D2F8C010D06B097827
:10B51000C1F30011C1F1010120B1002BE7D131B11C
:10B5200001207047B2F8C4000028F9D1F5E7D08EA9
:10B53000003818BF01207047E00A002108B5094B08
:10B5400093F8B720022A07D11A7B42F001021A733E
:10B55000BDE80840FFF78ABF40F24D212720FDF7E4
:10B5600079FF00BFE00A0021F8B52C4C0646E56AD9
:10B57000D4F8C03095F8CB2005F1A80794F87600F0
:10B5800023630AB1031DD8B2FF2895F86F1004D1C8
:10B590001EB995F86E30994203D015F0ADFE97F8BC
:10B5A00023205AB3D4F8800016F032F994F82830EA
:10B5B000D4F88010003B206B18BF012384F8A03022
:10B5C000D7E92023C4E9262315F060FC3EB995F89D
:10B5D0006F0010F00C0018BF282016F079F96A6986
:10B5E00041F64B539A420FD895F86E200021012066
:10B5F00016F0D6F9022384F8B730F8BD206B16F0A8
:10B6000007F915F09DFCE1E7002195F86E2008464A
:10B6100016F0C6F9022384F8B730F8BDE00A00211D
:10B620002DE9F041444C82B006460F4694F8B7200D
:10B63000E56A012A5FFA82F805F1A80577D12B7C2B
:10B640006BB1E38E0021042043F004032974E386E8
:10B65000A36B984794F828300BB185F81280A16F3E
:10B660000A7802F00302032A44D04B78EBB102239C
:10B67000AB7595F8233023B3E36A93F86F1094F811
:10B6800028300139003B18BF012384F8A030D5E9E8
:10B690002023C4E9262394F87620072942D8DFE83E
:10B6A00001F03E0941074141413B0123AB75E0E711
:10B6B0004FF0030800214346012000911F4915F077
:10B6C00087FB012F11D186B9D4F8C830304698478E
:10B6D00058B194F8413043B93046FFF7FDFE20B928
:10B6E00002B0BDE8F041FFF73FBF02B0BDE8F04156
:10B6F000FFF7BCBEAB7D63B9E38E022043F00203CB
:10B70000E386A36B9847A16F0B7803F00303032B29
:10B71000ABD10323AB75ACE74FF00208CAE74FF09B
:10B720000008C7E740F222410620FDF793FE40F2F1
:10B7300075412720FDF78EFEE00A0021680B0021ED
:10B7400070B50B4C94F8B73073B906460D4603F04C
:10B75000FF02012104F14400227703F039FAC4F812
:10B76000C060C4F8805070BDD0212720FDF772FE64
:10B77000E00A0021044A92F8B73003F0FF000BB949
:10B78000107770470C207047E00A0021024B01221D
:10B7900083F84020704700BFE00A00212DE9F04304
:10B7A00085B0BD4C02AD85E8030094F8B7100C9845
:10B7B000002940F0EC81002B18BF002A00F0E7813F
:10B7C000002800F0E48101F0FF06C4F8C830C4F896
:10B7D000BC0004F12803A26384F8406084F841604F
:10B7E00084F8CC6084F8B86084F8B060E686A686F9
:10B7F00095E8030083E80300E56A15F003FE15F001
:10B800009FFB95F9720005F1A80715F0BBFE286AA9
:10B8100015F0E2FFA86915F0C1FE97F8330015F0A6
:10B82000C7FE94F82830002B00F0AD8004201BF0F8
:10B83000C9F96A6941F64B539A4200F2C18001206E
:10B8400016F0A8F84D2015F011FD95F86F100120A5
:10B8500016F0B4FD002800F0AC80904815F0C2FF4F
:10B860002888FEF74FFFE0672888FEF719FF95F854
:10B870007B30C4F8D0001BB9696F002940F0CF803D
:10B88000D7F89430DFF818C2D7F88800D7F88C10B2
:10B89000D7F89020ACE80F00D7F89830C4F8A13062
:10B8A000D7F89C30CCF80D3094F82830002B40F0BD
:10B8B0008B80E36A93F8C520263A012A40F2D680AD
:10B8C00093F8C620262A00F0D18093F86E10042940
:10B8D00000F0148111F00C0FA88F18BF4FF42960ED
:10B8E00002F004F82B8F95F86F10834297F823909D
:10B8F000B5F8408028BF03460829B5F8420008BFC4
:10B90000042184F8773001F0F1FFB9F1000F01D183
:10B91000043080B2404528BF40465FFA80F884F882
:10B92000D48004F019FA20B1B8F12B0F38BF4FF0D2
:10B930002B0894F8281084F87680002940F0D380F2
:10B9400097F82230002B00F0B580012395F86E6047
:10B9500084F8A030013E6869D7E91E23C4E9262394
:10B9600041F64B53984294BF04200020072E00F26A
:10B97000E580DFE816F09800FA00E3009700E300A6
:10B98000E300E300FC0003201BF01CF96A6941F6A8
:10B990004B539A4210D8012015F0FCFF4D2015F0B2
:10B9A00065FC95F86E10002016F008FD00287FF465
:10B9B00054AF05B0BDE8F083962015F057FCF0E7D2
:10B9C000962015F053FC40E7E26A92F8C530A3F1E7
:10B9D0002601012934D992F8C600262830D0A3F1D7
:10B9E00021011346012900F2C880242840F0AB80D1
:10B9F00092F8671092F866310B4092F86E105A0771
:10BA00007CD413F0010275D19B077FF563AF042945
:10BA100074D0082972D0012918BF022124E0B7F898
:10BA20004A20BB8A93427FF42BAFB5F878201344A9
:10BA30000122A7F84A3095F87A0017F05FFE1FE759
:10BA400092F8D63392F86E10002B3FF443AF0829DA
:10BA500054D0042952D0082B50D0042B4ED00129A9
:10BA600001D0012B15D10121A88F39E793F832239A
:10BA700093F86E10002A3FF42DAF08293ED0042918
:10BA80003CD0082A3AD0042A38D00129EBD0012A28
:10BA9000E9D00221E8E700BFE00A002108510301D4
:10BAA000680B0021032100220B463E490092FB2235
:10BAB00015F08EF90120FFF7D3FB3B4BD3F850353F
:10BAC00023F00803032B67D0002397F83320C4E941
:10BAD0000033A360A3812988BB8A218022716380FF
:10BAE00005B0BDE8F08397F823305BB90120FFF77C
:10BAF0003BFDE2E7042901D0082946D108214FF493
:10BB00002960EDE695F86F300122D7E92001013B6D
:10BB100084F8A020C4E92601072B0FD8DFE803F042
:10BB200005290E040E0E0E2B032600213346424635
:10BB3000012000911B4915F04BF9D7E740F2224153
:10BB40000620FDF787FC92F8663192F86E105A07CE
:10BB5000D4D413F0010214D198077FF5BBAE0829A5
:10BB6000CCD004297FF457AFC8E701219BE702211D
:10BB700099E70126D9E70226D7E724287FF4A5AE66
:10BB800036E70829BAD00429B8D011466CE740F24C
:10BB900045112720FDF75EFC40F202212720FDF72A
:10BBA00059FC00BF680B00210080004110B5174C04
:10BBB00094F8B730DBB194F828307BB194F8B73003
:10BBC000022B1ED1E36AD3F8100315F057FEE36A87
:10BBD00093F87B200AB9596F61B910BD94F8B7305A
:10BBE000012BF4D040F21A212720FDF733FCFFF798
:10BBF0003DFCECE7114693F87A00BDE8104017F0E1
:10BC00007DBD40F21E212720FDF724FCE00A002123
:10BC1000FFF72CBC014B1877704700BFE00A0021EA
:10BC2000014B93F8B0007047E00A0021024B988E58
:10BC3000C0F38020704700BFE00A0021014B93F859
:10BC4000CC007047E00A00212DE9F0411E4F820729
:10BC500082B00546FC6A0E4604F1A80411D4EB0735
:10BC60000CD5217ED4E92032013342F100020129B2
:10BC7000C4E920320CBF00230123237602B0BDE8C3
:10BC8000F081FB6BDBB1B7F8C4201846396B033287
:10BC900091F801801AF04CFE0DF1020201A93863FF
:10BCA000D7F8D0001DF082FD01981DF043FD012260
:10BCB00030604146D7F8D0001DF06CFCCFE740F271
:10BCC00066412720FDF7C6FBE00A00212DE9F04779
:10BCD000002386B0A54C06468DF80F300F46E56A66
:10BCE000CDE9043394F8B730A835022B5FFA83F816
:10BCF00040F08981A38E13F0400106D1A36B402050
:10BD00009847A38E43F04003A386002E61D095F898
:10BD10002330002B40F00A81236B597889B2A4F8B4
:10BD2000C410002940F016810022E2631A78E87DF1
:10BD3000A38EC2F3800143F480738842A38600F08F
:10BD4000DF80E16A94F8280001F1A80999F816103B
:10BD5000D9B1022900F03E81002189F8161020B1E6
:10BD600099F81230002B40F02B8199F81130002BFC
:10BD700040F0028199F81730012B0CBF00230123FA
:10BD800089F81730236B1A78A38E43F480634FF041
:10BD90000009A386C2F3C0022B7E934228D103F090
:10BDA000DBFF002800F0BD80226B137803F0030353
:10BDB000013B012B00F2B580527894F8D4309A42BE
:10BDC00040F2AF8094F8413043F0100384F84130E2
:10BDD0000EE095F82320002A40F0C38043F400735E
:10BDE0004FF00009A38694F8CC30013384F8CC30AE
:10BDF00095F822303BB394F8283041F64B52B3FA11
:10BE000083F35B0984F8A030E36A586993F86E10F5
:10BE1000904294BF042000200139D5E91E23C4E9D3
:10BE20002623072900F2C480DFE801F07804C275F8
:10BE3000C2C2C2064FF00108002243464C4900929C
:10BE4000FB2214F0C5FF002F45D194F8CC30012B14
:10BE500041D8D4F8C8300120984700283BD094F846
:10BE60004130002B37D10120FFF736FB0746002871
:10BE700031D1FFF7F5F99DF80F30002B32D1B9F130
:10BE8000000F06D094F82830002B3BD16389013392
:10BE9000638166B3E38800223648013384F8CC20FE
:10BEA000E38004F0F9FB049840B11DF043FCE16A23
:10BEB00000230E220130037203F044FC059B33B1D2
:10BEC000E16A00202A221872059803F03BFC97B91A
:10BED00006B0BDE8F08715F0C7FD9DF80F300127CB
:10BEE000002BCCD005A90220FFF7AEFEC7E72389BF
:10BEF00001332381D7E7FFF7B9FA06B0BDE8F08731
:10BF0000B14647E7E3882189AA8A0B4313439BB2D2
:10BF1000002BBED0BAE74FF003088DE74FF00008C2
:10BF20008AE70DF10F00FFF753F961E715F04CF8C0
:10BF300015F02EF8236B597800287FF4EFAE002916
:10BF40003BD01B782A7EC3F3C0039A4255D089B2F6
:10BF5000A4F8C410D4F8D0001DF0A7FA236BE06356
:10BF6000E4E615F06BF8A38E38E700BFE00A002185
:10BF7000680B0021080B00214FF0000A89F811A07E
:10BF8000FEF7FAFF002848D0E38E5146082043F020
:10BF90000803E386A36B9847D9F878300133C9F8D2
:10BFA0007830D9F87C3043F10003C9F87C30E1E601
:10BFB00040F222410620FDF74DFAA4F8C410B3E682
:10BFC000E38E102089F8121043F01003E386A36B70
:10BFD0009847CAE604A9E06F1DF042F9C0B1D9F84C
:10BFE000783094F828000133C9F87830D9F87C30DB
:10BFF00043F10003C9F87C30AEE6012384F8B83081
:10C00000FFF734FA64E740F2EA412720FDF722FA0D
:10C0100040F2E3312720FDF71DFA40F2FA312720E4
:10C02000FDF718FA464B9A786AB393F803118142E8
:10C030002FD0012A27D093F80411814229D0022A57
:10C0400021D093F80511814223D0032A1BD093F805
:10C05000061181421DD0042A15D093F807118142A0
:10C0600017D0052A0FD093F80811814211D0062A63
:10C0700009D093F8091181420BD0072A03D093F815
:10C080000A21824205D01A78013AD2B290421A703F
:10C0900000D17047D200C10002F2531201F25311D5
:10C0A00010B59C581A4403EB010CD2F804E05C5024
:10C0B0009A781978CCF804E06AB393F803418C427B
:10C0C0002FD0012A27D093F804418C422BD0022A8A
:10C0D00021D093F805418C4229D0032A1BD093F834
:10C0E00006418C4221D0042A15D093F807418C4296
:10C0F0001FD0052A0FD093F808418C421DD0062A84
:10C1000009D093F809418C4215D0072A03D093F83F
:10C110000A218A4200D010BD0722134483F803018C
:10C1200010BD0022F9E70122F7E70322F5E702221A
:10C13000F3E70422F1E70622EFE70522EDE700BF6F
:10C14000B80B0021044B9A78824203D9184490F826
:10C150004301704700207047B80B002108B50B4B16
:10C1600040F2D312002118461AF058FC0022034670
:10C170004FF0FF314FF4617083F8DC2183F8DD214B
:10C18000A3F8DE01C3E9751108BD00BFB80B00219B
:10C190002DE9F84FDFF804A105469AF80040002C7D
:10C1A0006BD091F800B0534691F801904FF0000E1B
:10C1B00091F80280CF780E79487906E00EF1010EF1
:10C1C00008335FFA8EF2944237D993F8532193F8EB
:10C1D00054C16A408BEA0C0C624493F855C189EA59
:10C1E0000C0C624493F856C188EA0C0C944493F802
:10C1F00057217A40944493F858217240624493F84E
:10C2000059C180EA0C0C1CEB020FD7D10EF12A0E9B
:10C210000AEBCE0E9EF80A3013F001000BD19AF80B
:10C220000120072A07D843F001038EF80A300132B3
:10C2300001208AF80120BDE8F88F9AF80130072B19
:10C2400002D90020BDE8F88F631C0F2C8AF800305B
:10C2500020D82A34E3B2DB00043308680AEBC404B4
:10C260004AF8030053448A889A80A37A9AF80120F6
:10C2700043F00103E570A372D9E79AF80130072B68
:10C2800001D92046D7E701224FF4AA732A248AF85D
:10C290000020E2E746212820FDF7DCF8B80B00215A
:10C2A0002B4B2DE9F04F1E7885B0002E4ED00B7928
:10C2B0000025074691F800B0019328464B7991F884
:10C2C00001A0029391F8029091F80380204B03960D
:10C2D00004E00135039AE8B2824233D993F853114E
:10C2E000083393F84C4193F84D2179408BEA0404CC
:10C2F00093F84EE18AEA0202019E214489EA0E0E79
:10C3000093F84FC10A4493F8501188EA0C0C93F843
:10C31000514172447140029E62447440114461185C
:10C32000D7D10B4A2A35537802EBC505013B537030
:10C33000AB7A61F30003AB72FFF774FE012005B026
:10C34000BDE8F08F002005B0BDE8F08F3046F6E77D
:10C35000B80B0021014B83F8DD017047B80B0021B9
:10C36000014B93F8DD017047B80B00215E4A13784A
:10C37000013B5BB2002BC0F2A48010B505E0DBB23C
:10C38000013B5BB2591C00F0988003F12A0002EBDC
:10C39000C0018C7AE407F2D592F801C0DBB291F8C3
:10C3A0000AE00CF1FF3C94786FF3000E82F801C0B4
:10C3B00081F80AE06CB392F803119942E0D0012CA5
:10C3C00027D092F804119942DAD0022C21D092F8A9
:10C3D00005119942D4D0032C1BD092F80611994232
:10C3E000CED0042C15D092F807119942C8D0052C54
:10C3F0000FD092F808119942C2D0062C09D092F8B9
:10C4000009119942BCD0072C03D092F80A11994225
:10C41000B6D011780139C9B28B421170B0D0C900C1
:10C42000C00001F25311033052F801E01144141816
:10C43000D1F804C042F800E091781078C4F804C044
:10C4400000299DD092F8034184423ED0012997D023
:10C4500092F8044184423AD0022991D092F80541E1
:10C46000844238D003298BD092F80641844230D0E0
:10C47000042985D092F8074184422ED005293FF443
:10C480007FAF92F80841844229D006293FF478AF63
:10C4900092F80941844224D007293FF471AF92F801
:10C4A0000A1181427FF46CAF0721114481F80331F6
:10C4B000013B5BB2591C7FF468AF002382F8DD3189
:10C4C00010BD002382F8DD3170470021EDE7012126
:10C4D000EBE70321E9E70221E7E70421E5E705218E
:10C4E000E3E70621E1E700BFB80B00212DE9F04F9B
:10C4F00085B000250393514B15701F780292002FD1
:10C5000070D00B792E4691F800B000934B7991F8DA
:10C5100001A0019391F8029091F80380474B03E04A
:10C520000135EEB2BE425DD293F85311083393F851
:10C530004C4193F84D2141408BEA040493F84EE1BD
:10C540008AEA0202214489EA0E0E93F84FC10A4496
:10C5500093F8501188EA0C0C93F851419644009AD4
:10C56000E6445140019A714454406118D8D10A46BA
:10C570003249029801EBC50595F85A31C3F300031F
:10C5800003708B7873B32D4890F80311B1422ED00D
:10C59000012B27D090F80421B2423DD0022B21D0AC
:10C5A00090F80521B2423AD0032B1BD090F8062117
:10C5B000B24237D0042B15D090F80721B24234D0C4
:10C5C000052B0FD090F80821B24231D0062B09D0AC
:10C5D00090F80921B2422ED0072B03D090F80A31EF
:10C5E000B34203D0012005B0BDE8F08F0722134607
:10C5F000039921B10A70114989789142F2D90F4A01
:10C60000134493F83B2193F84B01012A08BF40F0F3
:10C61000010005B0BDE8F08F01221346E8E70222D1
:10C620001346E5E703221346E2E704221346DFE759
:10C6300005221346DCE706221346D9E7B80B002192
:10C640002DE9F04F6A4D85B0044628780391CDE975
:10C650000123002800F0BE804B794FF0000E91F8C6
:10C6600000B00093F44691F801A02B4691F8029097
:10C6700091F803800F7907E00EF1010E08335FFA9D
:10C680008EFC604540F29B8093F8541193F853213F
:10C690008BEA01066240911993F855618AEA060611
:10C6A000721893F8561189EA01018E1893F85721F0
:10C6B00088EA0202911993F85821009E7A400A44B0
:10C6C00093F8591171406646D142D5D1AC78002C0F
:10C6D0004AD095F80321624578D0012C44D095F8D2
:10C6E0000421624572D0022C3ED095F805216245A6
:10C6F0006CD0032C38D095F80621624566D0042C06
:10C7000032D095F80721624560D0052C2CD095F8E1
:10C71000082162455AD0062C26D095F80921624599
:10C7200054D0072C20D095F80A0160450CBF122088
:10C73000072005B0BDE8F08F431C0F282B7052D89E
:10C7400000F12A02D3B2DB0004330399064605EB5D
:10C75000C2020868E8502B4489889980937AD47083
:10C760006FF30003AC7893722701DDF80480621C3C
:10C770002C44F81C4146AA701022284400F022FFE5
:10C7800007F1830010222844029D294600F01AFF79
:10C790001021284600F0AAFE03461021404684F8E6
:10C7A000433100F0A3FE0023024684F803611846DB
:10C7B00084F83B3184F84B2105B0BDE8F08FAB78AD
:10C7C000072BB9D9072005B0BDE8F08F122005B0BE
:10C7D000BDE8F08FAB78072BF4D801232A222B7009
:10C7E0004FF4AA73B1E746212820FCF733FE00BFBF
:10C7F000B80B0021774B1A78002A75D02DE9F04F3D
:10C8000085B00B79002691F800B001934B7937463B
:10C8100091F801A091F8029091F8038002936D497C
:10C82000039204E00136039BF7B2BB4258D991F85A
:10C830005341083191F84C5191F84D3144408BEA05
:10C84000050591F84EE18AEA0303019A2C4489EA2E
:10C850000E0E91F84FC1234491F8504188EA0C0C18
:10C8600091F8515173445440029A634455401C441A
:10C870002D19D7D1574A907898B392F80331BB421B
:10C8800035D001282CD092F80431BB4200F09280C0
:10C89000022825D092F80531BB4200F08E80032893
:10C8A0001ED092F80631BB4200F08A80042817D0CF
:10C8B00092F80731BB4200F08680052810D092F82C
:10C8C0000831BB4200F08280062809D092F8093175
:10C8D000BB420BD0072803D092F80A31BB4266D086
:10C8E000002005B0BDE8F08F1046704706252B46A6
:10C8F000421EDFF8E0C0D2B29A428CF8022049D042
:10C900001001E3462B01C41C02EB420103F1030EAC
:10C910006244A4445BF804A00BEB0E048330DCF803
:10C9200008808333DCF804904900DCF80CC04BF835
:10C930000EA001F20B11C4F80CC0C4F80490C4F8A6
:10C9400008805C465BF8008004445846D4F804E054
:10C950001844D4F808C0E4684BF8038005EB45039D
:10C96000C0F804E05D44C4605B00C0F808C05C46E9
:10C9700092F8030103F20B1385F8030160185BF8CA
:10C9800001104BF803105B448188998092F83B3189
:10C9900085F83B310F4B03EBC60696F85A5115F05C
:10C9A00001009ED13846FFF73DFB012099E707259E
:10C9B0002B469DE701252B469AE702252B4697E754
:10C9C00003252B4694E704252B4691E705252B46A6
:10C9D0008EE700BFB80B00217D4A9378013B59B226
:10C9E0000029C0F2E58002EB01102DE9F04F01EBC8
:10C9F000410E01F58275033002EB4E0E15440EF226
:10CA00000B1E09E001391038AEF1060E49B24B1C7D
:10CA100000F0CC809378013BDBB2C9B293708B42BB
:10CA200015F801CD38D01E01F41C833602EB040842
:10CA300052F80490971903EB4304D8F808A0134464
:10CA4000D8F804B06400D8F80C80C0F8009004F264
:10CA50000B14C0F804B0C0F808A0C0F80C8052F85D
:10CA600006A0D7F80490FE68D7F80880C0F88C605C
:10CA70001619C0F880A0C0F88490C0F8888093F898
:10CA800003712F701459CEF80040B488AEF80440FA
:10CA900093F83B3185F838300CF12A0302EBC304DC
:10CAA000A47AE407AED4947874B392F8036166452F
:10CAB000A8D0012C28D092F804616645A2D0022C9F
:10CAC00022D092F8056166459CD0032C1CD092F8C8
:10CAD0000661664596D0042C16D092F8076166452B
:10CAE00090D0052C10D092F8086166458AD0062CAB
:10CAF0000AD092F80961664584D0072C04D092F8D8
:10CB00000A4164453FF47EAF1478013CE4B2A44589
:10CB100014703FF477AFE400DB0004F253140333E6
:10CB2000165914446468D65013445C6093781478A2
:10CB3000002B3FF467AF92F80361A64239D0012B76
:10CB40003FF460AF92F80461A64234D0022B3FF468
:10CB500059AF92F80561A64231D0032B3FF452AF92
:10CB600092F80661A64228D0042B3FF44BAF92F80E
:10CB70000761A64225D0052B3FF444AF92F8086127
:10CB8000A64220D0062B3FF43DAF92F80961A642A1
:10CB90001BD0072B3FF436AF92F80A31A3427FF443
:10CBA00031AF0723134483F803C12BE7BDE8F08FAF
:10CBB00070470023F6E70123F4E70323F2E702239B
:10CBC000F0E70423EEE70523ECE70623EAE700BFDE
:10CBD000B80B0021014B83F8DC017047B80B002132
:10CBE000014B93F8DC017047B80B0021421E4AF25A
:10CBF000B711034692B28A4204D8034A0120A2F830
:10CC0000DE31704700207047B80B0021014BB3F8AC
:10CC1000DE017047B80B0021444B2DE9F04F1F781F
:10CC200085B0002F6FD00B79002591F800B00193EB
:10CC30002E464B7991F801A0029391F8029091F859
:10CC400003803A4B039703E0EEB2039AB2425AD9FB
:10CC500093F85311083393F84C41013593F84D2163
:10CC600041408BEA040493F84EE18AEA0202019FF4
:10CC7000214489EA0E0E93F84FC10A4493F85011EB
:10CC800088EA0C0C93F8514172447940029F624447
:10CC90007C4011446118D7D1244B9B789BB3234827
:10CCA00090F80321B24234D0012B2CD090F804210B
:10CCB000B24230D0022B26D090F80521B2422CD0BF
:10CCC000032B20D090F80621B24220D0042B1AD09A
:10CCD00090F80721B24222D0052B14D090F80821F9
:10CCE000B2421ED0062B0ED090F80921B2421AD0C3
:10CCF000072B08D090F80A11B1420CBF072008207A
:10CD000005B0BDE8F08F082005B0BDE8F08F032026
:10CD1000FAE70846F8E70120F6E70220F4E70420E6
:10CD2000F2E70520F0E70620EEE700BFB80B002190
:10CD3000044B9A78824203D903EB0010833070478A
:10CD400000207047B80B0021044B9A78824203D927
:10CD500003EB00100330704700207047B80B002130
:10CD600010B40D4CA378834203D8002310BC18469E
:10CD70007047204490F803312A33D80004EBC303F2
:10CD80000430DB780B7021182058012310BC106090
:10CD90001846898891807047B80B002170B5064607
:10CDA0000D4614F0DDFD13F07FFF0A4B93F8DC41D4
:10CDB00014B1997811B90C46204670BDD81C833344
:10CDC0003246002D08BF184613F03AFF13F092FFC9
:10CDD000204670BDB80B002108B513F0A1FF08B9BB
:10CDE000FF2008BDBDE8084013F0D0BF13F098BF86
:10CDF000074B9A78824209D9184490F8032103EB33
:10CE0000C20393F85A0100F00100704700207047F8
:10CE1000B80B0021F8B5414C2678002E54D00025DF
:10CE200028462B4603E00135EBB2B3424CD203F166
:10CE30002A0104EBC102927AD207F4D5A2787AB320
:10CE400094F803C19C4540D0012A29D094F804C12C
:10CE50009C4547D0022A23D094F805C19C4545D073
:10CE6000032A1DD094F806C19C4543D0042A17D04C
:10CE700094F807719F4241D0052A11D094F80871A7
:10CE80009F423FD0062A0BD094F809719F423DD0B3
:10CE9000072A05D094F80A719F423BD0102AC2D8C5
:10CEA0004FF0100C04EBC10322180135471C194642
:10CEB00082F8D4C1DA78FFB2043114F027FB267867
:10CEC000EBB23846B342B2D3F8BD4FF0000C634624
:10CED000234493F83B21012AE4D093F84B31002BF3
:10CEE000A1D0DFE74FF0010C6346F1E74FF0020CF1
:10CEF0006346EDE74FF0030C6346E9E74FF0040C9F
:10CF00006346E5E74FF0050C6346E1E74FF0060C9A
:10CF10006346DDE74FF0070C6346D9E7B80B002105
:10CF20002DE9F843144DAF781FB300263146334640
:10CF300005EB03094A1C013605EB010899F83BE1B2
:10CF4000D4B20846BEF1010F02D099F84B216AB164
:10CF500099F8031188F8D4312A3105EBC103194639
:10CF6000DA78043114F0D2FAAF782146F3B2BB423A
:10CF7000DED3BDE8F88300BFB80B00218C46024623
:10CF8000012108B5054B03EB0C1303F1830013F0EB
:10CF900057FEBDE8084013F0ADBE00BFB80B00213E
:10CFA000074B10B593F8DC4114B1997811B90C46D0
:10CFB000204610BD0246D81C13F042FE204610BD8C
:10CFC000B80B0021F8B5114DAE7856B100240746D4
:10CFD0002346E91891F8431121B10134E3B2B34279
:10CFE000F7D3F8BD03EB4301013405EB03133A46D5
:10CFF00005EB410103F1830001F20B11FEF784F808
:10D00000AE78E3B2B342E4D3F8BD00BFB80B002161
:10D0100000487047980D0021084B9A7882420AD93F
:10D020001A1892F8432132B900EB400003EB40009C
:10D0300000F20B1070470020704700BFB80B0021B2
:10D0400001EB4101044B0268490001F20B115A50F7
:10D05000194483888B807047B80B0021064B9A785F
:10D06000824206D9184490F83B01B0FA80F040099A
:10D0700070470020704700BFB80B00212DE9F04F2A
:10D080000C4683B0062105462046009200F02EFA99
:10D09000064658B14B48827822B1009900F23B1005
:10D0A00019F0BCFC304603B0BDE8F08F454B187852
:10D0B0000028F7D094F800B0B64694F801A094F890
:10D0C000029094F80380277994F805C034463D4BCC
:10D0D000019603E05FFA8EF4A04262D993F85321DF
:10D0E000083393F84C610EF1010E93F84D116A402C
:10D0F0008BEA06068AEA0101164493F84E21314470
:10D1000089EA020293F84F610A4493F8501188EAC1
:10D1100006067940164493F8512131448CEA020204
:10D120005118D7D127480A46019E8378002BB9D0E1
:10D1300090F80311A1422AD0012BB3D090F804211A
:10D14000A24235D0022BADD090F80521A24231D0B9
:10D15000032BA7D090F80621A2422DD0042BA1D0FA
:10D1600090F80721A24229D0052B9BD090F80821E6
:10D17000A2421BD0062B95D090F80921A2421FD0C5
:10D18000072B8FD090F80A31A3428BD107220D4B89
:10D1900001261A443046009B82F83B3103B0BDE8BB
:10D1A000F08F019E304603B0BDE8F08F0522EEE718
:10D1B0000122ECE70222EAE70322E8E70422E6E79D
:10D1C0000622E4E7B80B0021002342F2107CA0F80D
:10D1D000482003644B1E0CFB0232B2FBF1F14164A8
:10D1E000704700BF70B50D46002106461CF012FDC9
:10D1F000686018B1002318462B7070BD04460121E9
:10D2000030461CF007FD686018B1012320462B70E2
:10D2100070BD022070BD00BF38B504460D4631B167
:10D22000012965D002292CD003295AD038BD4FF4EA
:10D23000816219F0F3FB49230122042184F817319C
:10D24000342384F8CD20072284F81931FE232B20C3
:10D2500084F8181184F81A217F21424A84F84E314B
:10D260004FF6FF7384F81B5184F81C5184F81D514C
:10D2700084F8160184F8C110C4F8B020A4F856311F
:10D2800038BD0023D0F8DC23416942F21075B0F8B4
:10D29000E203A4F8F630B4F8FA3001FB03F3B3FB71
:10D2A000F2F3A4F8FA30531E05FB0030B0FBF2F0A5
:10D2B000A4F8F800D4F8E80000FB01F1B1FBF2F1AA
:10D2C000C4F8E8102849B1FBF2F10131A4F8FE10CE
:10D2D000B4F8F01005FB0133B3FBF2F3C4F8EC3003
:10D2E00038BD00F1CE01CD30BDE8384000F0A2BD20
:10D2F000436900251D49B0F8FA00D4F8E820194424
:10D3000003FB00F003FB02F2A4F8165384F80B535E
:10D31000A4F8F650B1FBF3F1B0FBF3F0B2FBF3F27B
:10D32000C4F8EC1040F6B831A4F8FA00581EC4F85E
:10D33000E820A4F8F01042F21071E28B01FB020029
:10D34000094A04F1CE01B2FBF3F2B0FBF3F3013270
:10D3500004F1CD00A4F8F830A4F8FE20BDE8384070
:10D3600000F068BD00E0FCFF005A62027FC3C90103
:10D3700038B504460D4631B1012964D002292BD0BD
:10D38000032959D038BD4FF45E7219F047FB492389
:10D390000122042184F81731342384F8CD20072298
:10D3A00084F81931FE232B2084F8181184F81A21EF
:10D3B0007F21404A84F84E31202384F81B5184F8A1
:10D3C0001C5184F81D5184F8160184F8C110C4F86A
:10D3D000B02084F8193338BD0023D0F840234169C8
:10D3E00042F21075B0F84603A4F8F630B4F8FA30FB
:10D3F00001FB03F3B3FBF2F3A4F8FA30531E05FB71
:10D400000030B0FBF2F0A4F8F800D4F8E80000FB1C
:10D4100001F1B1FBF2F1C4F8E8102749B1FBF2F1D8
:10D420000131A4F8FE10B4F8F01005FB0133B3FB92
:10D43000F2F3C4F8EC3038BD00F1CE01CD30BDE8D8
:10D44000384000F0F7BC436942F210751B4AB0F84F
:10D45000FA001A44D4F8E81003FB00F003FB01F1D2
:10D46000B2FBF3F2B0FBF3F0C4F8EC2040F6B832B4
:10D47000A4F8FA00581EA4F8F020E28B05FB020085
:10D480000D4AB1FBF3F1B2FBF3F2B0FBF3F301325F
:10D49000A4F8F8300023C4F8E81004F1CD0004F13A
:10D4A000CE01A4F8FE20A4F8F630BDE8384000F024
:10D4B000C1BC00BF00E0FCFF005A62027FC3C9018B
:10D4C00070B5047934F01F040ED1451E061D15F801
:10D4D000010F02F079FD0444B542E4B2F7D1012C0A
:10D4E00094BF0020012070BD002070BD002964D0D1
:10D4F0004B1E062B00B562D98B0800F1040E0246C4
:10D500004FF0000C013BDBB20EEB830E52F8043BF4
:10D51000724543EA0C0CF9D1CCF30723CCF3074254
:10D520004CEA0303134301F0FC0243EA1C6331F0AD
:10D53000FC0CDBB23CD010F802C043EA0C0302F151
:10D54000010C5FFA8CFC614532D910F80CC043EA3B
:10D550000C0302F1020C5FFA8CFCDBB2614527D9A7
:10D5600010F80CC043EA0C0302F1030C5FFA8CFCC8
:10D5700061451DD910F80CC043EA0C0302F1040CFC
:10D580005FFA8CFC614513D910F80CC043EA0C0318
:10D5900002F1050C5FFA8CFC614509D9063210F8DE
:10D5A0000CC0D2B243EA0C03914201D9825C13430E
:10D5B000B3FA83F040095DF804FB012070470022B4
:10D5C0001346B8E762B102F1FF3C0A44431E5FFA1A
:10D5D0008CF1084412F8011D03F8011F9842F9D19B
:10D5E000704700BF30B51C468DB0C37B15464278EE
:10D5F0008DF80030837B8DF80E208DF80130437B51
:10D600008DF80230037B8DF80330C37A8DF8043037
:10D61000837A8DF80530437A8DF80630037A8DF8D9
:10D620000730C3798DF8083083798DF80930437954
:10D630008DF80A3003798DF80B30C3788DF80C30F3
:10D6400083788DF80D30037868468DF80F30CB7BEA
:10D650004A788DF810308B7B8DF81E208DF81130B4
:10D660004B7B8DF812300B7B8DF81330CB7A8DF815
:10D6700014308B7A8DF815304B7A8DF816300B7A82
:10D680008DF81730CB798DF818308B798DF81930EB
:10D690004B798DF81A300B798DF81B30CB788DF8DB
:10D6A0001C308B788DF81D300B788DF81F301CF0F6
:10D6B000E7FF8DB39DF82F009DF82E109DF82D20CB
:10D6C0009DF82C30207061709DF82B009DF82A1079
:10D6D000A270E3709DF829209DF8283020716171B7
:10D6E0009DF827009DF82610A271E3719DF8252072
:10D6F0009DF82430207261729DF823009DF822105D
:10D70000A272E3729DF821209DF82030207361738E
:10D71000A273E3730DB030BD08AD0FCD2060616022
:10D72000A260E3600DB030BDA0F10B03042B08D95B
:10D73000A0F121032F2818BF062B94BF0120002041
:10D7400070470120704700BF0D2900F28380DFE899
:10D7500001F00D11171D232939454B51585E6707FC
:10D760002A3A042A8CBF002001207047B2FA82F0C6
:10D7700040097047073A012A8CBF002001207047FA
:10D780000B3A022A8CBF0020012070470E3A012A72
:10D790008CBF002001207047113A0C2A8CBF00205A
:10D7A00001207047002B41D1A2F11303012B49D96D
:10D7B00090F85E30002B47D0143A082A8CBF002026
:10D7C00001207047A2F11103032B3BD990F85E00B2
:10D7D0001D2A8CBF002000F001007047A2F1040058
:10D7E000B0FA80F040097047A2F10100B0FA80F071
:10D7F0004009704703BBA2F10500B0FA80F0400970
:10D8000070471E3A022A8CBF002001207047A2F107
:10D8100021002F2A18BF062894BF0120002070473E
:10D82000A2F12900B0FA80F040097047123A0B2AA1
:10D830008CBF002001207047A2F11000B0FA80F0E8
:10D840004009704701207047183A042A8CBF002015
:10D850000120704700207047F8B504460D46D0E916
:10D86000046716F0CDF908B3DDB1236962699B1B2B
:10D8700062EB0702012B72F1000114DB6FF0010073
:10D880000021984271EB020215DB6A1E1344B3FBC0
:10D89000F5F303FB05F5AE191D4647F10007C4E992
:10D8A00004672846F8BD00252846F8BD40F211213E
:10D8B0002920FBF7CFFD40F21B212920FBF7CAFDF1
:10D8C000904238B5044606D2121A742A38BF742220
:10D8D00015188D4202D92546284638BD0321104629
:10D8E00017F002FA0028F6D1F6E700BF11F00C039A
:10D8F0000CD04B0712D44FF474734022984219464F
:10D9000012D9401A90FBF2F080B2704702290DD074
:10D91000702809D97038C0F3CF00704740F20E2349
:10D92000102298421946ECD8002070473C28FBD9B9
:10D930003C38C0F38F0070470B68C0F86A307047FE
:10D94000034610F0010007D19A0704D413F0040035
:10D9500018BF082070470220704700BF2DE9F84F1C
:10D96000894607460846924601F09CFA0546484615
:10D9700001F09CFA10F00104064659D1820700F12B
:10D98000928010F0040474D1A34615F001084CD124
:10D99000AB0700F1838015F0040803D04FF0010BB2
:10D9A0004FF0080813F0FAF80640F6B2002E08BF50
:10D9B000002413F0F3F8054097F86E30EDB2002D17
:10D9C00008BF4FF00008A34226D08AF8004097F81D
:10D9D0006F3043452FD044EA0803DBB28AF8018058
:10D9E000002B4CD0D4B3082C06D05846BDE8F88F95
:10D9F000042B01D0082B37D197F86431012BF4D1D7
:10DA0000B7F86831012B97F86E3050D0082BECD066
:10DA100008238AF80030E8E700238AF8003097F8F6
:10DA20006F20424529D04346D8E74FF0010BB9E7B4
:10DA30004FF0010BA9E700238AF80130002CD2D166
:10DA4000484601F039FAB7F8BC3047F6FD72DB43BF
:10DA500003449BB2934288BF4FF0000B97F86E309F
:10DA6000022BC5D8002BC0D14FF436710620FBF72E
:10DA7000F1FC4FF0010B082487E78AF80130484693
:10DA800001F01AFAB7F8BC30DB43184447F6FD73CF
:10DA900080B2984288BF4FF0000BA3E74FF0010B14
:10DAA0004FF002087EE74FF0010B02246DE7042BD4
:10DAB000AED004238AF8003097E700BF012805D0D4
:10DAC000022803D010F00C0018BF0420704700BFDC
:10DAD000C1F3072384B05FFA80FC012B0190C9B227
:10DAE000C0F307201ED101291CD10CEA000001401F
:10DAF0000B401A46990731D413F0010102D113F0FB
:10DB0000040131D190072DD412F0010303D112F09A
:10DB1000040318BF0823002061F3070063F30F20FC
:10DB200004B07047022901D1022BDED0042901D1B3
:10DB3000042BDAD0BCF1010F01D10128D5D0BCF102
:10DB4000020F01D10228D0D0BCF1040F01D104286A
:10DB5000CBD00CEA030300EA0102CBE790074FF0B9
:10DB60000201D1D50223D6E793070DD412F00103A9
:10DB700003D112F0040318BF0823BDF80620012AC0
:10DB800014BF08210421C6E70223F6E7082908BFCD
:10DB9000012884460CBF012000200FD0A1F1040011
:10DBA000BCF1010FB0FA80F04FEA501008BF00201E
:10DBB00000B97047082113805180704704211380F9
:10DBC00051807047162A01D000207047A0F10C0246
:10DBD000032A0CD9212806D00029F5D00A78012A79
:10DBE00005D9162AF0D1232201201A7070472A2263
:10DBF00001201A70704700BF013908B5072914D8F1
:10DC0000DFE801F0071013041313130440F6A660B5
:10DC100008BD034640F2E24240F6C410002B08BFA4
:10DC2000104608BD40F6C41008BD40F2A1312920BD
:10DC3000FBF710FC41F27073A0F57A729A4205D995
:10DC4000064BA3FB0030C0F38F207047044BA3FBAF
:10DC50000030800900F5506080B270475917B7D185
:10DC6000D34D62106FF45063C318062B04D940F2F1
:10DC7000E24303FB00F070474FF47A73A0F5506065
:10DC800003FB00F0704700BF41F64B53994208D99F
:10DC9000C0EB401300EB830000EB8000400080B23B
:10DCA000704700EB800000EB80008000704700BFF1
:10DCB00041F64B53994205D9054BA3FB0030C0F305
:10DCC00087207047034BA3FB0030C0F34710704719
:10DCD0005917B7D11F85EB5141F64B53994294BF69
:10DCE000642340F2E24303FB00F0704741F64B53DC
:10DCF000994205D9054BA3FB0030C0F38F20704734
:10DD0000034BA3FB0030C0F34F1070475917B7D136
:10DD10001F85EB5141F64B53994209D9094B40F20B
:10DD2000E242A3FB00139B0A02FB1303C01A7047D5
:10DD3000054B6422A3FB00135B0902FB1303C01A0B
:10DD4000704700BF5917B7D11F85EB51A0F5E3709D
:10DD5000884294BF091A491A1868012910B400EBC7
:10DD6000510494BF002001201C60136810BCA3EB79
:10DD700051011160704700BF074B93F90030184400
:10DD8000142804DC10F17F0F03DB40B2704714202D
:10DD900070476FF07E007047A80D002100B583B07A
:10DDA0007F230DF107008DF8073013F0E7FD20B950
:10DDB0009DF9070003B05DF804FB0A4A9DF907309E
:10DDC0005078404240B21844142806DC10F17F0F0E
:10DDD00005DB40B203B05DF804FB1420EAE76FF006
:10DDE0007E00E7E7A80D0021074B1A7803463AB9F1
:10DDF00006490122086809791860104619717047B0
:10DE000000221046704700BFAC0D00211C0000210D
:10DE1000034606494FF0FF0C054A00681B7982F85B
:10DE200000C008600B710023137070471C000021B4
:10DE3000AC0D002170B5441C05468C4204D00B6823
:10DE4000C0F801300B7923716B790022AE1D03F00D
:10DE50001F03EA726B7114F8010B02F0B5F8207120
:10DE6000B442EB7A1844E872F5D170BD81EA1141F1
:10DE7000844689B24A4008B5D3B293FAA3F3120A92
:10DE800092FAA2F2120E1B0E43EA022303EB0313D3
:10DE90000B449AB2DBB293FAA3F3120A92FAA2F2FB
:10DEA000120E1B0E43EA022303EB03130B449AB238
:10DEB000DBB293FAA3F3120A92FAA2F2120EA0486E
:10DEC0001B0E43EA022303EB03130B444B409BB2AC
:10DED000A0FB03201A1A00EB5200400900EBC0021D
:10DEE00000EB82000122181AC0F3C40100F0070EF3
:10DEF000614402FA0EF24978114201D0C0B208BD65
:10DF00009CF80B1001FB03F39CF806104FEA134E2C
:10DF10001B140EF10100C2B28A425BD9501AC2B280
:10DF20009CF80730934280F09A80D01AC2B29CF8D5
:10DF300008309A4240F2D980D01AC2B29CF8093017
:10DF40009A420AD9D01AC2B29CF80A30934280F0A1
:10DF500013819D214620FBF77DFA9CF80430D907F8
:10DF600005D5501E10F0FF0201D1032281E0980771
:10DF700005D5501E10F0FF0201D1032238E05907E9
:10DF800005D5501E10F0FF0201D103223BE0180717
:10DF900005D5501E10F0FF0201D103223BE0D90647
:10DFA00005D5501E10F0FF0201D103223BE0980678
:10DFB00005D5501E10F0FF0201D103223BE05906A7
:10DFC00000F118811806BFD5501E10F0FF02BBD11A
:10DFD000032242E09CF80110C80703D5002B00F093
:10DFE000108172468B0708D5501E10F0FF0204D135
:10DFF000012000EBC200C0B208BD480705D5501E85
:10E0000010F0FF0201D10220F3E70B0705D5501EE7
:10E0100010F0FF0201D10320EBE7C80605D5501E22
:10E0200010F0FF0201D10420E3E78B0605D5501E56
:10E0300010F0FF0201D10520DBE7480605D5501E90
:10E0400010F0FF0201D10620D3E70B067FF568AF81
:10E05000501E10F0FF027FF463AF0720C9E79CF861
:10E06000023013F0010106D0501E10F0FF0202D161
:10E070000A460020BDE7980705D5501E10F0FF02A4
:10E0800001D10122B4E7590705D5501E10F0FF0257
:10E0900001D10122B7E7180705D5501E10F0FF0285
:10E0A00001D10122B7E7D90605D5501E10F0FF02B5
:10E0B00001D10122B7E7980605D5501E10F0FF02E6
:10E0C00001D10122B7E7590605D5501E10F0FF0215
:10E0D00001D10122B7E718067FF529AF501E10F0D5
:10E0E000FF027FF424AF0122B7E79CF80330D90781
:10E0F00005D5501E10F0FF0201D10222B9E79807A2
:10E1000005D5501E10F0FF0201D1022270E7590719
:10E1100005D5501E10F0FF0201D1022273E7180747
:10E1200005D5501E10F0FF0201D1022273E7D90677
:10E1300008D5501E10F0FF0204D1022273E700BF81
:10E140004D91CFBA980605D5501E10F0FF0201D1AF
:10E15000022270E7590605D5501E10F0FF0201D1CA
:10E16000022270E718067FF5E9AE501E10F0FF029C
:10E170007FF4E4AE022270E79CF80530D90705D59C
:10E18000501E10F0FF0201D1042272E7980705D556
:10E19000501E10F0FF0201D1042229E7590705D5CE
:10E1A000501E10F0FF0201D104222CE7180705D5FC
:10E1B000501E10F0FF0201D104222CE7D90613D41F
:10E1C000980603D5501E10F0FF021CD0590603D547
:10E1D000501E10F0FF0218D01B067FF5BAAE012AC0
:10E1E0007FF4B7AE042238E7501E10F0FF02E7D1EB
:10E1F000042218E7501E10F0FF027FF4E3AE032262
:10E2000021E71A4635E7042215E704221BE700BF81
:10E2100090F830C00CF1FF33242B14D88AB110B51C
:10E22000044690F8250080B1012853D1A28A04F158
:10E2300025008969FFF71AFE0346002084F8333071
:10E2400010BD104670471220704794F8311094F8B2
:10E25000323002FB0132994B83FB0213012113443C
:10E260005B1103EBC30E03EB8E03D21AD2B204EBA5
:10E27000D20384F8322093F826E002F0070301FA73
:10E2800003F31EEA030F65D194F82B10B2FBFCF3E5
:10E290000CFB1322D2B2531CDBB28B425DD95B1A4A
:10E2A000DBB294F82C209A4280F093809B1ADBB268
:10E2B00094F82D20934240F2CA809B1ADBB294F866
:10E2C0002E20934240F2FC809B1ADBB294F82F2060
:10E2D0009A4201D21F2010BD94F82A20D10704D5FC
:10E2E000013B13F0FF0300F04C81910704D5013B83
:10E2F00013F0FF0300F04781510704D5013B13F0F1
:10E30000FF0300F04281110704D5013B13F0FF0326
:10E3100000F04581D10604D5013B13F0FF0300F066
:10E320004081910604D5013B13F0FF0300F03B81CF
:10E33000510604D5013B13F0FF0300F036811206AD
:10E34000C8D5012BC6D10423072202EBC30384F8EE
:10E35000333010BD84F8332010BD94F8261011F02E
:10E36000010F03D0002A00F0F38013468A0704D57A
:10E37000013B13F0FF0300F0DA804A0704D5013BAC
:10E3800013F0FF0300F0D6800A0704D5013B13F019
:10E39000FF0300F0D280CA0604D5013B13F0FF034F
:10E3A00000F0CE808A0604D5013B13F0FF0300F095
:10E3B000CA804A0604D5013B13F0FF0300F0C68073
:10E3C0000A067FF56EAF013B13F0FF037FF469AFE0
:10E3D000BAE794F8272012F0010104D0013B13F0B2
:10E3E000FF0300F0B880910704D5013B13F0FF0351
:10E3F00000F09C80510704D5013B13F0FF0300F0AF
:10E400009880110704D5013B13F0FF0300F09480BE
:10E41000D10604D5013B13F0FF0300F09080910674
:10E4200004D5013B13F0FF0300F08C80510604D5A6
:10E43000013B13F0FF0300F0888012067FF538AF30
:10E44000013B13F0FF037FF433AF01237CE794F823
:10E450002820D10703D5013B13F0FF037DD091079E
:10E4600003D5013B13F0FF0379D0510703D5013BDE
:10E4700013F0FF0375D0110703D5013B13F0FF0321
:10E4800071D0D10603D5013B13F0FF0371D0910683
:10E4900003D5013B13F0FF036DD0510603D5013BBB
:10E4A00013F0FF0379D012067FF509AF013B13F09B
:10E4B000FF037FF404AF022346E700BFA7C867DD70
:10E4C00094F82920D10703D5013B13F0FF034CD06A
:10E4D000910703D5013B13F0FF0348D0510703D543
:10E4E000013B13F0FF0348D0110703D5013B13F0A4
:10E4F000FF0344D0D10603D5013B13F0FF0346D000
:10E50000910603D5013B13F0FF0342D0510603D51A
:10E51000013B13F0FF033ED012067FF5D7AE013B5F
:10E5200013F0FF037FF4D2AE03230DE70123012292
:10E530000BE70123022208E70123032205E7012359
:10E54000042202E701230522FFE601230622FCE65E
:10E5500003460022F9E60B46FBE70223F9E7022314
:10E56000E5E70223E6E70223E7E70323F1E70323D6
:10E57000DDE70223E4E70223E5E70323DAE70323E9
:10E58000DBE70423E5E70423D1E70423D2E70323F1
:10E59000D6E70323D7E70323D8E70223D6E70423EC
:10E5A000CBE70423CCE70423CDE70423CEE700BF69
:10E5B00008B5037801F00F0223F00F031343037033
:10E5C000082917D8DFE801F0080508050813080B2B
:10E5D00010000C23437008BD0623437008BD0022C1
:10E5E0000123C270437008BD0E23437008BD22236F
:10E5F000437008BDA8212A20FAF72CFF0B68C0F849
:10E6000003308B88A0F80730704700BFD0F8033084
:10E610000B60B0F807308B80704700BF0B68C0F804
:10E6200009308B88A0F80D30704700BF8B0101784E
:10E6300003F0400321F0400119430170704700BF0F
:10E640000078C0F380107047037803F07F0343EA3B
:10E65000C1130370704700BF0078C009704700BF46
:10E660001F2A38B507D8144605460930063418F075
:10E670005FF96C7038BDEE212A20FAF7EBFE00BF7F
:10E680001F2A38B507D8144605460930063418F055
:10E690004FF96C7038BD4FF488712A20FAF7DAFE12
:10E6A0000278034602F00F02032A18D0052A14D17B
:10E6B00090F820C0C27F90F8210042EA0C0293F843
:10E6C00022C0024393F8230042EA0C0220F01F000C
:10E6D000024302D05A78222A08D00020704740789E
:10E6E000A0F10C00B0FA80F04009704710B56FF44B
:10E6F0005060B3F81920B3F8174002EB000C93F800
:10E7000016E0BCF1060F8CBF002001F0010088B9B3
:10E71000911F40F67A4C89B261450AD80EF1FF315B
:10E72000072906D8944298BF964534BF012000209F
:10E7300000D310BDB3F81B20B2F5FA7F0AD2B3F8AC
:10E740001D0040F676430A3880B298428CBF002004
:10E75000012010BD002010BD10B5002900F08980F7
:10E7600014461A46C37813F03F033CD090F804E0F7
:10E770001EF0010F3CD0002C6BD01EF0020F41D1D7
:10E780004FF00B0C012C2ED01EF0040F41D0022CA8
:10E790004FD00CF1010C1EF0080F5FFA8CFC3DD03D
:10E7A000032C46D00CF1020C1EF0100F5FFA8CFC0B
:10E7B00039D0042C3DD00CF1030C5FFA8CFC1EF018
:10E7C000200F40D0052C34D00CF1120C5FFA8CFCD9
:10E7D0001EF0400F3AD0062C2BD00CF1010C5FFA42
:10E7E0008CFC072C39D040F226312A20FAF732FE71
:10E7F000002CF8D01EF0020F18D0012C36D04FF0AC
:10E800000B0CC1E7012C2DD01EF0040F4FF0110CA2
:10E81000BDD1022CE7D01EF0080FC1D1032CE2D0ED
:10E820001EF0100FC5D1042CC9D1DCE74FF0050C48
:10E83000A8E7ACF1040414443F2C1FDC6044BDE89D
:10E84000104018F075B8052CC2D1CCE7062CC8D101
:10E85000C9E701244FF0050CEDE7ACF10404A34235
:10E86000E9DAC0E707244FF00B0CE4E74FF0050CA2
:10E87000E1E740F225312A20FAF7ECFD40F227319A
:10E880002A20FAF7E7FD00BFC378844613F03F0063
:10E890005CD09CF80430DA072FD5002953D09A07B2
:10E8A00032D40B2201294CD000B513F0040E32D023
:10E8B000022942D0013213F0080ED2B230D003291F
:10E8C0003BD0023213F0100ED2B22ED0042934D035
:10E8D0000332D2B213F0200E39D005292DD01232D6
:10E8E000D2B213F0400335D0062926D00132D2B27D
:10E8F00007291FD000205DF804FB11B39A0717D534
:10E90000012920D00B22CFE7012926D0112200B502
:10E9100013F0040ECCD10229ECD013F0080ECED1A6
:10E920000329E7D013F0100ED0D10429D2D1E1E7AA
:10E930000522B7E7131F9842DCDB0CEB02005DF801
:10E9400004FB0020704705210CEB010070470529EE
:10E95000C7D1CFE70629CBD1CCE70B21F4E700BF25
:10E96000C37803F03F0343EA8113C370704700BFCD
:10E97000C1F3801CC1F380036344C1F3001C0CEBA2
:10E980004C0C6344C1F3401C0CEBCC0C00B503EB06
:10E990004C03C1F3400EC1F3000C1344F444C1F323
:10E9A000C00E0CEB4C0CF44403EB4C0313F0FF03D0
:10E9B00019D003F1010E023301715FFA83FC0EF0EE
:10E9C0003F015FFA8EF380F801C090F803C02CF08D
:10E9D0003F0C41EA0C01C1701AB10433511E9B1A5D
:10E9E000C1545DF804FB19464FF0010CEBE700BF82
:10E9F00003464078DB78013803F03F03C01AC0B209
:10EA0000704700BF10B5864690F803C0D8439EF803
:10EA100001400CF03F0C0444A4EB0C04E4B294421B
:10EA200028BF144641B10CF1040C084622469C4410
:10EA30000EEB0C0117F07CFF204610BD00B5C3782B
:10EA4000017913F03F0318BF012303EA511201EAD1
:10EA5000030E03EA510C03EAD10002EBC202F444B4
:10EA600010440CEB4C0C00EB0C0203EA910003EA9F
:10EA7000911C03EA1113604403EB4303034403EBCB
:10EA8000420010F0FF0001D00130C0B25DF804FB7D
:10EA900038B503780446407803F00F03072B11D8EC
:10EAA000DFE803F0041204101010040A06381F28CF
:10EAB0008CBF0020012038BD0028FCD0E3789A09E3
:10EAC000032A07D1002038BDA0F10C00B0FA80F075
:10EAD000400938BD03F03F05A842F3D92046FFF7AF
:10EAE000ADFF8542EED30DB32379D8061ED503F0D2
:10EAF0000102002A15BF11220B220B21052113F060
:10EB0000020F08BF0A46590748BF01321B0701D54B
:10EB10000232D2B2A35C144403F03F03242BD1D8B9
:10EB2000A0785F288CBF0020012038BD012038BDAF
:10EB300038B50378044603F00F03072B05D0082BE4
:10EB40003BD0042B32D0002038BDC3789A09032A69
:10EB5000F9D003F03F054378AB42F4D9FFF76EFFDD
:10EB60008542F0D3002D2FD02379D8062CD503F081
:10EB70000102002A15BF11220B220B21052113F0DF
:10EB8000020F08BF0A46590748BF01321B0701D5CB
:10EB90000232D2B2A35C144403F03F03242BD2D838
:10EBA000A0785F288CBF0020012038BD407806384F
:10EBB0001F288CBF0020012038BD4078A0F10E0036
:10EBC000B0FA80F0400938BD012038BD4078704768
:10EBD00001F00303017821F003011943017070472C
:10EBE000007800F0030070474B01017803F0200328
:10EBF00021F0200119430170704700BF0B7883702A
:10EC0000704700BF43785BB1C2782A2A06D805490D
:10EC1000885CC01AB0FA80F0400970470120704744
:10EC200018467047185103012A2908B5C17003D846
:10EC3000064B5B5C437008BDFF2902D10123437082
:10EC400008BD40F275412A20FAF704FC185103016F
:10EC50001B2A08B507D8844603308CF80120BDE88C
:10EC6000084017F065BE40F27F412A20FAF7F2FB18
:10EC7000B0F80700704700BFB0F80900704700BF48
:10EC80000B0AC17203737047B0F80B00704700BFE6
:10EC900030B5B0F80730B0F80940B0F8055090F83A
:10ECA00004E0B0F80B206FF4506003EB000CBCF1F3
:10ECB000060F8CBF002001F0010088B9991F40F6B3
:10ECC0007A4C89B261450AD80EF1FF31072906D87E
:10ECD000AB4228BF73458CBF0120002000D830BD57
:10ECE000B4F5FA7F08D20A3A40F6764091B28142F2
:10ECF0008CBF0020012030BD002030BD0B68436078
:10ED00000B790372704700BF43680B60037A0B7185
:10ED1000704700BFB0F80900704700BF0079704726
:10ED20000A684B6842608360704700BF426883682E
:10ED30000A604B60704700BF0B888381704700BF3B
:10ED400083890B80704700BF0A684B68C0F80E20AB
:10ED5000C0F81230704700BFD0F80E20D0F8123043
:10ED60000A604B60704700BF0B68C0F816307047F0
:10ED7000D0F816300B6070470A684B6842608360B9
:10ED8000704700BF426883680A604B60704700BFED
:10ED90000B68C360704700BFC3680B60704700BF5B
:10EDA000007970470B0A0171437170470B0A81713A
:10EDB000C37170470B0A0172437270470B0A81726C
:10EDC000C372704780887047C08870470089704759
:10EDD0004089704703891A2B0DD94389B3F5A47F65
:10EDE00009D383881A2B06D9C088B0F5A47F34BF15
:10EDF0000020012070470020704700BF043001F15F
:10EE0000200310B50C68103151F80CEC103051F89B
:10EE100008CC51F8042C994240F8104C40F80CEC06
:10EE200040F808CC40F8042CECD10B88038010BDCE
:10EE3000031D01F1200C70B50E68103151F80C5C07
:10EE4000103351F8084C51F804EC614543F8106C4C
:10EE500043F80C5C43F8084C43F804ECECD1098807
:10EE6000198011685368C0F82610C0F82A3070BDA8
:10EE70000379024613F0070004D0507910F0070020
:10EE800018BF0120704700BF0379024613F0070046
:10EE900004D0507910F0070018BF0120704700BF60
:10EEA0000171704700797047417170474079704730
:10EEB0000B0A8171C3717047C0887047027943792A
:10EEC00002F0070203F00703501E591E02400B40D8
:10EED00013430CBF01200020704700BF0171704731
:10EEE0000079704741717047407970470B78037122
:10EEF0004B7843718B788371CB78C3710B79037234
:10EF00004A790B7902F00F0CD20943EA0C2343EA49
:10EF1000C2331B1243728B798372CB7903F00F03D8
:10EF2000C3720B7A03734B7A43738B7A03F00F032C
:10EF30008373CB7AC3730B7B03744B7B03F00F0398
:10EF40004374CB898374CB891B0AC3740B8A037502
:10EF50000B8A1B0A43758B7C8375CB7CC3750B7D39
:10EF600003764B7D43768B7D03F0F002C3F30303FE
:10EF700013438376CB7DC3760B7E0377B1F81930CC
:10EF80004377B1F819301B0A8377CB7EC3770B7FA9
:10EF900080F820304B7F80F821308B7F80F8223042
:10EFA000CB7F80F8233091F8203080F82430B1F8FE
:10EFB000213080F82530B1F821301B0A80F8263046
:10EFC000704700BF0B7803714B7843718B78837166
:10EFD000CB78C3710B7903724B794372CB88837200
:10EFE000CB881B0AC37270470B6803710B681B0A3E
:10EFF00043710B681B0C83710B681B0EC3710B797B
:10F0000003724B7943728B798372CB79C3720B7A1B
:10F0100003734B7A43738B7A8373CB7AC3730B7B03
:10F020000374B1F80D304374B1F80D301B0A8374CA
:10F03000704700BF0B7803714B7843718B788371F5
:10F04000704700BFFB2901D84170704740F2A961A9
:10F050002A2008B5FAF7FEF903781BB1406890F84A
:10F060000A3303B97047002380F80A3304F092BDD5
:10F07000024B987DC04300F001007047B00D0021A5
:10F08000034B987D80F00200C0F34000704700BF42
:10F09000B00D0021034B9B7DC3F38003184380F028
:10F0A00001007047B00D00212DE9F043047A87B0CC
:10F0B000D4B1012C13D1878804A9C688D0F8008068
:10F0C0003846FEF78FF830B9059DA8357EBB012381
:10F0D0001C4685F82430204607B0BDE8F0830024A4
:10F0E000204607B0BDE8F083868802A9C488076877
:10F0F0003046FEF777F8002851D1039DA835002C43
:10F10000E5D03046FBF7FEFA0646002800F0858081
:10F11000214619F08DFF18B1444B5B88A34243D2BE
:10F12000012400F027F9204607B0BDE8F0833846F7
:10F13000FBF7E8FA074600286FD0314619F078FF50
:10F140000028EDD0394B5B88B342E9D3014601AAD0
:10F1500038464FF000091AF0D3FA019BA3F800904B
:10F1600083F8029095F8243001984B450CBF214656
:10F170000221FFF72DFD019841463246033017F07A
:10F18000D7FB3146384619F0D2FF0446002848D054
:10F190009DF8103083BB002385F824309BE70124C1
:10F1A000204607B0BDE8F08301466A4630464FF07E
:10F1B00000081AF0A5FA009B0221A3F8008083F84A
:10F1C00002800098FFF704FD00982246394603307C
:10F1D00017F0AEFB2146304619F0A9FF044600B3F4
:10F1E0009DF80830002BD6D0039890F80A3373B9F5
:10F1F0000023A0F80233CEE7059890F80A33002BDD
:10F20000F6D080F80A9304F0C5FC0598F0E780F882
:10F210000A8304F0BFFC0398EAE767212B20FAF782
:10F2200019F97C212B20FAF715F900BFB00D002148
:10F23000032201230A800B71704700BF30B583B0F1
:10F24000002957D0002288800C464A72FBF728FA22
:10F2500005461AF028FA0146002846D001AA284699
:10F260001AF04EFAE08000283AD0FB2833D80198F3
:10F27000FFF7B6FC012801D0022818D120722068BF
:10F28000D0B10199E288033117F052FB28461AF0F9
:10F290005CFAD8B1002128461AF02DF888B1174B36
:10F2A000DA7D12B11A8B013A1A8303B030BD4FF4E4
:10F2B0008E711020FAF7CEF840F223111020FAF7E1
:10F2C000C9F840F22D111020FAF7C4F84FF49471E8
:10F2D0001020FAF7BFF84FF486711020FAF7BAF849
:10F2E0004FF485711020FAF7B5F840F2051110209F
:10F2F000FAF7B0F8FC211020FAF7ACF8B00D0021B5
:10F30000094900220B464A604A6103F8040B8A61EE
:10F31000DA608A84C3E90122C1E9072201220433A9
:10F320000A74C1E901337047CC0D0021084A00235B
:10F33000111D53609384CB60C1E90133C2E90533E9
:10F34000C2E90733012304311374C2E90111704784
:10F35000CC0D0021014B024A1A6070475800002171
:10F360003DF20001014B024A1A607047580000212B
:10F370003DF200010D4B1A7F02B170470C4A9A61B1
:10F3800002221A77EFF3108072B603F1080299682F
:10F390005A6111B1097A012900D05A6805491160F2
:10F3A000596000B962B6187817F05ABACC0D00212E
:10F3B00031F20001E00D00212DE9F84FAD4E074676
:10F3C000DFF8B482DFF8B4A2DFF8B492B5682B7A24
:10F3D0002A2B4ED02B7A012B0DD0EFF3108372B66F
:10F3E000B2681268B26053B962B62C7A54B9B56883
:10F3F0002B7A012BF1D100242046BDE8F88F2C7A1E
:10F40000002CF4D0A31EE4B22F2B00F26781DFE8BA
:10F4100013F0D300A1000001500070005800A100BB
:10F42000390013013900390039001C013900650128
:10F43000500070005800390039005000700078000A
:10F440003B01780039004D01580058003900500048
:10F4500039003900B30039005000650144019900BA
:10F46000DC00F2006800680068000701BB00CA0009
:10F47000990098F81730002BACD0B8F81830002B52
:10F48000A8D1B8E76B68002B00F056814FF0000B55
:10F490003946284698470023212C2B7200F0A18082
:10F4A000142C00F00B81222C5CD0BBF1000F8DD10D
:10F4B00013E06B68002BE9D140F2BB111020F9F783
:10F4C000C9FFDAF80030002B00F0058122463946EA
:10F4D000686898471E2C40F0FE8004242046BDE852
:10F4E000F88F6B68002BD1D140F2C7111020F9F7CB
:10F4F000B1FF6B68002BC9D140F23F211020F9F712
:10F50000A9FFD9F80030002B00F0E580D5F804B051
:10F5100022463946584698473B781E2B06D01B2B6F
:10F5200040F0D9803B79002B00F0D5800421BBF856
:10F530000800FAF7A7FE0028CFD04FF40071102082
:10F54000F9F788FF6B68002BA0D140F26F211020E3
:10F55000F9F780FF6B68002B98D140F24B21102007
:10F56000F9F778FFFFF784FD00287FF42FAFBBF198
:10F57000000F7FF42BAFB0E76B68002B86D14FF400
:10F580002B711020F9F766FF6B68002B00F0CF801D
:10F5900039462846984700232B7200289DD008241E
:10F5A0002046BDE8F88F6B68002B7FF46FAF40F208
:10F5B000B7211020F9F74EFF6B68002B7FF466AF80
:10F5C0004FF4D2711020F9F745FF1F234FF0000BC5
:10F5D0003B80D5F8090078600023212C2B727FF442
:10F5E0005FAFFFF74DFD00287FF4F0AEBBF1000FD9
:10F5F0007FF4ECAE71E7234B1B68002B73D06A6875
:10F60000002A78D002241088394698472046BDE861
:10F61000F88F0CF0ADFD002867D14FF0010B3AE7F1
:10F620006B68002B71D00022394628462A72984711
:10F6300000283FF452AFB2E76B68002B7FF426AF8F
:10F6400040F281211020F9F705FF6B68002B65D08F
:10F650001C882046FBF756F800285BD001230F22B8
:10F66000FC8000213A8004243B813B7119F043FE69
:10F67000C2E600BFCC0D0021B00D00215C000021CE
:10F6800060000021580000216B68002B7FF4FEAE63
:10F690004FF403711020F9F7DDFE6B68002B7FF447
:10F6A000F5AE40F2AD111020F9F7D4FE6B68CBB384
:10F6B000394628464FF0010B9847ECE6B87B00F03E
:10F6C0000100FFF7E7FC00287FF480AEBBF1000FDC
:10F6D0007FF47CAE01E74FF0000BDCE640F2BD2189
:10F6E0001020F9F7B7FE022486E66B6843B139466D
:10F6F0002846984780E640F29F211020F9F7AAFE9D
:10F7000040F233211020F9F7A5FE40F2CF1110206E
:10F71000F9F7A0FEAE211020F9F79CFECE211020B3
:10F72000F9F798FE40F263211020F9F793FE40F2BA
:10F73000E1111020F9F78EFE40F296211020F9F722
:10F7400089FE00BF037A10B5BBB941600272EFF3C6
:10F75000108472B60B4B03F108020260996811B174
:10F76000097A012900D05A681060586004B962B65D
:10F770001878BDE8104017F073B840F21731102028
:10F78000F9F768FECC0D0021037A03B1704710B47D
:10F7900041600272EFF3108472B6094B03F1080264
:10F7A0000260996811B1097A012900D05A68106085
:10F7B000586004B962B6187810BC17F051B800BF91
:10F7C000CC0D00212DE9F04100F10A0C4FF00008AA
:10F7D000162786460D460E1D8EF8088033462F806C
:10F7E000DCF80000DCF80410DCF808209EF8084083
:10F7F00007C3002CF0D1BDE8F08100BF70B586B022
:10F8000005460C46FFF73CFC60B923462B2223F843
:10F81000042BD5F80A00D5F80E106A8A03C31A80A3
:10F8200006B070BD0022A5F5EB7369462A721E88EA
:10F8300030461BF089FBD8B9BDF8063003A8BDF8E7
:10F840000810BDF80220ADF80E30BDF80430ADF858
:10F850000C60ADF81010ADF81220ADF814301BF0AC
:10F8600040FB0028D1D04FF483712C20F9F7F2FD32
:10F87000FD212C20F9F7EEFD4068704710B590F897
:10F880006E40B1F804E014F00C0FB1F808C022D1BA
:10F8900093B3137813F00C0F04D0BEF5296F38BF63
:10F8A0004FF4296E90F86F3013F00C0F03D153789A
:10F8B00013F00C0F04D0BCF5296F38BF4FF4296C3E
:10F8C000CB884A88A0F84EE0A0F84C20A0F8503031
:10F8D000A0F852C010BDBEF5296F90F86F4038BF38
:10F8E0004FF4296E14F00C0FE5D1002BE8D05378BB
:10F8F00013F00C0FE4D0DEE790F86F3013F00C0F2C
:10F90000D9D1DDE7BDF800C08182C2820383A0F8AF
:10F910001AC070471B234FF01B120384838342617C
:10F9200003828260C0F82A20838451B94FF4A47204
:10F93000064B4284C28383614282C360C0F82E308A
:10F9400070474FF42962024BF3E700BF48014801BA
:10F95000900A900A0346B0F84420B0F8500010B561
:10F96000824293F86F105C8F28BF024611F00C0F93
:10F97000D88F4FD1B3F84810B3F852C0614528BFB3
:10F980006146884208BF9442B3F842C0D98714BF89
:10F990000120002061455A87B3F838E038BF61463E
:10F9A000B3F83CC0A3F84210B3F840108A4238BF05
:10F9B0000A46B3F84C10A3F84020B3F846208A4218
:10F9C00028BF0A4693F86E1011F00C0F1FD1B3F840
:10F9D0004A10B3F84E40A14228BF214693F8644034
:10F9E000022C09D172454FF0000428BF72466145D0
:10F9F00083F8644028BF6146964518BF40F0010077
:10FA00001A8799878C4518BF40F0010010BD4FF44C
:10FA10002961E3E74FF42961B3E700BF13468C4641
:10FA200021220B4900B5BCF814E05881BCF816003F
:10FA3000A3F80CE0D881BCF81800BCF81AC05DF837
:10FA400004EB18821846A3F812C0FFF77BBE00BF74
:10FA5000FDF7000130B5CB89CC8DB1F808E0B1F8E5
:10FA60000CC09C4250814889A2F80CE0A2F80EC05C
:10FA70001082538211D00125147D65F300041475A2
:10FA800048851046A1F82CE01422CB85A1F830C09F
:10FA90000849BDE83040FFF777BE4C8D8442EAD17B
:10FAA0000C8E6445E7D18D8DB5EB0E0518BF012591
:10FAB000E2E700BFC5F70001F8B5436941F64B5EC8
:10FAC00090F86EC073458CBF4FF0960E4FF04D0E00
:10FAD00090F86F501CF00C04038F2CD09B014FF456
:10FAE0002967B0F8406003F574739BB29F4228BF4A
:10FAF0001F4615F00C0F36D1012D56D0022D71D1B5
:10FB0000B0F852300F36B0F84800B6008342B6B2B3
:10FB100028BF03463648B342007828BF3346002842
:10FB20005BD106323B4402EB4E0E73448B4294BFD2
:10FB3000C81A0020F8BDBCF1010F32D0BCF1020F91
:10FB400050D10F339B009BB2B0F84A70B0F84E60B2
:10FB5000B74228BF3746B0F840609F4228BF1F46D3
:10FB600015F00C0FC8D0B601214806F57476007860
:10FB7000B3B2B3F5296F28BF4FF429630028D0D062
:10FB80004FF46960834238BF03461CBBBCF1010FD0
:10FB900025D0BCF1020F25D1E820874238BF0746A7
:10FBA000BFE70E33DB009BB2CEE7B0F8525006F150
:10FBB0000E03B0F84800DB00A8429BB228BF2846DD
:10FBC000834228BF03460A4800780028A9D04FF492
:10FBD000E470D7E74FF46960DFE7E820D2E74FF43D
:10FBE000E470DAE740F226210620F9F733FC00BF83
:10FBF000F20D00212DE9F04141F64B5E446990F889
:10FC00006EC0744594BF4FF04D0E4FF0960E90F8B5
:10FC10006F601CF00C05038F34D09B014FF42968F2
:10FC2000B0F8407003F574739BB2984528BF9846AE
:10FC300016F00C0F3ED1012E5ED0022E79D1B0F815
:10FC4000486007F10F03B0F852709B00BE429BB2B0
:10FC500028BF3E46B34228BF3346384E3678002E82
:10FC600062D1063243449644026B7344944294BF7B
:10FC7000C1EB0401C1EB0201994238BF194641634F
:10FC8000BDE8F081BCF1010F32D0BCF1020F50D1C0
:10FC90000F339B009BB2B0F84A80B0F84E70B84565
:10FCA00028BFB846B0F84070984528BF984616F06F
:10FCB0000C0FC0D0BF01214E07F574773678BBB268
:10FCC000B3F5296F28BF4FF42963002EC9D04FF434
:10FCD0006966B34238BF33461DBBBCF1010F25D066
:10FCE000BCF1020F25D1E825A84538BFA846B8E7E2
:10FCF0000E33DB009BB2CEE7B0F8526007F10E0383
:10FD0000B0F84870DB00BE429BB228BF3E46B3420B
:10FD100028BF3346094E3678002EA2D04FF4E47641
:10FD2000D7E74FF46965DFE7E826D2E74FF4E475DB
:10FD3000DAE740F226210620F9F78CFBF20D0021CC
:10FD4000006801F19C03984203D9401A9C3840088E
:10FD500070470020704700BF014B1878704700BF04
:10FD6000F20D0021C34300EA400203EA430302EA22
:10FD7000420203EA430302EA420203EA430302EABD
:10FD8000420203EA430302EA420203EA430302EAAD
:10FD9000420203EA430313430FD1C31683EAA0636D
:10FDA0005A1E1A4210B5044605D0E3B25A1E13403B
:10FDB0005A1E134203D1002010BD00207047A0B28C
:10FDC00000F032F90B28F6D8204600F00FF9182879
:10FDD000F1D8A3B2B3EB144F07D0074B63405A1EC0
:10FDE0001A4214BF0120002010BD84EA142313F02E
:10FDF000FF1FE0D0F1E700BFD6BE898E2DE9F047A6
:10FE00004FF0000982B02326DFF810814F4600F042
:10FE1000B9F80446FFF7A6FF0546002866D0CDE9ED
:10FE2000007703E0009B9B699C4254D06846FAF738
:10FE300077FA0028F6D00123CDE900778DF8063057
:10FE400003E0009B9B699C4245D06846FAF768FA3C
:10FE50000028F6D00323CDE900778DF8063003E0C3
:10FE6000009B1B689C4236D06846FAF759FA002876
:10FE7000F6D00423CDE900778DF8063003E0009B2F
:10FE80001B689C4227D06846FAF74AFA0028F6D049
:10FE900000214FEA144A08EA94294FF0160E4FF059
:10FEA0001F0C084610E04FEAC932BEF1010E4FEABE
:10FEB000CC3392B29BB24FEA59094FEA5C0C42EA4A
:10FEC000500043EA510113D08AEA000361EA0303B8
:10FED0000133E8D1A146013E01D0002D97D1B9F1FF
:10FEE000000F15D0484602B0BDE8F0870125F2E7C3
:10FEF0000B4B2AF4004542F6AA22A14653449542F0
:10FF000018BF012B8CBF0125002585F00105E2E714
:10FF100040F267110F20F9F79DFA00BFE0FF3F00A4
:10FF2000ACAAFFFF38B5094C08212046F9F726FD99
:10FF3000D4E900231343F7D0054D08212846F9F7EB
:10FF40001DFDD4E902231343F7D038BDF40D002181
:10FF5000FC0D002109490A48D1E90023534002FB66
:10FF600000F083EAB2124FEAF06082EA43224FEADD
:10FF7000F34300EB8000C1E900237047F40D00213A
:10FF8000BB79379E09490A48D1E90223534002FB55
:10FF900000F083EAB2124FEAF06082EA43224FEAAD
:10FFA000F34300EB8000C1E902237047F40D002108
:10FFB000BB79379E002802DB884203DA704749424A
:10FFC0008842FBDA08B27047430800F0550003F09E
:10FFD00055031844830800F0330003F0330303444F
:10FFE00003F00F0000EB1310704700BF80EA6003BE
:10FFF000580803F0553300F055301844830800F0DA
:020000040101F8
:10000000333003F033331844030900F00F3003F0AA
:100010000F331844030A00F0FF1003F0FF131844D5
:1000200000EB1040C0B2704740F34E0345F2555C00
:1000300043F233319BB2584040F60F730CEA500242
:1000400000EA0C00104400EA010201EA90010A44AF
:1000500002EA030003EA1213184400EB1020C0B2B6
:10006000704700BFF8B5164B06460C4630F8DC5C0E
:100070001B680BB134389847124B1B680BB12846EC
:1000800098470C230027A4F80550284623802771A1
:10009000737AE371FAF704FB19F06EF960B1284640
:1000A000FAF716FF39462846FAF7ECF828460121F8
:1000B000BDE8F840FAF7E6B860216320F9F7CAF91D
:1000C00064000021680000212DE9F04109230F465A
:1000D00086460E46A0F5077800F10A0C002227F8A4
:1000E000043B8EF808203B46DCF80000DCF80410E6
:1000F000BCF808509EF80840A8F82A2003C31D80C9
:100100003271002CEDD1BDE8F08100BF0A22A0F5CC
:1001100079730A801B888B800369C268C1F80A3032
:10012000C1F80620838ACB81704700BF0D22A0F55D
:1001300036730A8090F80AC0827B1B8881F804C05D
:100140000A72CB80704700BF0E22A0F536730A807A
:10015000827A1B880A71CB80704700BF02460B462B
:100160004FF0080C23F804CBD2F80D10B2F811C0F0
:10017000D0F80900D27C03C3A3F800C09A7070477E
:1001800070B504780D46ECB946682346214696F8CA
:10019000C62006F1A800FDF7D7FA88B3AB680121A5
:1001A0006A68204603F00703A6F8024186F80411A6
:1001B000C6F81A31042386F8C630134B1340C6F82C
:1001C000163170BD4368D3F8B42012F0010117D185
:1001D000A86842F001026E680C46C3F8B42000F033
:1001E0000702A3F802112046C3F81A2193F804214C
:1001F000013283F80421044A3240C3F8162170BD4D
:100200000124204670BD00BF2F4904372DE9F84373
:100210004668054690F800800F4606F1A8040721BD
:100220004346627F204606F5D479FDF78DFA70B318
:10023000BB687A6803F00703C4F87230164B1340AA
:10024000C4F86E30002384F858306377B8F1000F9B
:1002500002D16B6883F86B8199F868401CB1002467
:100260002046BDE8F883338809F1600089F86940C9
:10027000A9F86A307A68BB680849C9F86C20082276
:10028000C9F87030FFF75EFA2046BDE8F883012414
:100290002046BDE8F88300BF2F4904375D01010106
:1002A000436893F8102203F5D47002B17047B3F895
:1002B00000C01A2308220349A0F86AC060304372C4
:1002C000FFF740BA5D01010110B5044610F060FC73
:1002D000034B01F007010340A160636010BD00BF44
:1002E0002F49043730B5456883B00C4610F050FCF8
:1002F000094A01F0070195F816C16B460240A8357E
:100300000CEA020CCDE900218DF800C003CB60603F
:10031000A16003B030BD00BF2F49043710B5446859
:1003200000210378A834627F2046FDF70DFA10B152
:100330000423637710BDAA211C20F9F78BF800BFB6
:1003400038B5057804468DB14268D2F8B410CB07B1
:100350001DD592F80431013B5BB2002B82F80431C9
:1003600011DB21F00101C2F8B41038BD40682B4602
:10037000294690F8C620A830FDF7E6F958B1636821
:1003800083F8045138BDB9211C20F9F763F8B7216F
:100390001C20F9F75FF8B2211C20F9F75BF800BFC9
:1003A0001023A0F5DB700B8003888B80704700BFA3
:1003B00001234FF0000C00B5A0F5847E0B8081F87E
:1003C00004C080F808C0BEF80020037AA1F8052018
:1003D000427ACA71D0F80A208A60002BF1D15DF808
:1003E00004FB00BFF8B547680E460578082107F101
:1003F000A80497F8C5202B462046F5B9FDF7A4F9C7
:10040000002843D094F85F30990722D5DB070FD43A
:10041000002D4FD0E36813F002015DD194F85C2009
:1004200043F00203A4F85A100132E36084F85C2020
:10043000637F012B24D00020F8BDFDF785F900284B
:10044000E0D1D7F8B430980729D494F85F309907F1
:10045000DCD43046FEF7A4FC84F86900B6F8052029
:1004600094F85F30A4F86A20B6F8072043F0020140
:10047000A4F86C20DA0784F85F1012D4CBB2C5E779
:1004800000231846637784F85830F8BD2B4697F858
:10049000C62029462046FDF757F90028B2D1012091
:1004A000F8BD03220E4904F16000FFF76DF994F8DE
:1004B0005F30ABE72B46A27F29462046FDF744F983
:1004C00030B10123A4F85A50A37784F85C30AFE729
:1004D00048214020F8F7BEFF4F214020F8F7BAFF2F
:1004E000B1030101F8B50578BDB9466896F8073142
:1004F00006F1A80406F5AC77980728D42B46627F4E
:1005000000212046FDF720F9A8B3012300226377DC
:1005100084F85830A4F85420F8BD446894F80731A2
:1005200004F5AC77990720D5D4F8B4309A070BD5E9
:1005300094F80421013A52B2002A84F8042116DB0F
:1005400023F00203C4F8B4300023BB74F8BD2B467B
:10055000204696F8C6202946FDF7F6F80028F3D085
:10056000002386F80451BB74F0E7A834C6E7802165
:100570004020F8F76FFF6E214020F8F76BFF00BFB7
:1005800029230B80D0F80A00486070472DE9F0431A
:100590000023A0F51D75A0F5E67483B00B8080469E
:1005A00095F86F000FF01AF8A3683A4E074603F566
:1005B000006396F9001043F307321B13914226DDC6
:1005C0005B4296F901205BB213447F2B2ADC13F1C6
:1005D000800F57DB4FFA83F9B9F1000F14D0A8F55B
:1005E000E4786FF000412268D8F800308B4208BFF1
:1005F000B2F1FF3F08D013F0D5FA2268D8F80030E6
:10060000904271EB030310D203B0BDE8F08396F97A
:1006100002109142F8DA5B4296F903905BB24B44C8
:100620007F2BD4DD4FF07F09D9E728886946FCF796
:10063000D9FD50BB791C4A4668460223C9B20EF068
:10064000E5FF0028E0D1367973019B1B62EB0202C3
:10065000520242EAD3525B029B1942F10005990112
:10066000AA01C91A42EA936262EB05028E1942F1AD
:10067000000513F097FA801945EB01052060C8F8D2
:100680000050C1E76FF07F09A9E789217A20F8F7C8
:10069000E1FE00BF040E00212DE9F8430446D0F826
:1006A0000490FDF77BFB7F28666809F1A8080546E2
:1006B00086F8C10024D037464149A8368B68D7F860
:1006C000B02002FB03F0C3F5805397F8DB2005FB55
:1006D00003F387F8C22003EB2033C7F8B0300A7B5E
:1006E000002A36D196F91B1097F82D206B1A1BB2F1
:1006F000002BB8BF5B429BB2934201D3FF2A01D1CA
:10070000BDE8F883337F0133DBB2337797F82E20CF
:100710009A4201D37F29F3D10023F576337799F8F4
:100720002C30012BECD1606890F8B03100F5D4701A
:10073000002BE5D1B9F800301F222249438198F8F7
:100740001930037398F81A304373BDE8F843FEF785
:10075000F9BF03F5006391F9000043F307321B135F
:10076000904225DD5B4291F901205BB2134403F115
:100770008002FF2A02D85BB2002BB3D06FF0004397
:10078000D6E900129A4208BFB1F1FF3FAAD013F098
:1007900009FAD6E90023904271EB0303A2D3606803
:1007A0003122094900F5D470CC30FEF7EDFF99E70E
:1007B00091F90200904295DA5B4291F90320D4E767
:1007C000040E0021810501018D0501010B4B00F58F
:1007D00000621B78584242F3073340B218447F2826
:1007E00007DC10F1800F06DB40B220EAE070C0B2F7
:1007F00070477F2070470020704700BF040E002123
:1008000007230B80D0F80A004860704702460B4669
:100810004FF02A0C23F804CBD2F80D10D0F80900C1
:10082000527C03C31A70704730B52F238C4600F1F9
:10083000090E00F129042CF8043BDEF800000EF14B
:10084000100E5EF80C1C65465EF8082C0CF1100CBE
:100850005EF8043CA6450FC5EFD1BEF80030ACF8F9
:10086000003030BD144B421E082933F811304FEAD6
:10087000C21203F2E73310B4104CA4FB03434FEA57
:10088000931311D0042908D00229134410BC14BFBB
:10089000F021602101FB0030704740F2BE2113447B
:1008A00010BC01FB003070474FF4D261134410BC00
:1008B00001FB0030704700BF44510301D34D62106B
:1008C000D928844628BF4FF0D90C0CF1300C1FFA00
:1008D0008CFC30B5BCF1FF0FBDF80C40864628BF3C
:1008E0004FF0FF0CA00737D0A00701F5A57124D564
:1008F000082A00F0BB80042A00F05081022A14BFAD
:100900004FF414754FF4967512F00C0F294400F053
:100910008C8001F61445E00705F1980C40F19680B3
:10092000082A00F0E480042A00F03581022A0CBF76
:100930006421C0210CEB010030BD002B5FD0082AE0
:1009400000F0E381042A00F0FE81022A40F6480507
:1009500008BF4FF48565D7E701F5A570DBB1082A1C
:1009600000F01F81042A00F0FE80022A00F0E581D9
:10097000BEF1D90F01F69210DED9AEF1D902C54B06
:1009800092B2F63283FB02131344DB1140F692124B
:1009900002FB030030BD082A00F01581042A00F094
:1009A000AC80022A00F0C2810CF1050CBEF1D90F17
:1009B0001FFA8CFC00EBCC0C0CF12800BCD9AEF17A
:1009C000D903B5491FFA83FEA1FB0E31AEEB01033B
:1009D00001EB5301C1F3C711C1EB411340F6921271
:1009E000C1EBC30302FB0100AEEB03039BB2002B80
:1009F000A2D00833282208249BB2053310E1082A2C
:100A000000F0DE81042A00F08381022A00F0768162
:100A10000CF1050C282508201FFA8CFC0CFB005C4F
:100A200012F00C0F61447FF474AF082A62D0042ADC
:100A300000F09680022A14BF4FF4B075B4259C31A3
:100A4000E0070D4405F1980C3FF56AAF8BB1082A19
:100A500000F0A981042A00F07381022A00F0E780E7
:100A6000BEF1D90F05F50E6087D830BD41F2D02513
:100A70004AE77346F12B28BFF123082A00F066816C
:100A8000042A00F04D81022A00F008811333BEF1E0
:100A9000D90F98B20CEBC00C0CF128007FF64CAFCC
:100AA000AEF1D90E7C4B1FFA8EFEA3FB0E23AEEBEC
:100AB000030203EB5203C3F3C713C3EB431240F625
:100AC0009211C3EBC20201FB0300AEEB02039BB227
:100AD000002B3FF431AF0833282208219BB20533A5
:100AE00000F5A57C03FB012303EB0C0030BD4FF4A4
:100AF000CA611FE74FF43565A1E70CF1050C4FF40F
:100B0000BF7110231FFA8CFC0CFB031CBEF1D90F24
:100B100060447FF611AFAEF1D9035F49042A1FFA92
:100B200083FEA1FB0E31AEEB010301EB5301C1F3D8
:100B3000C71140F09780C1EB411341F20832C1EB7D
:100B4000C30302FB0100AEEB03039BB2002B3FF497
:100B5000F3AE08334FF4BF7210249BB205335FE04D
:100B600040F2EE356BE741F2BE1CBEF1D90F604496
:100B70007FF6E2AEAEF1D90E464B042A1FFA8EFE86
:100B80000EF1F60E83FB0E1373444FEAE31363D1A9
:100B900041F20832FCE640F2AE21CBE640F2CE55FF
:100BA000B2E644F2DA32BEF1D90F01EB02007FF671
:100BB000C3AEAEF1D901374B89B2F63183FB0143A5
:100BC0000B44DB11E4E60CF10503BEF1D90F9BB237
:100BD00000EB831C0CF5C8707FF6AEAEAEF1D90EFB
:100BE0002D4B44F2DA311FFA8EFEA3FB0E23AEEB3F
:100BF000030203EB5203C3F3C713C3EB431201FB1E
:100C00000300C3EBC203AEEB030E1FFA8EF3002BFF
:100C10003FF492AE08334FF4C87240249BB20533C0
:100C200000F5A57C03FB042303EB0C0030BD4FF45F
:100C30008561BEF1D90F0CEB01007FF67DAEAEF100
:100C4000D901144B042A89B201F1F60183FB014357
:100C50000B444FEAE3139BD0022A7FF497AE40F295
:100C6000725295E6022A7FF4B7AEC1EB411340F20F
:100C70007252C1EBC30302FB0100AEEB03039BB254
:100C8000002B3FF459AE0833182204249BB20533DD
:100C9000C6E700BFC9F9A98491F35309133318209B
:100CA00004219BB203FB0103BEF1D90F03EB0C003F
:100CB0007FF642AEAEF1D90E514B042A1FFA8EFEDA
:100CC000A3FB0E13AEEB030103EB5103C3F3C713F6
:100CD0007ED1C3EB431241F20831C3EBC20201FBE8
:100CE0000300AEEB02039BB2002B3FF425AE0833AA
:100CF0004FF4BF7210219BB20533F1E60CF1050CE5
:100D0000182504201FFA8CFC88E644F29025FBE5A8
:100D10000CF1050C4FF4BF7510201FFA8CFC7DE61A
:100D200013334FF4BF7010219BB2BBE70CF10503E6
:100D300018211FFA83FC0423E6E64FF4856C14E7C0
:100D400041F2BE1175E741F2BE15DDE51333BEF188
:100D5000D90F98B20CEB801C0CF5C8707FF6ECAD87
:100D6000AEF1D90E264B44F2DA311FFA8EFEA3FB08
:100D70000E23AEEB030203EB5203C3F3C713C3EB23
:100D8000431201FB0300C3EBC203AEEB030E1FFAD9
:100D90008EF3002B3FF4D0AD08334FF4C8724021DE
:100DA0009BB205339CE644F22830BEF1D90F2844AB
:100DB0007FF6C2ADAEF1D901124B44F2DA32FBE656
:100DC0000CF1050C4FF4C87540201FFA8CFC25E689
:100DD000022A7FF472AEC3EB431240F27251C3EBAE
:100DE000C20201FB0300AEEB02039BB2002B3FF4F7
:100DF000A3AD0833182204219BB2053370E600BF6F
:100E000091F35309C9F9A9842DE9F8432B4E4FF00A
:100E1000000815460746D6F800C062F307080C46DE
:100E2000DCF80F3062F30F288B619CF815309CF8CA
:100E300014201B0443EA02239CF8132013430B6283
:100E4000BCF81900FCF70EFF336881466061987D9D
:100E50004946FCF719FF336820854946B3F8170067
:100E6000FCF73AFF33686062B3F81B20A283B3F843
:100E70001D20E283D3F81F20C4F8CE2093F823204E
:100E800084F8D22093F82430A4F86E8003F01F0277
:100E90005B0984F8D92084F8F832FF2315F00C0F91
:100EA00004F1300084F8703014BF01210021FEF7F6
:100EB00031FD3B7C84F87230BDE8F883140E0021CC
:100EC00090F8D63010B50446A3BB2378FF29084616
:100ED00084F8D7301DD004F1D90204F1D801FBF712
:100EE0003FFF68B394F8D83043F0020384F8D83059
:100EF00094F947307F2B1ED07F2084F8DF302022EA
:100F0000124984F8470004F1CE00BDE81040FEF716
:100F100019BC0F4B19680B4613F8032BC2F3801250
:100F200084F8D820D1F80320C4F8D9209B88A4F8ED
:100F3000DD30DDE710BD40F66C612D20F8F78AFA50
:100F400041F208012D20F8F785FA00BF0D080101D4
:100F5000140E002170B515238E460E4600F1090CC3
:100F600000F129042EF8043BDCF800000CF1100C11
:100F70005CF80C1C75465CF8082C0EF1100E5CF841
:100F8000043CA4450FC5EFD19CF8003001248EF835
:100F900000303379F47103B970BDB6F805502146BD
:100FA000284618F037FE0028F6D00088F9F790FFA1
:100FB00021462846F9F766F90028EDD04FF4147160
:100FC0002D20F8F747FA00BF70B50D460446486972
:100FD0001646FCF72FFEAB8BEA8BA4F8A830A4F8DA
:100FE000A600A4F8AA20A37E95F8F82284F8AC20E5
:100FF0005BBB94F882301BB194F86830012B4BD066
:101000000022C4F89A20A4F89E20284BFF2E1B68CB
:101010001A78C2F3801284F893202FD0D3F80310EB
:1010200004F194023046C4F8A01004F19301B3F81F
:101030000730A4F8A430FBF793FE90B394F89330F4
:1010400043F0020384F8933070BD94F86830012BAC
:10105000D6D194F86E3003F0C003402B05D094F83D
:101060008220002ACCD0002BCAD1D4F86920B4F851
:101070006D30C4F89A20A4F89E30C6E7D3F8030078
:101080000022C4F89400B3F80730C4F8A020A4F8F4
:101090009830A4F8A42070BD94F86E3003F0C0031B
:1010A000E1E740F68B412D20F8F7D4F9140E00212A
:1010B000F8B50446C07E0E46FBF73AFEA37E0BB1A0
:1010C000054680B994F8823063B1237F53B194F818
:1010D0006830012B1CD0314604F16900BDE8F840AE
:1010E000FAF748B8F8BDE07EFBF72CF80028E9D104
:1010F00004F16907012328463246394684F86830EE
:10110000FAF702F8E17E3846BDE8F840FBF798BFF1
:1011100094F86E3003F0C003402BDCD1FBF778FF6E
:10112000324604F16901BDE8F840F9F7EDBF00BFB0
:101130004FF0180C0A46034622F804CBD0F80A00F8
:10114000B3F80EC04860C0B2A2F804C018B133F8BA
:10115000AE3C1B0700D5704710B5CC880121204656
:1011600018F058FD38B10088F9F7B2FE0121204689
:10117000F9F788F800B910BD40F28F212D20F8F75B
:1011800069F900BF2DE9F043914D87B0914B0026DE
:10119000AA6A0446904902A8526804F130070293F3
:1011A0008E4B6E7184F881600592049303912E82B8
:1011B000AE60AE7110F016FB10F024F910F0DAF901
:1011C00010F0CEFB0FF070FD854810F0E7F9854870
:1011D00010F002FB304615F0F5FC384601F09EFB9E
:1011E000384601F0A1FB10F0E3F92179252010F039
:1011F00083F894F9100010F0C5F92179304611F008
:10120000DDF8E86028B901232B71002007B0BDE8A4
:10121000F08304F15001E06C19F023F9064604F163
:101220005801E06C19F02CF907462EB194F82430DF
:1012300013B14FF0010803E0002F40F08280B84660
:10124000237F23B9A37E13B9638858073DD56FF078
:101250000043D4E918129A4208BFB1F1FF3F73D09E
:1012600012F0A0FCD4E91823904271EB03036BD376
:10127000FBF7CCFC804612F095FC4FEA48134FEA8E
:10128000D862B3EB080362F10002520242EAD35281
:101290005B0213EB080342F1000C9A014FEA8C1E2B
:1012A000D21A4EEA936E6EEB0C0C12EB08034CF163
:1012B0000002181842EB0101C4E91801012120467F
:1012C000FFF7F6FE6388590762D43E4394F88430F2
:1012D000F6B2002E41D1002B3FD1FBF79BFD2868D1
:1012E0000330FBF75DFE6388A874DB078DD5266AA3
:1012F00000230122FF2106F10A0785F82010CDE91D
:1013000000338DF806206846F9F70AF800287FF4C4
:101310007CAF009CA642F6D03B46727A04F10A01EB
:10132000607AF9F785FE0028EDD0A2782E4B85F87B
:101330002020D4F80320C5F82120B4F807209A8093
:1013400063E794F825807BE7B8F1000F90D13E4326
:1013500094F88430F6B2002EBDD06388DA06BCD48F
:10136000666CC6F30B26FEF7F5FDC0F30B039E4239
:10137000F9D094F84630C0F30321002284F84500E8
:1013800023F00F030B4384F8463084F88420A4E74D
:10139000E07EFBF7D9FC8046002896D01021FCF7B0
:1013A000A5F8002891D14FF00109404604F17708D3
:1013B0004A4684F876904146F9F7A6FE41462868E9
:1013C000FDF72CF949462868FDF73EF97DE700BF97
:1013D000140E0021D91A0101E9160101CD150101F0
:1013E000D6BE898E55555500350E002103292DE9AD
:1013F000F8430446164632D090F880302BB10025D1
:1014000010F0C6F82846BDE8F8830D4610F0C0F885
:101410000746052D41D0DFF8F0804FF0010998F81C
:10142000123053BBD8F8001004F1700394F86F2009
:1014300011F8030BC0F38010F9F7FAFD3378054675
:10144000FF2B3ED018B363885907DBD4AFBB637C56
:101450003BB34B4525D000252846BDE8F88310F066
:1014600097F8638807469B07F5D5DFF89C804FF017
:10147000020998F81230002BD4D0FBF7ADFCFF28FE
:101480003070CFD0FBF7B4FC0743FFB2CAE7E57E6C
:10149000ED1AB5FA85F56D09D5E76388DA07BAD490
:1014A000D9E7D8F8001011F8030BC0F38010FBF750
:1014B000B3FB0446FBF7D2FDE0B901252846BDE8A1
:1014C000F8830028BFD0D8F8001011F8030BC0F340
:1014D0008010FBF7A1FB0646FBF7C0FD0028B2D049
:1014E0003046FBF731FC0028ADD01021FBF7FEFFA2
:1014F0000546A8E72046FBF727FC0028DDD0102191
:10150000BDE8F843FBF7F2BF140E002138B5B0F880
:10151000483004462B4D0133AA7CA0F84830B2B9BC
:1015200000232B7194F881305BB9637B1BB1B4F855
:1015300048209A4212D220460021BDE8384002F0ED
:10154000C1BC20460121BDE8384002F0BBBC10F010
:1015500007FA0FF0A9FB0023AB74E1E70121204655
:1015600002F0B0FC6388DB070FD5236A1D880FF0FB
:10157000FBFA68B921784322637BA4F8BC5084F855
:10158000BB1084F8BA2093B10FE00FF0EDFA00B170
:1015900038BD20784FF6FF714322637B84F8BB008F
:1015A000A4F8BC1084F8BA200BB194F8483004F1C8
:1015B000B00084F8BE3016220349BDE83840FEF77B
:1015C000C1B800BF140E00213111010160B951B141
:1015D000074A084B92F804C0D2E90A1063440A692A
:1015E00052F8233018477047014BD86AFFF78EBF77
:1015F000140E0021FCFFFF3F2DE9F041394D84B06E
:10160000FF2604462B680DF107028DF807600521BF
:10161000D3F8030013F8038B029020469B88ADF8A3
:101620000C30FFF7E3FE002855D062792046216A8E
:101630000027FFF7E9FB216A84F88F704FF6FF70EF
:101640000B889DF80720A4F8AE002046A4F890303F
:1016500084F8AD60FFF7B8FC206A012221460388B8
:10166000A4F8CA3090F8CD3084F8CC3002F0EEFB0C
:10167000286808210780FCF79BFF39462868FDF79A
:101680006FF93A4628684FF00301FDF771F93A46C1
:10169000062304F169012868FDF75EF894F86810E4
:1016A0002868FCF7C3FFC8F380112868FCF7CCFF5B
:1016B0000623012202A92868FDF74EF86179304619
:1016C0000FF01AFE286810F0A3F8092301202B71EF
:1016D00004B0BDE8F0812046FFF718FF012004B0F8
:1016E000BDE8F081140E0021F0B5554C85B00646DA
:1016F0002379022B03D02379032B40F09480E56AF1
:101700002B7B002B38D12F6A0FB197F873708EB9ED
:10171000A37C1BB110F024F90FF0C6FAE06A02F0C6
:10172000EBF978B30FF04AFFA36A9B6805B0BDE8F8
:10173000F0401847216805F1690395F8682011F811
:10174000096BF009F9F774FC0028E1D006F00F06E8
:101750002068052E2CD03946FCF7A2FF0028D7D0F0
:101760002379E06A022B13D02379032B10D040F6A3
:1017700006512D20F7F76EFEFCF710FB85F84700A9
:10178000E56AC0E7E06A05B0BDE8F040FFF7BEBE1D
:10179000A36A314625795A692A4B2B4452F82330E3
:1017A0009847A37C002B43D10028B7D105B0F0BDEA
:1017B00090F8243003F01F03102BCCD9E56AEB7BA3
:1017C000002BC8D0FF230DF10F02314628468DF8BB
:1017D0000F30FFF70BFE00289AD095F8E830002B69
:1017E00096D1226805F1E901D31C2332D3F800C059
:1017F000103353F80C7C103153F8086C53F8040C78
:10180000934241F810CC41F80C7C41F8086C41F847
:10181000040CEBD11B88252205F1E0000B800A495E
:10182000FDF790FF74E740F62D512D20F7F712FEDB
:10183000019010F095F80FF037FA0198B4E700BF67
:10184000140E0021FEFFFF3F290801012DE9F041A0
:1018500004460E46002940F08A80724D0023286815
:1018600094F8767003806388103B0D2B00F2CA80D9
:10187000DFE803F078C8731EC807C8C8C8C8C8C85E
:10188000C8070121FCF794FE2868037823F02003A1
:1018900043F020030370002F00F0978004F17701DC
:1018A000FCF7BCFE28680121FCF7CEFE286809E0A1
:1018B0000021FCF77DFE2868037823F0200343F025
:1018C0002003037004F16901FCF798FE94F8681096
:1018D0002868FCF7ABFE638823F008039BB2152B46
:1018E00061D128680FF094FF04232B71FEB1638847
:1018F000102B75D004F13007D5F80C80384601F074
:10190000ABF806463846013E01F07EF82822618891
:10191000301AC0B201F0E0F8638880441B0764D439
:1019200022794146002010F0F5F8002874D0638831
:10193000103B0D2B6BD8DFE803F00E6A07076A0730
:101940006A6A6A6A6A6A6A07227901210020BDE828
:10195000F04110F025B8BDE8F0810621FCF728FE23
:101960002868AFE70221FCF723FE2868AAE700F108
:101970003007384601F048F8E0B963881A073CD5CB
:10198000384601F069F80546384601F03DF8281A56
:10199000244DC0B201F09AF8AB6803443846AB60FE
:1019A00000F0BCFF07E094F85420216D2868FCF794
:1019B00057FE96E71B4D384600F0B6FF0FF0F8FDD6
:1019C000217925200FF098FC48E704F17001FCF71D
:1019D00025FE286894F86F10FCF736FE286871E73A
:1019E0002179002010F0EAFBA1E7AB68984401F0F0
:1019F00045F84044C4F8200192E72046BDE8F04194
:101A0000FFF784BD40F272612D20F7F723FD40F609
:101A1000BC512D20F7F71EFD40F6A8512D20F7F7F9
:101A200019FD00BF140E002138B54388102B20D0BB
:101A3000124D0446AB7C63B928680FF0E9FE61885B
:101A400011F004010BD000200FF042FF02232B7194
:101A500038BD0FF00DF940200FF076FFECE7084697
:101A600022790FF09DFF00200FF032FF02232B712F
:101A700038BD0121BDE83840FFF7E8BE140E002153
:101A80000121FFF7E3BE00BF024B0121D86AFFF737
:101A9000DDBE00BF140E002170B50C4E337963B962
:101AA00003780546FF2B08D0FFF76CFB044610B9FE
:101AB0003379012B04D1204670BD0C24204670BD23
:101AC00001462846FFF7C2FE204670BD140E0021D5
:101AD0000121FFF7BBBE00BF70B5194CE56A2B7B37
:101AE00023BBA37CEBB9E06A02F006F8A0B1E06A80
:101AF000438803F0180383B12379022B02D02379A2
:101B0000032B18D12179A26A0E4BD2680B44BDE891
:101B1000704052F823301847E06ABDE87040FFF784
:101B2000F5BC0FF01DFF0FF0BFF8DCE7FCF736F94E
:101B300085F84700D5E740F637412D20F7F78AFCB6
:101B4000140E0021FEFFFF3F38B5214C2379002BF6
:101B500038D02379E56A022B1ED02379032B1BD0C2
:101B600015F072F81B4B1B788BB1284601F0C4FFAF
:101B700068B1E46A63881B071ED404F1300000F0EA
:101B800043FFC8B92046BDE83840FFF7BFBC284630
:101B9000BDE83840FFF7BABC2B7BA3B9A37C002B70
:101BA000DED00FF0DDFE0FF07FF815F04DF8094B99
:101BB0001B78002BD9D1EAE720460121BDE8384047
:101BC000FFF744BE38BDFCF7E9F885F84700E5E7C4
:101BD000140E00212100002130B50546086883B0AD
:101BE000002853D00C4600F037FF94F80CE0627BDD
:101BF000BEF1040F39D0284B042A284933F81E308F
:101C000003F2E73321D0A1FB0313BEF1080F4FEA23
:101C1000931C00F1FF334FEAC31323D0BEF1020F30
:101C200014BFF0216021634401FB0031A3882846E2
:101C300000930023FEF744FEA36800F593708342EF
:101C400034BF0020012003B030BDA1FB0323BEF14F
:101C5000080F4FF008024FEA931C00F1FF334FEAE0
:101C6000C313DBD14FF4D261DDE7042A00F1FF3367
:101C700005D0DB014FF02C0C4FF4D261D3E74FF0CD
:101C80002C0CDB0108224FF4D261CCE740F20C416E
:101C90002D20F7F7DFFB00BF44510301D34D621045
:101CA0002DE9F84390F880302BB100260FF070FC3E
:101CB0003046BDE8F883044603F0FF060FF068FCE9
:101CC0000746638813F00108F2D0784DAB7C002BF7
:101CD00040F09580296804F1700394F86F2011F8A2
:101CE000030BC0F38010F9F7A3F9002840F0C0807F
:101CF00063885B07DCD44FF0FF097FB9637C012B5D
:101D0000D6D8296811F8030BC0F38010FAF784FFC6
:101D10000746FBF7A3F9002840F09D802968644B33
:101D200011F8030B95F82020C0F38010F9F780F923
:101D300007460028BCD1216A20462B68FF261A7866
:101D400091F8CD3003EA5213012203F0010381F828
:101D5000CD30FFF759F8216A4FF6FF7084F88F7085
:101D60000B884A4684F8AD60A4F89030A4F8AE0021
:101D70002046FFF729F911224E4904F18600FDF7AC
:101D8000E1FC236A4C4904F1C0001A88A4F8CA2077
:101D9000052293F8CD3084F8CC30FDF7D3FC236ACC
:101DA0001E880EF0E1FE88B92278637BA4F8BC603F
:101DB00084F8BA0084F8BB20002B49D116223F4991
:101DC00004F1B00084F8BE30FDF7BCFC00222146CF
:101DD000206A46462A7102F039F82B683046226A9A
:101DE000D3F80310C2F80310B3F80710A2F80710D5
:101DF0001B78226AC3F380139370BDE8F883FAF767
:101E0000EBFFFF2881463FF465AFFAF7F1FF296841
:101E1000074304F1700311F8030B94F86F20FFB22D
:101E2000C0F38010F9F704F920B1638858073FF533
:101E300075AF62E7E07EA0EB0900B0FA80F04009E0
:101E400063885A077FF559AF00283FF431AF65E743
:101E500094F84830B2E73846FAF776FF00283FF4A6
:101E60005DAF1021FBF742FB00283FF421AF55E79F
:101E7000296811F8030BC0F38010FAF7CDFE8146F4
:101E8000FBF7ECF830B963884FF0FF0959073FF5CD
:101E900045AF32E74846FAF757FF0028F3D0102144
:101EA0004FF0FF09FBF722FBCAE700BF140E002129
:101EB000350E0021550F0101010801013111010109
:101EC0000329F8B509D0052921D1534B1B6803B369
:101ED000984780F00100C0B2F8BD04460FF058FBEF
:101EE000054663889E0712D54C4EB37C9BB931687A
:101EF00004F1700394F86F2011F8030BC0F3801005
:101F0000F9F796F800286DD163885B073CD501206E
:101F1000F8BD1846F8BDFAF75FFFFF280746E6D080
:101F2000FAF766FF3168054304F1700311F8030BFB
:101F300094F86F20EDB2C0F38010F9F779F800281B
:101F400040D06388580720D5237B002B45D13068CB
:101F5000002504210580FCF72BFB04F169013068A2
:101F6000FCF74CFB94F868103068FCF75FFB94F8C2
:101F70005C20A16D3068FCF783FB0523306833716A
:101F80000FF046FC2846F8BDFF27002DDCD1637C0E
:101F900013F0FD0FBBD1316811F8030BC0F38010B3
:101FA000FAF73AFE0546FBF759F80028CCD0284648
:101FB000FAF7CAFE0028C7D01021FBF797FA0028CD
:101FC000A5D0C1E7E07EC01BB0FA80F0400963886D
:101FD0005A07DAD500289AD0B6E739462046FEF7E8
:101FE0006FFFB4E7316811F8030BC0F38010FAF704
:101FF00013FE0746FBF732F820B96388FF2759071D
:10200000A2D4C2E73846FAF79FFE0028F5D0102187
:10201000FF27FBF76BFADAE798000021140E002186
:1020200008B590F88E3033B990F8C8301BB990F8E5
:10203000B80010B908BD012008BD0EF095FD80F074
:102040000100C0B208BD00BF094810B5037913B143
:102050000C24204610BD03F0FF0424220430214646
:1020600014F0DCFC0FF07CFC0EF01EFE204610BDD0
:10207000140E0021002310B50D4C2371237920602C
:1020800023B140F22D312D20F7F7E4F903F0FF01E1
:102090002422201D14F0C2FC0FF062FC0EF004FE9E
:1020A000A36A03B110BD4FF44C712D20F7F7D2F99C
:1020B000140E002130B54FF4B07285B00D460021EA
:1020C000044614F0ABFC7F23FF21132284F8473031
:1020D00042F210732170E3846280F8F775FC0022ED
:1020E0000146E064684618F014F800220121E06C13
:1020F00018F00DF90422E16C684618F00AF8002285
:10210000E06C114618F003F904F13000257400F07A
:10211000E3FB02A8FBF768FE30B102A904F1360028
:10212000FBF788FE05B030BD40F24A312D20F7F7AD
:1021300091F900BFFF23C86C0B7017F0DEBF00BF22
:10214000014B024A9A627047140E00217C00002164
:1021500003490448044B054A08601A60704700BFF1
:1021600098000021A11C010194000021F915010132
:102170000078FF3818BF0120704700BFF0B5044653
:1021800083B030300E4600F067FC6588E90611D454
:10219000AA0721794CBFB4F85C70B4F85470FEF70C
:1021A00061FB62790146334638460095FEF788FBAD
:1021B00003B0F0BD2822294603B0BDE8F04000F08E
:1021C00061BC00BF438813F0180F01D00120704795
:1021D00030B585B08468828800F1300508466946CC
:1021E0000095ADF804300294ADF80C20FFF7F4FC34
:1021F00005B030BD80687047407C003818BF0120B2
:10220000704700BF10B5837C04469A1E012A08D986
:1022100013F0FD0003D1BDE81040F8F733BF607E36
:1022200010BD00F1700190F86F00FAF7F5FC082876
:1022300001D0012010BDA37CEAE700BFF8B5837C84
:10224000044613F0FD0546D100F1690184F8685099
:102250002846F8F7D1FE002800F08580A37C0821ED
:1022600094F86820023BE176DBB2012B8CBF0021A1
:102270000121012AA17645D0012B25774BD9FAF708
:10228000C5FC064611F08EFC00257301F20E9B1B67
:1022900062F10002520242EAD3525B029B1942F100
:1022A000000C9A014FEA8C1ED21A4EEA936E6EEB26
:1022B0000C0E93194EF100021B18204642EB01024E
:1022C0002946C4E91832FEF7F3FE638884F8765095
:1022D0005B0728D4F8BD0121427E80F86810002AEF
:1022E00046D0023B0822D0F81300DBB2E276B4F805
:1022F0001710012BC4F86900A4F86D108CBF0022E0
:102300000122A27694F86E50012B6FEA0505C5F301
:10231000C0152577B3D804F1700194F86F00FAF76F
:102320007BFCE076ABE7E07EFAF70EFD0546002881
:10233000D0D01021FBF7DAF80028CBD1012604F128
:1023400077070246284684F8766039460B4CF8F742
:10235000DBFE39462068FCF761F931462068BDE8AC
:10236000F840FCF771B940F2B9412D20F7F772F847
:1023700040F2BD412D20F7F76DF800BF140E00218B
:102380000B680122C0F813308B884276A0F8173012
:10239000704700BF2DE9F04F844699B00C4690F885
:1023A000058090F80EA005460DAF07AEBCE80F0003
:1023B0000FC7BCE80F000FC79CE8070087E80700BD
:1023C000304600F089FA237D2278013B617894F849
:1023D0000AB0DBB20392022B00F2D9806E4A01F000
:1023E0007F07C906134493F8149008D4A37D013BDA
:1023F000DBB2022B00F2CB80134493F81480BAF1C5
:10240000010F09D1B9F1080F08BF4FF00409B8F165
:10241000080F08BF4FF00408617A304600F064FAF4
:10242000237D022B71D00121A27E30460132D2B22F
:1024300000F05CFA3A076CD50023227E0293A2F1E9
:102440000103E86CB3FA83F35B090593A37C04935F
:1024500018F0FCF88246E86C18F005F9029B50452C
:1024600038BF504680B200283BD1049AAC46ADF844
:1024700036700DAF8DF845204FF0000E039A0F9384
:10248000059B8DF846B08DF834208DF838908DF886
:1024900039808DF840300FCFACE80F000FCFACE89B
:1024A0000F0097E807008CE8070096E8030095F80E
:1024B00046302863A986E27A12F0FD0F14BF01228C
:1024C000724685F86F20E2682A67228AA5F8742090
:1024D000E27D62F3071385F84630704619B0BDE817
:1024E000F08F17F0180F0996ADF828700B938DF840
:1024F00030908DF83180B8D109A9FFF76DFB029BB0
:102500000028B2D14FF0450EE7E7617D0131C9B235
:102510008AE7304600F0A0FA63788246DB0626D5CB
:102520002822394600F0AEFA00F2EF221B4821794A
:10253000A0FB0232E37843EA01236179520A43EABD
:10254000014340F2712101FB02F201FB03F39A42C5
:102550007FF673AFE079A37943EA0023207A43EA58
:10256000004301FB03F3934228BF134665E7F8F7E6
:1025700073FA0346504649469A46FEF773F901231B
:102580000146424650460097FEF79AF9CCE740F2E2
:10259000EA210620F6F75EFF445103015917B7D12F
:1025A000438813F0100005D013F0040F14BF00206F
:1025B0001F2070479A0702D4DB0701D5EE20704731
:1025C000F8F74ABA08B5438813F0100004D083F036
:1025D0000403C3F3800008BD9A07FCD413F0010084
:1025E000F9D1F8F739FA003818BF012008BD00BF4B
:1025F000438800221D2BA0F8482008BF11464173D4
:10260000704700BF007B704790F91000704700BF13
:10261000408800F0010070474088C0F340007047D8
:102620004088C0F3401070474088C0F3C000704736
:102630004388DA0610B509D483F00203C3F34004DB
:10264000C06C17F0ACFF2043C0B210BD0124F7E707
:102650004088C0F3001070474088A0F10900B0FA2C
:1026600080F04009704700BF40797047024B9A6A7A
:10267000D8621368184700BF140E002190F8683024
:1026800001624B72D0F86930C1F80A30B0F86D3091
:10269000CB81704738B52F4C2379012B01D0002016
:1026A00038BDB0F848300546A27C0133A0F8483068
:1026B000002A36D10023237195F8813063BB6B7BF0
:1026C0001BB1B5F848209A4204D20021284601F0F7
:1026D000F9FBE4E70121284601F0F4FB6B88DB07F6
:1026E00026D52B6A1C880EF03FFA0028D7D129780E
:1026F00043226B7BA5F8BC4085F8BB1085F8BA2057
:102700000BB195F848301622134905F1B00085F851
:10271000BE30FDF717F8C2E70121284601F0D2FBD1
:10272000BDE70FF01DF90EF0BFFA0023A374C1E757
:102730000EF01AFA0028B2D128784FF6FF71432222
:102740006B7B85F8BB00A5F8BC1085F8BA20002B80
:10275000D9D0D6E7140E00213111010138B5B0F8F7
:10276000483004462B4D0133AA7CA0F84830B2B95A
:1027700000232B7194F881305BB9637B1BB1B4F8F3
:1027800048209A4212D220460021BDE8384001F08C
:1027900099BB20460121BDE8384001F093BB0FF002
:1027A000DFF80EF081FA0023AB74E1E70121204647
:1027B00001F088FB6388DB070FD5236A1D880EF0C4
:1027C000D3F968B921784322637BA4F8BC5084F81C
:1027D000BB1084F8BA2093B10FE00EF0C5F900B138
:1027E00038BD20784FF6FF714322637B84F8BB002D
:1027F000A4F8BC1084F8BA200BB194F8483004F166
:10280000B00084F8BE3016220349BDE83840FCF71A
:1028100099BF00BF140E00213111010138B5438862
:1028200004461A0730D4DB071AD5236A1D880EF038
:102830009BF988B921783C22637BA4F8BC5084F8CA
:10284000BB1084F8BA20E3B916221A4904F1B0008B
:1028500084F8BE30FCF776FF012384F8813038BD60
:102860000EF082F90028F7D120784FF6FF713C2254
:10287000637B84F8BB00A4F8BC1084F8BA20002B5A
:10288000E2D094F84830DFE7016A3C204FF6FF734E
:10289000FF2284F88F00088884F8AD201122A4F864
:1028A000900004F18600A4F8AE300349FCF74AFF1B
:1028B0006388B8E731110101550F010180F88010DC
:1028C000704700BFFF2380F88430704780F82410E1
:1028D00080F82520704700BF002240F20113C0F8A5
:1028E00002200380704700BF8170704708B590F8E0
:1028F00002C00170CCF380034270CCF340000CF0B6
:10290000010C0344634403FB01F101FB02F2FE2AC4
:1029100000DC08BD5C212E20F6F79CFD00234371EE
:10292000A0F80330704700BF08B582780346D1078E
:102930000DD5C07810F0010C09D1597993F801E058
:102940000131C9B28E45597142D0252008BD90078A
:1029500003D5D97811F0020C23D0510713D459793B
:1029600058780131C9B28842597108D1D87800210C
:102970009042597103D11A79D97001321A713921F3
:102980002E20F6F767FDD97811F0040CE7D15879BD
:1029900093F801E00130C0B28645587126D0272057
:1029A00008BD587993F801E00130C0B286455871EE
:1029B00001D0262008BD41F0020183F805C08A42FB
:1029C000D970F6D11A7983F803C001321A71F0E791
:1029D00040F0010083F805C08242D870B5D11A7961
:1029E000252083F803C001321A7108BD41F00401AB
:1029F00083F805C08A42D970D1D11A7983F803C00F
:102A000001321A71CBE700BF00B5837890F801C09E
:102A1000C3F3400EC3F3800103F00103C278714495
:102A200090F804E019440378A3EB0E0390F805E056
:102A300003FB0CF0C2F3800301FB00F0C2F3400182
:102A400002F001020B44A0EB0E00134403FB1C0038
:102A5000C0B25DF804FB00BF827890F801C0C2F3F9
:102A60004001C2F38003007802F001020B440CFB2A
:102A700000F0134403FB00F0C0B2704740F2EF20B7
:102A8000704700BF0138022808B519D8132907D8A4
:102A900011290CD810290FD10B4B33F8100008BDA9
:102AA000152909D1084B03EB4000008908BD064BEE
:102AB00003EB4000008A08BDD8212F20F6F7CAFC9E
:102AC000CA212F20F6F7C6FC5C51030140F25A33AD
:102AD00003FB00F0704700BF08B5431EDBB2012BBB
:102AE00001D91D2924D110390D291CD8DFE801F0A6
:102AF0000C1B07071B161B1B1B1B1B1B1B110E4A4A
:102B000002EB4303188C08BD0B4A02EB4303188BFE
:102B100008BD40F25A3303FB00F008BD064A02EB41
:102B20004303988B08BD4FF481712F20F6F792FC78
:102B3000EE212F20F6F78EFC5C51030140F28B3121
:102B4000062008B5F6F786FCF0B583B0002800F043
:102B5000D6800446082900F2C680DFE801F0879499
:102B6000525282C47C49C0008B250123002104F508
:102B70009876A4F8385184F83B31304684F8301107
:102B8000FAF76AFEB4F84831082B00F2A18001334D
:102B9000D4F814219BB2A4F8483112B1092B00F0EB
:102BA0009C80022294F8583184F83A2103F0FF0106
:102BB000F3B96FF00043D4E954029A4208BFB0F170
:102BC000FF3F79D02046D4E95057FFF7D7FAD4F821
:102BD000503100F24710D4F854215B1B62EB07021E
:102BE0001B1A62F10002002A66DA2046FFF716FE81
:102BF00094F8100110F0B0FF002384F8283103B0DE
:102C0000F0BDFFF725FD0028AED02046FFF700FD00
:102C100000286CD089277F250DF1060014F088FD6F
:102C20000DF107009DF9066014F088FD9DF807304E
:102C30001E4376B2002E18BF3D4614F035F800282A
:102C400093D01835ADB290E70321E81A12F04CF892
:102C5000C4F8345130B3204603B0BDE8F040FFF76C
:102C60007DBD03B0BDE8F0400FF092B8FFF7FEFC69
:102C7000002848D1D4F83401A0F59B7003B0BDE81A
:102C8000F04011F013BFFFF7CFFC014650B92046CA
:102C9000FFF774FAD4F8343100F247159D42D3D8C7
:102CA000C4F834512046FFF7F5FC0028A7D040F2C5
:102CB000A9213020F6F7CEFB314694F8100111F02F
:102CC000ADF800289BD140F28E613020F6F7C2FBB0
:102CD000D4F81431002B3FF464AF012262E7EB21FA
:102CE0003020F6F7B7FBEF213020F6F7B3FB204694
:102CF000FFF792FC00288DD17F2775258CE7CB212B
:102D00003020F6F7A7FB40F275213020F6F7A2FB42
:102D10002DE9F04F044689B00020174600930E4677
:102D200094F86F300590039318F01FFE94F8F82282
:102D30000B2A00F27D83AF4B94F8C61033F8125083
:102D400087F0010201912844029285B22FB3B4F8B2
:102D500080A304F55678B4F8BC90A6EB0A0AA6EB5B
:102D600009090FFA8AFA0FFA89F9BAF1000FC0F2CD
:102D7000CF81A14ADDF800B0127802F0FF07002AE7
:102D800040F0D78194F83C33032B00F25883DFE8FE
:102D900013F03701FC0097002F0094F83C23032A1E
:102DA000D5D10E29D3D1B4F8D423B242CFD1B4F8BF
:102DB00082232046B4F816130A44C4F83823D4F802
:102DC0004423C4F830236269C4F8342303F000FEBE
:102DD000D4F8D8236262B4F8D6232285D4F8DC2351
:102DE0006261D4F8E023E261022284F83C23AEE77A
:102DF0006569009B05FB0AF2002B40F00C8294F8F9
:102E00005333002B00F0B6827B4B5868D4F8443320
:102E1000D71BEB1A0597A3F5E375D4F878338542F1
:102E200028BF0546DF19D4F87C3304F13000C4F81C
:102E3000105343F10003C4F86873C4F86C330023E3
:102E400084F858338323A4F86033FCF715FD054458
:102E5000A4F88063C4F85C53D4E9DA23C4E9DE2320
:102E600003F0A0FD20B1D4F85C331E33C4F85C330A
:102E7000B4F8001300238E1B84F8623336B29E42EE
:102E800002DD022384F86233019A0E2A009A00F0D0
:102E90003582002A40F0358294F83C33002B40F014
:102EA0005782414694F8840310F0B8FF002800F0E0
:102EB000BA82029B002084F8503309B0BDE8F08F3D
:102EC000636A2946D4F83403184413F003F92946F9
:102ED000C4F84003606913F0FDF841F64B53626992
:102EE00094F86F909A42454D98BF0230C4F844035D
:102EF00048460EF0D1FD4DF6417219F00C0F4FF41B
:102F0000A87102442046A5FB023214BF28230023E7
:102F100003EB9212C432FCF76DFEB4F816331BB902
:102F2000009B002B40F02B82D4F83433626AD4F833
:102F3000405313445B1B0593D4F83033D4F8382343
:102F400094F86FA002FB0355238D1AF00C0F05F1C6
:102F5000300503EB450540F058814AF2A13950464F
:102F60000EF09AFD254B8144A3FB09394FEA9919CC
:102F70004D4450460EF088FD1F4B2844059A656964
:102F80005860012384F83C3340E7D4F84423636954
:102F9000D4F838139B1AB4F816530AFB03F3A94468
:102FA000D4F840530593CB43303594F86FA099443F
:102FB000D4F830331AF00C0F03FB015502FB09590A
:102FC000258D05EB490540F01D814AF2A139504697
:102FD0000EF062FD094B8144A3FB09394FEA9919B0
:102FE0004D4450460EF050FD034B2844059A58605E
:102FF00065690BE780510301440E0021D34D621037
:1030000094F86F104AF2A13B94F80F03FAF7F4FD1D
:103010008146606A2946DFF82CA3484413F05AF829
:103020002946C4F84003606913F054F8626941F618
:103030004B5307A99A4298BF0230C4F8440306A82C
:103040000EF01AFDDDE90623D4E9DE0112F0C0F826
:1030500094F86F300546184603930EF01DFD039B50
:103060004DF641724FF4A87113F00C0F0244204644
:10307000AAFB023214BF2823002303EB9212C432AE
:10308000FCF7B8FDD4F88833626A94F86F000593B2
:1030900003920EF001FD5844039AAAFB0031059BF0
:1030A000A3F12000D4F840331044C01A4844B4F8C7
:1030B0002890401B03F1300594F86F3009F1220984
:1030C000A0EB911013F00C0F4FEA4505059040F06E
:1030D0009F80184603930EF0DFFC8344AAFB0B3A53
:1030E000039B4FEA9A1A4D4418460EF0CDFC964BBE
:1030F0005544059A28445860D4F88833D31AB3F558
:103100000A7FBFF475AF40F2DC413020F6F7A2F938
:103110000022CA464FF0010B84F853238A4AD4E9AF
:10312000DC011278C4E9DE0102F0FF07002A3FF457
:1031300029AE13F089F8074600283FF423AEB4F80F
:103140002823012A40F2CB8094F83C23022A00F085
:10315000C68094F85223002A40F0C180606941F68D
:103160004B57B84240F23E8194F8F8220B2A00F205
:103170005F81764B33F8125094F83C3305F5C865FF
:10318000012BADB240F0308194F8C930032B40F0F0
:103190003F81D4F83403676A0744294612F09AFF46
:1031A000D4F8303302463846D4F838732946D31A57
:1031B000C4F8302303FB07F712F08CFFD4F8403338
:1031C0002946C4F84003C31A60691F4412F082FF05
:1031D000636941F64B529342B4F81633D4F838235E
:1031E0004B4498BF0230D243A3EB0A031344D4F8F4
:1031F0004423C4F84403801A00FB0377012384F8B6
:103200005233BFE54FF06509EAE64FF06509AFE6D6
:103210004FF0650A67E7B4F81633002B7FF4EFAD83
:1032200084F85333D4F8441301FB1A2A94F8C520C8
:10323000262ACDF814A054D094F8C620262A50D0BF
:10324000BBF1000F27D033BBD4F88CB3BBF1000F18
:1032500000F0F08094F86F0010F00C0F40F0C08088
:103260000EF01AFC4AF2A133364D0344D4F88CB365
:1032700094F86F00A5FB0335AD091035AAF1100ACB
:103280000EF002FCB4F816330AEB0B02D4F8441328
:10329000551B2D1A059503EB090B039801FB0BFB3E
:1032A00010F00C0F0BF1300B4FEA4B0B65D14AF2CB
:1032B000A1350EF0F1FB234B0544A3FB0535AD0909
:1032C00003980EF0E1FB05441F4B05EB0B0065690D
:1032D000586041F64B539D4275D9059A96E50027F3
:1032E00050E5B4F8D423B21A1204A9D4039894F880
:1032F000D723002A18BF10460390A1E7002A3FF405
:10330000D0ADB4F82823CAB1B4F82A0394F82C132A
:1033100000FB011101308A427FF7C3AD002B3FF45F
:10332000C0AD0023A4F82A0384F86233FCF712FE30
:1033300000F00700013084F82C03B2E5A4F82A233A
:10334000AFE500BFD34D6210440E00218051030150
:10335000D4F8443340466169C91AFAF77DFA83B25A
:10336000002B3FF49EAD129A0120002A3FF4A5AD38
:103370001380A2E5B4F8163354E76525A0E7D4F826
:103380003433626A94F86FB003EB020A58460EF0C9
:1033900083FBAAF12003D4F88C2381465846D4F845
:1033A00040B303EB020A0EF06FFB4AF2A132AAEB24
:1033B0000B034A441B1AA5FB0225A3EB9513D4F873
:1033C00040530593B8E5284605AB1F4A5946FAF71E
:1033D000BDFC1E4B84F85303059A5868656915E5D2
:1033E00075254BE71746CDE4294612F073FE636955
:1033F000BB42B4F81673D4F8443398BF02304F443C
:10340000C4F84403A7EB0A07C01A00FB07F7F5E668
:10341000676A94F86F1094F80F03FAF7EDFB07440E
:10342000D4F83403B9E640F28C513020F6F712F8A4
:10343000FFF784FB40F22E513020F6F70BF840F2F4
:1034400043513020F6F706F8480E0021440E0021C3
:103450002DE9F04700260546012782B080F8186163
:103460008A46D0F814013946D5E9508980F80F23EF
:1034700085F8286185F82971F9F7CEFED5F8144151
:10348000324631462046C4E9DC8995F81031C4F84B
:1034900088A384F88433334684F83C63A4F88063BB
:1034A000C4E9DE890096FFF733FCC8B984F83C73A1
:1034B000C4F83803C4F83003A4F84E03A4F84C034E
:1034C000B4F8BC3084F85103013BA4F88203A4F89B
:1034D000BC300EF015F902B0BDE8F04710F028B985
:1034E00040F219213020F5F7B5FF00BF70B584B068
:1034F000002800F040810446082900F22881DFE816
:1035000011F08A00DB00090009006C00260171003F
:103510007900220110F046FBD4E9DC23801A61EB2C
:103520000301012871F10003C0F237816FF001023D
:10353000002382428B41C0F22B8163690BB1B0FB47
:10354000F3F394F8C6200E2A00F0F480B4F8BC20FF
:10355000B4F84E1313449BB2C81A00044CBF591C54
:10356000013194F8513389B2A4F84E1323B9B4F859
:1035700004338B4200F0F280B4F8F830B4F8F6501F
:10358000013BB4F882035B1B01301344A4F88203AF
:103590009EB2731A1A0400F1AA800DF10E050023E1
:1035A000204600951A46FFF7B3FB002840F08980BB
:1035B000636F73B3B4F8F220B4F84E339B1A1BB2A6
:1035C000002B26DDB4F878100B44013BB3FBF1F37C
:1035D00003FB0123A4F8F2301BE004B0BDE8704007
:1035E0000EF0D6BB012010F079F804B0BDE87040B1
:1035F000F8F70EBB90F83C33042B40F0C580002355
:1036000094F8840384F83C3310F0A6FA202384F85D
:10361000843304B070BD002290F85033C0F88C237E
:10362000002B76D0B0F84E33B0F8BC20934200F0B7
:103630009A809A1AA0F8BC30A0F806232046D4E954
:10364000DA23C4E9DC2303F063F810F07BFA94F882
:103650006F20D4F8443302F00C02216B03F2A11561
:10366000002A15BF282300234FF413724FF4097268
:1036700083282CBF2D18833520461D44FCF71CFAE7
:10368000034661692A4620461D46FCF715FA0346A3
:103690004449D4F85C239D420C7CA2F1B40028BFBD
:1036A0001D464861002C08BF2B46C1E9023504B015
:1036B000BDE8704011F0FAB904B0BDE8704003F005
:1036C00063B901285BD1B4F84E13B4F800238B1A08
:1036D00013F4004FBDF80E30194489B2A6EB010374
:1036E00023D11BB2A4F84E13002BBFF658AF94F8A9
:1036F000C93004F1DC000B222B49002B0CBF3E2308
:10370000082384F8E530FCF71DF8204603F052F951
:1037100075E7B0F84C33B0F8BC10B0F84C235B1A26
:10372000A0F8BC20A0F8063388E71B0413D4A4F843
:103730004E1334E7B4F84E13B4F8BC20013189B20B
:10374000A4F84E1318E7BF213020F5F783FEC321FC
:103750003020F5F77FFEB31A1146C2E7013189B276
:10376000A4F84E1308E7B0F80423D31AA0F8BC203D
:10377000A0F8063362E797213020F5F76BFE40F2A0
:1037800049613020F5F766FEB9213020F5F762FE79
:1037900040F20A613020F5F75DFE40F20961302009
:1037A000F5F758FE440E002165000101D0F8140120
:1037B000704700BF2DE9F043002385B002220126A7
:1037C000CDE900338DF806206846F6F7A9FD0446DA
:1037D00020BB009D95F82831002BF5D0012128460B
:1037E00085F85861FFF76AF895F82831002BEBD07F
:1037F00095F8100110F0CCFE95F8100111F096FB31
:1038000095F8100110F0A8F900283AD085F8284161
:103810006846F6F785FD04460028DAD0DFF87880A0
:10382000012600254FF6FF7788F8186019E0029B03
:10383000DBB193F83C23C2B11888B8421BD00121F8
:1038400016F0E8F9814608B390F8840311F06EFB96
:1038500099F8840389F83C4310F07EF9202389F815
:103860008433CDE902558DF80E6002A8F6F758FDB5
:1038700004460028DBD0002088F8180005B0BDE819
:10388000F08340F205213020F5F7E4FD4FF490710C
:103890003020F5F7DFFD00BF440E0021054B00226C
:1038A000012142F210701A74588319701A76FFF7CA
:1038B00081BF00BF440E002190F82831002B40F05A
:1038C000D9802DE9F041044682B00D460146714889
:1038D000164603F0FF0810F0F7F82028074638D006
:1038E0004146502204F5887013F098F8012384F8BB
:1038F0001071C4F8145184F8283135B1FCF742FB3B
:1039000000F00700013085F82C032046FEF7A0FEEA
:1039100018B32046FEF77CFE002800F0A1804FF08F
:1039200089087F250DF1060013F002FF0DF1070055
:103930009DF9067013F002FF9DF807301F437FB218
:10394000002F18BF454613F0AFF938B11835ADB2A6
:1039500004E00C2002B0BDE8F0818B254FF48173A8
:103960000027A4F83851A4F83A3184F8307112F0E5
:10397000CBFB054610F0E6F8B4F83831DF3583426A
:103980002CBFED182D182046ADB2FEF74DFE0028D5
:103990003FD017F0EAFF00F5CD6130464FF0010847
:1039A00089B212F097FB3044C4F8340110F0FAF8F1
:1039B0002818E78441F10001C4F8400184F8188117
:1039C0002046C4F84411FEF747FE00283ED0A6F278
:1039D000435641462046FEF7D1FB361AC4F81C6117
:1039E0004FF0FF326FF00043C4E9542304F598719F
:1039F00094F8100110F012FA002845D00025204656
:103A00002946A4F84851FEF759FF284602B0BDE800
:103A1000F08101462046FEF7B1FB1F4F00F2471030
:103A2000C4F83401788B08B1E08C28BB054410F051
:103A3000B9F82D1841F10001C4E95051002ECFD042
:103A4000751941F10001C4E95451CFE74046FFF731
:103A50003DF86FF4A3731E44361AC4F81C61BFE727
:103A60002046FEF7D9FD00287FF459AF4FF07F08BC
:103A7000752557E70C207047FCF784FA7B8BB0FB69
:103A8000F3F202FB1300D1E74FF4F4713020F5F7A5
:103A9000E1FC00BF492B0101440E002190F82831C0
:103AA0000BB900207047012110B5044680F8581169
:103AB000FEF704FF94F828310BB9002010BD94F8EC
:103AC000100110F065FD94F8100111F02FFA94F830
:103AD000100110F041F820B10023002084F82831B3
:103AE00010BD40F205213020F5F7B4FC014B1874ED
:103AF000704700BF440E002190F8582182B910B5DC
:103B000002F0FF0490F8182112B90122104610BDEE
:103B1000D0E947319942F9D9FEF780FE2246F5E710
:103B200000221046704700BF2DE9F041124D0746B4
:103B3000D5E902840DF0DAFB0646414620463246BE
:103B4000F9F7BEFEEB680446834205D06869C01AE7
:103B50002044686110F0AAFFA642EC6009D87A6997
:103B600041F64B539A4204D9287E80F00100BDE80B
:103B7000F0810020BDE8F081440E002140F26A216E
:103B800008B5FCF7DDF8B0F5296F28BF4FF42960C0
:103B900080B208BD90F80B33002B65D170B503F0EF
:103BA000FF0590F83C3384B00446032B01D004B0E9
:103BB00070BD0FF0F7FFD4E9DC23801A61EB03013D
:103BC000012871F10003F2DB6FF00103834275EB12
:103BD00001034CDB6369B4F8BC20002B45D0B0FB7B
:103BE000F3F080B20132B4F80433104480B2A4F888
:103BF0004C03B4F84C239B1A1BB2002BD7DD94F86E
:103C0000840310F0C5FC0028D1D0B4F8BC50FF23C9
:103C1000B4F8F810B4F8F6200D4484F85133B4F831
:103C20004C33013DAD1AADB2EB1A1A04BFD40DF1FD
:103C30000E06B4F84C1300230122204689B20096E8
:103C4000FFF766F80028B2D0012815D1B4F84C333C
:103C5000BDF80E2013449BB2A4F84C33B4F84C3397
:103C6000EB1A1B04E5D5A2E770471846BAE74FF4F4
:103C7000B8613020F5F7EEFB40F2F9513020F5F74E
:103C8000E9FB00BF2DE9F047044682B0052900F2A8
:103C9000D280DFE801F04C1603131C30042384F8B3
:103CA0003C330DF02DFD0FF043FD0023B4F8BC2094
:103CB000A4F88233A4F84E2384F8513302B0BDE84F
:103CC000F087032380F83C3302B0BDE8F0870DF0A5
:103CD00007FB054694F86F00C4F88C530DF0D4FE32
:103CE000574B2D1AD3E9022129441544C3E9025147
:103CF00002B0BDE8F08790F86F50524E28460DF0A4
:103D0000CBFE4DF64172034615F00C0F20464FF4E2
:103D1000A8711A4414BF28230023A6FB024203EB18
:103D20009212C43202B0BDE8F047FBF763BFD0F88F
:103D30008C339BB9424B1B7E03F0FF02002BADD1AD
:103D4000B4F80413012320460092FEF7E1FF002897
:103D5000A7D040F2B5613020F5F77CFB90F85233E4
:103D6000002BE7D090F83C33032BE3D190F86F9011
:103D700017F0FBFD94F8F8320B2B5AD8324AD4F8DE
:103D80008C5332F81330C61803F5C86348469FB207
:103D90000DF07AFE19F00C0FA5EB0008B6B24846FC
:103DA0003BD10DF079FEDFF89CA000F2E733D4F8A8
:103DB00010534846AAFB0323A8EB93180DF064FEAA
:103DC0002D1A48460DF068FE4AF2A1330344AAFBBF
:103DD00003239B09EB1AA3F160025B0806FB02F2C6
:103DE0002933B2FBF7F26032A3EB5201520841458E
:103DF0001CD81344434519D33146606912F06AF95F
:103E000041F64B5362699A424FF0000398BF02306B
:103E100084F85233C4F844038CE7D4F81053A8F163
:103E20003C080DF031FE65232D1AD3E717F06BFE29
:103E3000E2E7FEF783FE4FF4E8613020F5F70AFB76
:103E4000440E0021D34D621080510301012A70B548
:103E5000064609D0022A14460D461ED04AB140F249
:103E60006A713020F5F7F6FA0DF040FAC6F88803CB
:103E700070BD0DF03BFA224601462846FFF7E8FAEE
:103E800032460F4995F810010FF04AFE0028EFD195
:103E900040F253713020F5F7DDFAD0F88813012293
:103EA0002846FFF7D5FA3246054995F810010FF07C
:103EB00037FE0028DCD140F264713020F5F7CAFAF1
:103EC000ED340101F0B5044683B061B1012940F041
:103ED0008C80002380F818310DF012FC03B0BDE88F
:103EE000F0400FF025BCC58C002D76D12046D4E9DA
:103EF0005076FEF77FF9284400224FF48173C019F1
:103F000084F8302146F10006C4F84001A4F83A31A3
:103F10002046C4F84461FEF79BFBE8B12046FEF75B
:103F200077FB002851D089277F250DF1060013F07B
:103F3000FFFB0DF107009DF9066013F0FFFB9DF8F4
:103F400007301E4376B2002E18BF3D4612F0ACFE7D
:103F500018B11835ADB200E08B2594F85831A4F8AB
:103F6000385103F0FF017BB96FF00043D4E95402EC
:103F70009A4208BFB0F1FF3F10D104F5987194F850
:103F800010010FF04BFFA8B30023A4F848310DF047
:103F9000B7FB03B0BDE8F0400FF0CABB2046D4E940
:103FA0005056FEF7EBF8D4F8503100F24710D4F831
:103FB00054215B1B62EB06021B1A62F10002002A0D
:103FC000DBDA2046FEF72AFCDEE72046FEF724FB7C
:103FD0000028A8D17F277525A7E7FBF7BBFFE58C55
:103FE000B0FBF5F303FB150580E740F27A71302052
:103FF000F5F730FA40F2D4613020F5F72BFA00BF24
:1040000090F82801704700BF014B5883704700BFEC
:10401000440E0021436893F8C620132A04D11422C9
:10402000002083F8C6207047022070474268D2F80B
:10403000B43013F004000ED1084943F0040349687A
:1040400091F804C1A1F802010CF1010C81F804C13E
:10405000C2F8B43070470120704700BF600E0021E5
:10406000FCF75CB910B5012304464068194690F886
:10407000C720A830F9F768FB18B96368082283F8ED
:10408000C72010BDFCF72EBAFCF75AB9014B99684E
:10409000FCF7BCB8600E0021014B9968FCF770B8C2
:1040A000600E0021014B9968FCF79CB9600E00215D
:1040B000344A402838B5938943EA0003938155D0A8
:1040C00000F00303032B57D010F0020311D0C407F4
:1040D000116110D4CB78052B22D00B2B04D153685F
:1040E00093F8C610122928D0850601D50823137528
:1040F00038BDC407F8D591F803C09160BCF1060F34
:1041000026D0BCF10B0F05D1516891F8C6C0BCF1A7
:10411000130F16D0002BE7D01169CB78052BDCD11B
:10412000536893F8C6101729DED100240025012119
:10413000C3E94A4583F8CB10D6E7002183F8CB10BA
:10414000D2E7002481F8CA40012481F80641E1E762
:10415000516891F8C6C0BCF1190FDBD100240025CD
:10416000C1E94845012481F8CA40D3E704215068D9
:10417000BDE83840FFF786BD40F6B2613120F5F763
:1041800069F900BF600E002130B583B0044601A874
:10419000F6F7B2FE002800F0F980322200210198E3
:1041A00012F03CFC019D03212846FAF711FD01980D
:1041B0002146037823F010030370FAF735FD2A2C0B
:1041C00028D8012C32D9A31E282B2FD8DFE803F0E2
:1041D000152E961B1B152E912E1B577ABC2E2EAE1C
:1041E0001B1B39395D642E2E2EC08153762E712E05
:1041F000893333332E2E2E2EA400694A019B526838
:1042000092F850211A71F6F78FFE002800F0C38053
:1042100003B030BDFF2C09D1614B01985B6893F866
:10422000CF23D3F8D013FAF713FDECE740F6614142
:104230003120F5F70FF95A4A204601990BF0AEF8F4
:10424000E1E7574C01986368B3F85010FAF7AAFDFC
:1042500063680198B3F85211FAF7A8FD63680198F2
:10426000B3F84C10FAF7A6FD63680198B3F8501143
:10427000FAF7A4FDC7E7019817F013FCC3E7019B09
:10428000222248491A725960BDE7454A019B52688B
:10429000B2F866219A80B6E7414B5B6893F86421D7
:1042A000012A14BFB3F86A20B3F86621019B9A80F3
:1042B000A9E73B4901980AF0B9FEA4E7019817F075
:1042C000F8FBA0E7364A019B526892F84A211A711E
:1042D00099E7334B0198596801F27111FAF78EFD95
:1042E00091E72F4B0198596801F5AC710AF0D0FEA7
:1042F00089E701992A48FBF7F5FF84E7284C0198E4
:10430000616801F54871FAF737FD6168019801F5B8
:10431000A271FAF73DFD76E7214B0198596801F249
:10432000931201F27111FAF783FD6CE71C4C0198AE
:10433000636893F84B11FAF7D1FD6368019893F81D
:104340004A11FAF7CFFD5EE70198FBF7BDFF5AE788
:104350000023284601218DF80030FAF745FC104A69
:1043600028469DF800306946556803F020042A7CF1
:104370006B7C032A03F01F0308BF002243EA821369
:1043800023438DF80030FAF739FC3CE740F6B531AD
:104390003120F5F75FF840F665413120F5F75AF81E
:1043A000600E00210C59004B40F20121312008B56C
:1043B000F5F750F808B54168094B5A68D1F8B430A0
:1043C00023F00403C1F8B43092F80431013B5BB22E
:1043D000002B82F8043100DB08BDFFF7E5FF00BFCA
:1043E000600E0021426808B592F8C630192B0ED134
:1043F000094B596891F80431013B5BB2002B81F8FD
:10440000043106DB1D23002082F8C63008BD0220DF
:1044100008BDFFF7C9FF00BF600E002108B5436863
:1044200093F8C620172A03D11B2283F8C62008BDA3
:1044300040F628013120F5F70DF800BF08B54368B4
:1044400093F8C620302A05D0172A12D11B2283F8F0
:10445000C62008BD094A0021526883F8C61092F8A8
:104460000431013B5BB28B4282F80431F1DAFFF791
:104470009BFF40F63D013120F4F7ECFF600E002178
:1044800008B5436893F8C620172A03D1192283F888
:10449000C62008BD40F622013120F4F7DBFF00BF43
:1044A00008B5436893F8C620162A06D101211722C1
:1044B00083F8051183F8C62008BD40F61B013120A2
:1044C000F4F7C8FF08B5436893F8C620122A06D14E
:1044D0000121132283F8051183F8C62008BD40F698
:1044E00013013120F4F7B6FF08B54368184993F873
:1044F000C52008690A2A00791BD0D3F8B42012F02D
:10450000080C07D1FF281ED1322283F8CCC383F8D0
:10451000C52008BD496822F00802C3F8B42091F80C
:104520000431013B5BB2002B81F80431F1DAFFF773
:104530003BFF93F849218242DFD1002283F8C52056
:1045400083F8002108BD40F2EA713120F4F782FFC0
:10455000600E002140F66A41312008B5F4F77AFF79
:10456000426808B5D2F8B430D80610D5990615D4EB
:104570000D4923F010034968C2F8B43091F80431B2
:10458000013B5BB2002B81F8043105DB08BD40F62E
:1045900085013120F4F75EFFFFF706FF40F6860144
:1045A0003120F4F757FF00BF600E002108B54368C3
:1045B00093F8C620232A00D01AB9242283F8C620F3
:1045C00008BD40F697013120F4F744FF10B50446CA
:1045D00040680123002190F8C520A830F9F7B4F80D
:1045E00020B16368102283F8C52010BD40F6710128
:1045F0003120F4F72FFF00BF10B5044640680123B7
:10460000002190F8C520A830F9F79EF820B1636822
:104610001E2283F8C52010BD40F67E013120F4F73C
:1046200019FF00BF10B5044640680123002190F82F
:10463000C520A830F9F788F820B16368212283F8F3
:10464000C52010BD4FF409613120F4F703FF00BF0E
:10465000436810B593F8C6201D2A2BD1002193F88A
:104660000621044683F8051192B91988012083F8C0
:10467000E2220C22A3F8E41283F8E60203F5367076
:104680000F49FBF75FF86368002283F8C62010BD6E
:1046900018880D2283F8061183F8E212A3F8E402C9
:1046A00003F536700749FBF74DF86368002283F87D
:1046B000C62010BD40F64E013120F4F7CBFE00BFFE
:1046C0002D01010149010101F8B5044640680123AB
:1046D000002190F8C620A830F9F736F808B9012073
:1046E000F8BD6368324D93F87310A868FAF7D0FAF2
:1046F000002845D06668A868B6F8BC20B0F80D3030
:10470000D243A6F8D433134447F6FD729BB29342CA
:104710000AD9282306F1DC000B22264986F8E53069
:10472000FBF710F80020F8BDFAF7A2FAF9F79AFAA9
:104730006768AB680646C7F8DC0331461879F9F7B5
:10474000A3FAAB683146A7F8D603B3F8050067684B
:10475000F9F7C2FA03466668A868C7F8D833FAF7CB
:104760008BFAA6F8E003A8686568FAF78DFA636823
:1047700001460E220020A5F8E21383F8C620F8BDFA
:104780006268D2F8B43013F00804A8D143F00803EB
:10479000D5E90110C2F8B430C378204682F8483118
:1047A00091F80431A1F80241013381F80431F8BDD8
:1047B000600E002165000101F8B504464068012340
:1047C000002190F8C620A830F8F7BEFF08B90120F4
:1047D000F8BD144E6768B068FAF79CFA6568A7F8E8
:1047E000D403B5F8D433B5F8BC20013B9B1A47F687
:1047F000FD729BB293420AD9282305F1DC000B22FB
:10480000094985F8E530FAF79DFF0020F8BDB0684A
:1048100005F2D631FAF778FA63680B22002083F8A4
:10482000C620F8BD600E00216500010138B50123E6
:1048300004464068194690F8C720A830F8F784FF6E
:1048400050B9064B65689868FAF768FA072285F848
:10485000C800636883F8C720002038BD600E0021BF
:10486000104B1A7DB2B958B95B6841F64B52596981
:10487000914204D9B3F854101A8F91420ED970475F
:104880009A89120708D55B6893F8C700083818BFE3
:104890000120704700207047012070471846FFF73D
:1048A00043B900BF600E00214368D3F8B43013F061
:1048B000300F01D0012070472DE9F0433C4D83B00B
:1048C0000446A868FAF786FAE8B96268D2F8B43004
:1048D00013F0080413D143F00803D5E90110C2F81E
:1048E000B430C378204682F8483191F80431A1F8F9
:1048F0000241013381F8043103B0BDE8F0830120A7
:1049000003B0BDE8F083A8686668FAF75FFA074667
:10491000A868FAF757FA8046A8683036FAF758FAC6
:104920008146A868FAF750FA4B460090424639464D
:104930003046FAF7E7FFAB899B0721D4636893F809
:10494000C5201E2A21D093F86420012A05D093F8AF
:104950005B2112B993F85A21DAB1D3F8B42042F0AE
:104960001002C3F8B4206B68002193F804210846B4
